:020000040800F2
:1000000000500020496A0008155A0008195A0008D3
:1000100000000000000000000000000000000000E0
:10002000000000000000000000000000295A000845
:1000300000000000000000002B5A00082D5A0008A4
:10004000996A0008996A00083D5A0008996A0008F0
:10005000996A0008455A0008555A0008655A000870
:10006000996A0008996A0008996A0008996A000864
:10007000996A0008996A0008996A0008996A000854
:10008000996A0008996A0008996A0008000000004F
:10009000996A0008996A0008996A0008996A000834
:1000A000996A0008996A0008996A0008996A000824
:1000B000355A0008996A0008996A0008996A000888
:1000C000002934D00123002210B488422CD301240B
:1000D0002407A14204D2814202D209011B01F8E7A0
:1000E000E400A14204D2814202D249005B00F8E759
:1000F000884201D3401A1A434C08A04202D3001B85
:100100005C0822438C08A04202D3001B9C082243B7
:10011000CC08A04202D3001BDC082243002803D0F5
:100120001B0901D00909E3E7101C10BC704701B599
:10013000002000F05FF802BD0029F8D003B5FFF7FA
:10014000C1FF0EBC4243891A1847C046002941D05E
:1001500010B4041C4C40A44601230022002900D501
:100160004942002800D5404288422CD3012424076C
:10017000A14204D2814202D209011B01F8E7E40046
:10018000A14204D2814202D249005B00F8E78842D2
:1001900001D3401A1A434C08A04202D3001B5C084A
:1001A00022438C08A04202D3001B9C082243CC08A7
:1001B000A04202D3001BDC082243002803D01B0905
:1001C00001D00909E3E7101C6446002C00D5404229
:1001D00010BC704701B5002000F00CF802BDC0460D
:1001E0000029F7D003B5FFF7B3FF0EBC4243891ACD
:1001F0001847C0467047C0468446101C62468C466D
:10020000191C634600E0C0461FB50BF05DFD0028D9
:1002100001D40021C8421FBD10B50BF0BDFC404207
:10022000013010BD10B50BF04FFD002801DB0020A0
:1002300010BD012010BDC04610B50BF045FD0028D3
:1002400001DD002010BD012010BDC04610B50BF02F
:10025000DBFC002801DC002010BD012010BDC046E1
:1002600010B50BF0D1FC002801DA002010BD0120F0
:1002700010BDC046002B15D1002A13D1002906DB82
:1002800001DC002806D00020C043410802E08021A4
:100290000906002007B4024801A14018029003BDDE
:1002A00055FFFFFF03B4684601B502980AF0A9FDA7
:1002B000019B9E4602B00CBC7047C046002B11D17A
:1002C000002A0FD1002900D1002802D00021C94303
:1002D000081C07B4024802A14018029003BDC046A2
:1002E00015FFFFFF03B4684601B502980AF018FD38
:1002F000019B9E4602B00CBC7047C04602B47146DA
:1003000049084900095C49008E4402BC7047C04658
:1003100003B47146490840004900095A49008E4417
:1003200003BC7047D0400B1CD1409C46203AD340C0
:100330001843524263469340184370479140031C50
:1003400090409C46203A9340194352426346D34022
:10035000194370471C2101231B04984201D3000C50
:1003600010391B0A984201D3000A08391B09984228
:1003700001D30009043902A2105C40187047C0463E
:10038000040302020101010100000000000000005E
:1003900010B5002903D1FFF7DDFF203002E0081C73
:1003A000FFF7D8FF10BDC04610B5064C2378002BD0
:1003B00007D1054B002B02D0044800E000BF012309
:1003C000237010BD5C0A002000000000C0CA0008B5
:1003D000044B10B5002B03D00349044800E000BFD4
:1003E00010BDC04600000000600A0020C0CA00081E
:1003F000024A136810218B4313607047007000405D
:1004000070B503689B6A4B6003681B695B045B0CF7
:100410008B6003681C68144B1C40260C3F20304046
:100420000870230A7F252B404B702C408C703F3D79
:100430003540CD70002A15D10509AA005219550082
:100440000F221040401908701D09A80040194500EE
:1004500013405B194B70200983001B18580014408F
:1004600024188C70002070BD7F7F7F0070B50368FA
:100470005B68144803401C0CCC70180A1F252840E8
:10048000487020351D408D705B0B072633400B7084
:10049000002A15D1220993009B185A000F231C40F3
:1004A000A418CC700409A2001219540018400019B5
:1004B000487028098200121850001D402D188D70B8
:1004C000002070BD3FFFFF00F8B504002023C35C8F
:1004D000012B00D1EAE020230120E0540133013058
:1004E000E054002A71D123689B685B0601D4002385
:1004F000CB70CE690B78100002E001300A3BDBB212
:10050000092BFAD80001C0B2184300044B7815003B
:1005100002E001350A3BDBB2092BFAD82D01EDB21E
:100520002B431B0203438878150002E001350A388B
:10053000C0B20928FAD82D01EDB228431843CB7870
:100540001B0418432023CD5C02E001320A3DEDB2CA
:10055000092DFAD81201D3B22B431B0603431E43C5
:100560004B691E434D688B691D432368CA225A623A
:100570002368773A5A624A6A80235B009A423DD0E8
:10058000226893684A490B4093602168CA68FF2338
:100590001A40484B1343CB6001F060FE070022680D
:1005A000D1688B075FD401F059FEC01BFA239B0072
:1005B0009842F4D92368FF225A622123FC3AE2547C
:1005C000013B0022E25403206FE023689B685B0636
:1005D00001D40023CB700E7836044B781B021E43E7
:1005E0008B781E43CB781B041E432023CB5C1B0659
:1005F0001E43CB691E434B691E43B3E722689368D1
:100600002D490B4093602168CA68FF231A402B4B89
:100610001343CB6001F022FE07002368DA68D2079B
:1006200011D401F01BFEC01BFA239B009842F4D9A1
:100630002368FF225A622123FC3AE254013B002244
:10064000E254032031E0DE6123685D642268916832
:1006500080235B000B4393602268916880235B01D9
:100660000B4393600EE0166223689D6422689168D4
:1006700080239B000B4393602268916880239B0139
:100680000B4393600E4B196880229202114319604C
:1006900099680A439A602368FF225A622123FE3A2E
:1006A000E254013B0022E2540020F8BD0220FCE7A6
:1006B000FFFDFFFF7FFDFFFFFFFEFFFF7FFEFFFF50
:1006C0000004014070B504002023C35C012B60D0FE
:1006D00020230122C25401330132C2540368C832BC
:1006E0005A620368773A5A6280235B00994222D0AB
:1006F0000268936828490B40936002689368274911
:100700000B40936001F0AAFD05002368DB689B079E
:1007100034D401F0A3FD401BFA239B009842F4D986
:100720002368FF225A622123FC3AE254013B002253
:10073000E25403202CE00268936819490B4093604F
:100740000268936817490B40936001F087FD05002C
:100750002368DB68DB0711D401F080FD401BFA231E
:100760009B009842F4D92368FF225A622123FC3A65
:10077000E254013B0022E254032009E02368FF22F7
:100780005A622123FE3AE254013B0022E254002047
:1007900070BD0220FCE7C046FFFDFFFFFFDFFFFF4B
:1007A000FFFEFFFFFFEFFFFF70B504000268D36894
:1007B000A0218B43D36001F051FD05002368DB6865
:1007C0009B0608D401F04AFD401BFA239B00984287
:1007D000F4D9032000E0002070BD70B50400036868
:1007E000DA68520601D5002070BD01225242DA605B
:1007F00001F034FD05002368DB685B0608D401F0D6
:100800002DFD401BFA239B009842F4D90320EBE70F
:100810000020E9E770B5041E4ED02123C35C002BF5
:100820003CD021230222E2542368C8325A62236852
:10083000773A5A622000FFF7D0FF002834D12268AF
:1008400093681E490B40936021688A686368256934
:100850002B43A5692B4313438B602368E2681A611D
:1008600021680B69A268120413430B612268D368E4
:1008700080218B43D3602268D36C7D398B43D36452
:100880002168CB6CE26965692A431343CB64236812
:10089000FF225A622123FE3AE25470BD2033002227
:1008A000C25404F031FEBCE72368FF225A622123C0
:1008B000FB3AE2540120F0E70120EEE7BFFF8FFF93
:1008C000F8B505000E002023C35C012B00D18FE09A
:1008D00020230121C15401330131C154002A5AD1CE
:1008E00003689B685B0601D40023F370337814001F
:1008F00002E001340A3BDBB2092BFAD82401E4B24E
:1009000023431B047478110002E001310A3CE4B275
:10091000092CFAD80901C9B20C4324022343B47844
:1009200002E001320A3CE4B2092CFAD81201D2B238
:1009300014431C43F3781B041C432B68CA225A62DD
:100940002B68773A5A622800FFF747FF071E33D11A
:100950002B68284A14401C602A68936826490B407B
:10096000936029688B68F2683069024313438B6097
:100970002A68D36880218B43D3602B689B689B06D1
:1009800026D52B68FF225A622123FE3AEA54013B06
:100990000022EA541AE003689B685B0601D4002336
:1009A000F3703478240473781B021C43B3781C431F
:1009B000F3781B041C43C0E72B68FF225A622123F3
:1009C000FB3AEA54013B0022EA5401273800F8BD03
:1009D0002800FFF7E9FE0028D3D02B68FF225A62D7
:1009E0002123FB3AEA54013B0022EA540127EDE7B8
:1009F0000227EBE77F7F7F00FFFFFBFF70B505005D
:100A00002023C35C012B00D180E020230120E85487
:100A100001330130E854002A06D14B78D80603D5BB
:100A2000102083430A334B70002A48D1CB7814003E
:100A300002E001340A3BDBB2092BFAD82401E4B20C
:100A400023431B044C78100002E001300A3CE4B25E
:100A5000092CFAD80001C0B20443240223438C7845
:100A600002E001320A3CE4B2092CFAD81201D2B2F7
:100A700014431C430B785B031C432B68CA225A6245
:100A80002B68773A5A622800FFF7A7FE061E21D18D
:100A90002B681F4A14405C602A68D36880218B430E
:100AA000D3602B689B689B0620D52B68FF225A6277
:100AB0002123FE3AEA54013B0022EA5414E04B7829
:100AC0008A78CC7824041B021C4314430B785B0304
:100AD0001C43D2E72B68FF225A622123FB3AEA54D7
:100AE000013B0022EA540126300070BD2800FFF7C8
:100AF0005BFE0028D9D02B68FF225A622123FB3AE3
:100B0000EA54013B0022EA540126EDE70226EBE716
:100B10003FFFFF0070B5002811DB8408134DC0347F
:100B2000A400625903231840C000FC331E00864015
:100B3000B24389010B4083401343635170BDC0B27F
:100B40000F220240083A920806329200084BD3184E
:100B50005D6803242040C000FF2214008440A543A8
:100B600089010A4082402A435A60E7E700E100E039
:100B700000ED00E01F2318401E3B8340014A136034
:100B80007047C04600E100E01F2318401E3B834031
:100B90000249802252008B507047C04600E100E0BD
:100BA0001F2318401E3B83400249C02252008B5035
:100BB0007047C04600E100E0F0B5C64600B506004B
:100BC0000C0017001D0001F049FB8046002F31D0BA
:100BD00033689B682340A34262D16B1CF8D0002D80
:100BE00005D001F03BFB4346C01AA842F0D9326859
:100BF0005368E0218B43536032681368A0398B43FC
:100C0000136080239B01B26A9A423DD05123012296
:100C1000F254013B0022F254032032E032681368A0
:100C200020490B4013603268116880239B010B43FD
:100C300013601DE033689B682340A34220D06B1CE7
:100C4000F8D0002D05D001F009FB4346C01AA84298
:100C5000F0D932685368E0218B43536032681368DF
:100C6000A0398B43136080239B01B26A9A42D5D08E
:100C700051230122F254013B0022F254032000E0F0
:100C8000002004BC9046F0BD3268136805490B4053
:100C900013603268116880239B010B431360B5E732
:100CA0000020EEE7FFDFFFFF7047000010B5041ED5
:100CB0003CD05123C35C002B32D051220223A354D9
:100CC00021680B68402083430B606368A1680B4375
:100CD000E1680B4321690B4361690B438021890063
:100CE000A06901400B43E1690B43216A0B43216872
:100CF000A06A03430B60618B04230B402168606A88
:100D000003434B602368E16A19612168CB69084895
:100D10000340CB61002363650133A354002010BD61
:100D200050330022C254FFF7BFFFC6E70120F6E7A9
:100D3000FFF7FFFF30B583B0040068460025C5808B
:100D40005120205C012804D05120205C222800D0B2
:100D5000A8E1002900D1A8E1002A00D1A7E1002BD9
:100D600000D1A6E15020205C012800D1A3E1502051
:100D7000012525540130205C012868D000206065E1
:100D8000A263A387E3872163A386E386A064E0646C
:100D900080239B01A26A9A425DD023681A6852069A
:100DA00003D41A6840210A431A6080231B01E268B9
:100DB0009A425CD06368002B07D082225200934293
:100DC0000DD1E38E9BB2012B09D1236B5A1C2263F8
:100DD00022681B78D360E38E013B9BB2E386E38EEF
:100DE0009BB2002B00D0ECE080239B01A26A9A42C8
:100DF00000D1CCE0069B002201212000FFF7DCFEA1
:100E0000002800D061E12368DB68A26B1370E38FD8
:100E1000013B9BB2E38780239B01A26A9A4200D1E7
:100E20000DE1069B012280212000FFF7C5FE00286E
:100E300000D019E151230122E25480239B01A26AD0
:100E40009A4200D116E150230022E2542BE15030A7
:100E50003135255492E722681368A0490B4013608E
:100E60002268116880239B010B43136095E7636838
:100E7000002B07D08222520093420ED1E38E9BB208
:100E8000012B0AD12368226B1288DA60236B0233AC
:100E90002363E38E013B9BB2E386E38E9BB2002B80
:100EA00034D180239B01A26A9A4214D0069B00226F
:100EB00001212000FFF780FE002800D0FDE023681C
:100EC000DB68A26B1380A36B0233A363E38F013B48
:100ED0009BB2E3879FE72268116880235B010B4385
:100EE0001360E3E7069B002201212000FFF764FE68
:100EF000002800D0E5E02368DB68A26B1380A36BB9
:100F00000233A363E38F013B9BB2E387E38E9BB283
:100F1000002B23D0069B002202212000FFF74CFE6D
:100F2000002800D0CBE02368226B1288DA60236BA4
:100F300002332363E38E013B9BB2E386E38E9BB2D5
:100F4000002BCFD180239B01A26A9A42CAD122688A
:100F5000116880235B010B431360C3E76368002BB8
:100F600000D058E7069B002201212000FFF724FE55
:100F7000002800D0A7E02368DB68A26B1380A36B76
:100F80000233A363E38F013B9BB2E38743E722680D
:100F9000116880235B010B4313602BE7069B002243
:100FA00001212000FFF708FE002800D091E023680F
:100FB000DA68A36B591CA1631A70E38F013B9BB2E3
:100FC000E387E38E9BB2002B22D0069B00220221F6
:100FD0002000FFF7F1FD002800D078E0236B5A1CB9
:100FE000226322681B78D360E38E013B9BB2E386C9
:100FF000E38E9BB2002BD1D180239B01A26A9A423F
:10100000CCD12268116880235B010B431360C5E7D4
:101010006368002B00D0FEE6069B00220121200021
:10102000FFF7CAFD002856D12368DA68A36B591C64
:10103000A1631A70E38F013B9BB2E387EBE6069B4B
:10104000002201212000FFF7B7FD002806D1236808
:10105000DB689BB26A46D380D388E2E6636D0222E6
:101060001343636503201EE0636D20221343636511
:10107000032018E023689A68D20600D4E3E6626D84
:1010800002210A4362651A6814490A401A602268FC
:10109000116880239B010B43136050230022E2540C
:1010A000012000E0022003B030BD0120FBE7012059
:1010B000F9E70120F7E70220F5E70320F3E7032033
:1010C000F1E70320EFE70320EDE70320EBE7032040
:1010D000E9E70320E7E70320E5E7C046FFDFFFFF7E
:1010E000F0B5C64600B5002338E0052600E000262E
:1010F000AE4035003D430234A400584EA551584C33
:1011000025684246D4432E0026404A68D20302D5C1
:10111000424615432E00524D2E606D682E0026402B
:101120004A68920302D5424615432E004C4D6E602C
:10113000AD682E0026404A68D20202D542461543C9
:101140002E00474DAE60ED682C404A68920202D5F1
:1011500042462A431400424AD46001330A6814000C
:10116000DC4077D001249C4022409046F5D04D6869
:10117000022D01D0122D0ED1DD080835AD002F58FB
:1011800007261E40B6000F22B24097430A69B240BC
:1011900016003E432E504D686E1E012E03D9112DB0
:1011A00001D0122D12D185685F000326BE40B543E1
:1011B0002E00CD68BD40354385604568A5434A682B
:1011C0001609012434409C402C43446007685E00AB
:1011D00003242500B540ED432F404A681440B44035
:1011E0003C430460C46825408C68B4402C43C46010
:1011F0004A68D200B1D51B4D6C6B012634436C6339
:101200009C08A51CAD00154EAF5903261E40B50025
:101210000F26AE40B743A026F605B04200D166E7E0
:10122000114EB0420ED0114EB0420DD0104EB04211
:101230000CD0104EB0420BD00F4EB04200D154E74C
:10124000062655E7012653E7022651E703264FE716
:1012500004264DE704BC9046F0BDC04600000140A6
:10126000000401400010024000040050000800503B
:10127000000C005000100050001C0050002A01D14A
:10128000816270478161FCE710B5054B5B691842CC
:1012900000D110BD024B586104F070F9F9E7C04667
:1012A0000004014070B504000E00150003689B693E
:1012B000DB0616D523689A69920614D4731CF9D0FC
:1012C000002E04D000F0CAFF401BB042F2D94123E7
:1012D0002022E25400232232A354023AA3540320D2
:1012E00024E0002022E01022DA6123681032DA6163
:1012F00023689A69920701D500229A6223689A6945
:10130000D20703D49A6901210A439A61226853687B
:1013100007490B405360042363643D332022E254A9
:1013200000232232A354023AA354012070BDC046C8
:1013300000E800FEF8B506000C0017001D00336839
:101340009B6923401B1B5A425341BB4213D16B1C68
:10135000F5D0002D05D000F081FF069BC01AA842F1
:10136000EDD941232022F25400232232B354023A11
:10137000B354032000E00020F8BD70B505000C0058
:1013800016002B689B699B061AD4320021002800A6
:10139000FFF788FF002815D1002C04D000F05EFF75
:1013A000801BA042EDD96B6C202213436B64412358
:1013B000EA5400232232AB54023AAB54032070BDEE
:1013C0000020FCE70120FAE770B504000D001600CC
:1013D00023689B695B072DD4320029002000FFF7AA
:1013E00061FF002828D123689A69920611D4002D44
:1013F00004D000F033FF801BA842E9D9636C20229F
:10140000134363644123E254013B0022E25403206E
:1014100070BD2022DA6121684B68084803404B60A8
:1014200000236364412162542232A354023AA3543C
:101430000120EDE70020EBE70120E9E700E800FEEE
:1014400070B504000D00160023689B699B0724D427
:10145000320029002000FFF725FF002818D16B1C5F
:10146000F2D0002D04D000F0F9FE801BA842EBD989
:10147000636C2022134363644123E254002322322D
:10148000A354023AA354064803F0F2FC032005E0FB
:10149000044803F0EDFC012000E0002070BDC046D0
:1014A0001CCB0008D8CA000810B5041E59D041232F
:1014B000C35C002B43D041232422E25422681368EA
:1014C00001218B4313602268274B61680B40136135
:1014D0002268936825490B409360E368012B34D060
:1014E000226884231B02A1680B439360E368022BEC
:1014F00032D0226851681E4B0B4353602268D36878
:101500001A490B40D360236962691343A26912022E
:1015100021681343CB602268E369216A0B4313609F
:101520002268136801210B43136000236364412286
:101530001F31A15423630132A354002010BD403356
:101540000022C25404F0A0F8B5E7226880231B02F1
:10155000A1680B439360C9E72368802212015A6097
:10156000C7E70120EAE7C046FFFFFFF0FF7FFFFF6C
:1015700000800002F0B585B004000D001700039351
:101580004123C35C202B00D0BDE02033C35C012B82
:1015900000D1BBE040230122C25400F05FFE0600F0
:1015A00023689A6912040ED500F058FE801B192892
:1015B000F6D941232022E25400232232A354023AD6
:1015C000A3540320A0E041222121A154013211396A
:1015D000A1540022626467626946898961856263F9
:1015E000628D92B2FF2A0ED9FF2222855A684B499A
:1015F0000A40A805800DFF2109040843484901431A
:101600000A435A6026E0628D92B22285D2B25968AE
:1016100042480140A805800D12040243414802439C
:101620000A435A6016E0636C042B00D070E001207E
:101630006AE0638D9BB22385DBB2206842683A4939
:101640000A40A905890D1B040B43802189040B4323
:1016500013434360638D9BB2002B38D032000A994C
:101660002000FFF7EDFE0028DDD1636A5A1C62629C
:1016700022681B789362638D013B9BB26385238D47
:10168000013B9BB22385002BE4D1638D9BB2002BE1
:10169000E0D000960A9B002280212000FFF74AFE3E
:1016A000002837D1638D9BB2FF2BC2D9FF2323853E
:1016B000206843681C4A1340A905890DFF221204C3
:1016C0001143802252040A4313434360C2E73200AD
:1016D0000A992000FFF751FE002804D0636C042B08
:1016E0001AD1012010E023682022DA6121684B68BA
:1016F0000E4D2B404B604123E25400232232A35471
:10170000023AA35400E0022005B0F0BD0220FBE73E
:101710000320F9E70320F7E70320F5E7009800FC32
:101720000020008100200082009C00FC00E800FEF8
:10173000F0B585B004000D00170003934123C35C8E
:10174000202B00D0BDE02033C35C012B00D1BBE0D7
:1017500040230122C25400F081FD060023689A69EB
:1017600012040ED500F07AFD801B1928F6D941230A
:101770002022E25400232232A354023AA35403202D
:10178000A0E041222221A15401321239A1540022A9
:10179000626467626946898961856263628D92B21B
:1017A000FF2A0ED9FF2222855A684B490A40A80514
:1017B000800DFF2109040843484901430A435A6048
:1017C00026E0628D92B22285D2B259684248014029
:1017D000A805800D12040243414802430A435A609F
:1017E00016E0636C042B00D070E001206AE0638D8A
:1017F0009BB22385DBB2206842683A490A40A905BA
:10180000890D1B040B43802189040B431343436060
:10181000638D9BB2002B38D032000A992000FFF76D
:10182000D3FD0028DDD123685A6A636A591C6162BE
:101830001A70238D013B9BB22385628D013A92B2CF
:101840006285002BE4D1638D9BB2002BE0D0009623
:101850000A9B002280212000FFF76CFD002837D171
:10186000638D9BB2FF2BC2D9FF2323852068436879
:101870001C4A1340A905890DFF221204114380223E
:1018800052040A4313434360C2E732000A9920001E
:10189000FFF773FD002804D0636C042B1AD10120DC
:1018A00010E023682022DA6121684B680E4D2B403E
:1018B0004B604123E25400232232A354023AA35442
:1018C00000E0022005B0F0BD0220FBE70320F9E7AD
:1018D0000320F7E70320F5E7009800FC00240081CF
:1018E00000240082009C00FC00E800FE30B51B4B89
:1018F000DB68F022134022D1184A926BD2000ED539
:10190000174A1268C02149010A40C02149018A4290
:1019100016D1C0221202904212D1012310E00F49C9
:101920008C6B8022520522438A630D4A1268C024C0
:10193000640122408C6B0B4D2C408C63E5E7002347
:101940000948026801218A431A4302600268114073
:10195000994201D0012030BD0020FCE70010024078
:1019600000700040FFFFFFEF0020024070B582B022
:1019700004000368DB0741D5BB4BDA680C23134036
:10198000082B33D0B84BDA680C2313400C2B29D02A
:10199000636880225202934258D0A022D20293421E
:1019A0005BD0B14B1A68B1490A401A601A688021AD
:1019B00049020A400192019A1A68AD490A401A6028
:1019C0006368002B55D000F049FC0500A64B1B684E
:1019D0009B0313D400F042FC401BA64B9842F5D960
:1019E000032069E2A04BDB68DB03D1D59E4B1B686B
:1019F0009B0303D56368002B00D156E223689B0745
:101A00005BD5994BDA680C231340042B44D0964BDA
:101A1000DA680C2313400C2B3AD0E368002B00D17A
:101A2000AEE091490A680920824313430B6000F03D
:101A300015FC05008C4B1B685B0700D597E000F098
:101A40000DFC401B0228F5D9032035E2864A1168B7
:101A500080235B020B431360B2E7834B196880223B
:101A6000D2020A431A601968802252020A431A609D
:101A7000A6E700F0F3FB05007B4B1B689B03BDD57D
:101A800000F0ECFB401B7B4B9842F5D9032013E29E
:101A9000754BDB68DB03C0D4734B1B685B0704D555
:101AA000E368012B01D0012006E26F494B68724ABE
:101AB00013402269120213434B602368DB063BD5B7
:101AC000694BDB680C221A4200D080E0664B1B6831
:101AD0009B0503D5E369002B00D1E8E1606A624B06
:101AE0005B68E0221202134098425CD9FFF7FEFEC9
:101AF000002800D0DDE15C4A536860490B40616A10
:101B00000B43536053681B021B0A216A09060B43EF
:101B10005360636A5A0B013280231B029340524A7E
:101B2000D16809090F220A4055498A5CD340554AB9
:101B30001360032003F0C6FC23681B0700D4A5E054
:101B40006369002B7CD0484A136D01210B43136558
:101B500000F084FB0500444B1B6D9B0700D595E00E
:101B600000F07CFB401B0228F5D90320A4E13E498C
:101B70004B68414A13402269120213434B609CE7B1
:101B8000394A136801218B43136000F067FB05009D
:101B9000354B1B685B0790D500F060FB401B0228AB
:101BA000F6D9032088E1304A536834490B40184382
:101BB000506053681B021B0A216A09060B435360DD
:101BC000606AFFF793FE0028A3D0012074E1E36967
:101BD000002B22D0244A116880235B000B43136042
:101BE00000F03CFB0500204B1B689B0506D400F071
:101BF00035FB401B0228F6D903205DE11A4A5368E1
:101C00001E490B40616A0B43536053681B021B0A59
:101C1000216A09060B4353608EE7134A13681A4979
:101C20000B40136000F01AFB05000F4B1B689B056F
:101C300082D500F013FB401B0228F6D903203BE1BC
:101C4000094A136D01218B43136500F007FB050062
:101C5000054B1B6D9B0719D500F000FB401B0228AC
:101C6000F6D9032028E1C04600100240FFFFFEFF26
:101C7000FFFFFBFF88130000FFE0FFFFFF1FFFFFD8
:101C800090CD000830000020FFFEFFFF23685B07B7
:101C900078D58B4B9B6BDB001BD4894A916B8023DF
:101CA0005B050B4393630125864B1B68DB0512D54F
:101CB000A36880225200934221D0002B37D1804B61
:101CC0001A6D81490A401A651A6D80490A401A65E1
:101CD0001BE00025E8E77B4A116880235B000B438B
:101CE000136000F0BBFA0600764B1B68DB05DFD4FF
:101CF00000F0B4FA801B6428F6D90320DCE0704AB7
:101D0000116D80235B000B431365A368002B28D063
:101D100000F0A4FA06006A4B1B6D9B0530D400F05E
:101D20009DFA801B6A4B9842F5D90320C4E0A0229B
:101D3000D200934209D0624B1A6D63490A401A657A
:101D40001A6D62490A401A65DFE75D4B196D013A69
:101D5000FF3A0A431A65196D802252000A431A6538
:101D6000D3E700F07BFA0600554B1B6D9B0507D5AA
:101D700000F074FA801B564B9842F5D903209BE083
:101D8000012D21D023689B063CD5A369002B21D0CF
:101D90004B4B99680120014399605A6B02435A6387
:101DA0004C4A116A80239B010B43136200F056FAE0
:101DB0000500434B9B689B0724D400F04FFA401B5F
:101DC0000228F6D9032077E03D4A936B42490B4045
:101DD0009363D7E73A4A936801218B4393603D4A66
:101DE000136A3E490B40136200F038FA0500344B89
:101DF0009B689B0706D500F031FA401B0228F6D9F4
:101E0000032059E0A36A002B55D02D4AD1680C223B
:101E10000A400C2A52D0022B12D0294A13683049AA
:101E20000B40136000F01AFA0400254B1B689B015D
:101E300039D500F013FA001B0228F6D903203BE045
:101E40001F4A136826490B40136000F007FA05008B
:101E50001B4B1B689B0106D500F000FA401B0228B3
:101E6000F6D9032028E01649CB681E4A1340E26ADF
:101E7000206B0243606B02431343CB600A688023EC
:101E80005B0413430B6000F0E9F904000C4B1B6882
:101E90009B0106D400F0E2F9001B0228F6D90320CA
:101EA0000AE0002008E0002006E0012004E0012014
:101EB00002E0012000E0002002B070BD0120FBE73D
:101EC0000010024000700040FFFEFFFFFFFBFFFF1D
:101ED0008813000000000140FFFFFFEFFFDFFFFF5E
:101EE000FFFFFFFEFFFF02FF10B5264BD9680C2352
:101EF0000B40082B42D00C2B11D0042B09D0214BC6
:101F00005A68520B07231340013380200002984087
:101F100010BD1C4B1B68DB0632D51B48F8E78A0C4A
:101F20000F231340194AD05C890D0322114001315F
:101F3000144BDB68DB030DD4124B1B68DB0613D597
:101F40004201121A93019B1ADB001B181802FEF7BC
:101F5000B7F8DDE74201121A93019B1ADB001B1848
:101F60005802FEF7ADF8D3E74201121A93019B1A0B
:101F7000DB001B189802FEF7A3F8C9E70448C7E77F
:101F80000448C5E70010024000093D00A8CD000844
:101F900000127A000024F40070B504000D005F4BBD
:101FA0001A68012313408B420BD25C490B68012253
:101FB00093432B430B600B681A40AA4201D00120C7
:101FC00070BD23689B0706D5554AD368F0218B4323
:101FD000A1680B43D3602368DB0764D56368022BD9
:101FE00009D0032B29D0012B2DD04D4A1268920520
:101FF00006D40120E4E74A4A1268920300D48AE03A
:102000004749CA68032082431343CB6000F026F996
:1020100006006368022B1CD0032B28D0012B34D080
:102020003F4BDB680C221A423DD000F017F9801BB1
:102030003C4B9842F4D90320C2E7394A1268920116
:10204000DED40120BCE7364A12685207D8D40120FA
:10205000B6E7334BDA680C231340082B23D000F08B
:10206000FDF8801B2F4B9842F3D90320A8E72C4B97
:10207000DA680C2313400C2B15D000F0EFF8801B0E
:10208000284B9842F3D903209AE7254BDA680C23B2
:102090001340042B07D000F0E1F8801B214B98423D
:1020A000F3D903208CE71D4B1A6801231340AB4280
:1020B0000BD91A490B68012293432B430B600B6821
:1020C0001A40AA4201D001207AE723685B0706D5AF
:1020D000134AD36814490B40E1680B43D36023686B
:1020E0001B0707D50E49CB68104A13402269D2005E
:1020F0001343CB60FFF7F8FE094BDA6812090F2390
:1021000013400B4AD35CD8400A4B1860032003F0FD
:10211000D9F9002054E7012052E7C04600200240D0
:102120000010024088130000FFF8FFFFFFC7FFFF09
:1021300090CD000830000020054B1868054BDA6888
:10214000120A07231340044AD35CD8407047C046A4
:102150003000002000100240A0CD0008054B186898
:10216000054BDA68D20A07231340044AD35CD840EF
:102170007047C0463000002000100240A0CD00088B
:10218000F0B54123C35C202B20D12033C35C012B4D
:102190001ED04024012202554125242343550668C0
:1021A000336893433360066833680A4F3B403360BB
:1021B000066833681943316001680B6813430B608C
:1021C0002023435500230355002000E00220F0BDEA
:1021D0000220FCE7FFEFFFFFF0B54123C35C202B9B
:1021E0001ED12033C35C012B1CD040240122025598
:1021F00041252423435506683368934333600668BA
:102200003368094F3B4009021943316001680B688C
:1022100013430B602023435500230355002000E0A7
:102220000220F0BD0220FCE7FFF0FFFF10B5064AD8
:10223000136802210B431360032003F043F903F0FA
:102240004BF9002010BDC04600200240024A13682E
:10225000013313607047C046780A0020014B1868AC
:102260007047C046780A0020024A536801218B4318
:102270005360704700580140024A536802218B4363
:102280005360704700580140024A536804218B4351
:10229000536070470058014030B52023C35C012BC8
:1022A00017D020230124C454212102224254026861
:1022B000CA2555620268773D55620568AA681A43C7
:1022C000AA600268FF25556244540022C2540020CF
:1022D00030BD0220FCE70000F8B504000168836807
:1022E0000269134342691343C26913430A68BE4833
:1022F000024013430B6022685368BC490B40E168FD
:102300000B435360A1692268B94B9A4201D0236AFA
:1023100019439368B74803400B4393602368B64A58
:10232000934220D0B54A934231D0B54A934263D00C
:10233000B44A934262D0AE4A93423DD01025022067
:1023400000F006FC2668AA4B9E425BD080231B024D
:10235000E2699A4200D190E0082D00D966E1AD0013
:10236000A94B5B599F46A94BDA6C03231340012B01
:1023700009D0002B05D0022B3AD0032B05D0102515
:10238000DDE70125DBE70425D9E70825D7E79F4BE3
:10239000DA6C0C231340042B0AD005D9082B29D062
:1023A0000C2B07D10825CAE7002B03D10025C6E76F
:1023B0000425C4E71025C2E7944BDB6CC022120150
:1023C00013408022D20093420ED009D980221201FC
:1023D000934215D0C0221201934207D10825AEE7DF
:1023E000002B03D10025AAE70425A8E71025A6E7BE
:1023F0000225A4E70225A2E70025A0E700259EE725
:1024000002259CE7022D2DD007D9042D30D0082DB0
:1024100000D0DFE08020000207E0002D00D0D9E0EE
:10242000FFF78AFE002800D1D6E0626853009B18AF
:10243000834200D9D2E01303834200D2D0E0070EDA
:10244000060250080021801979410023FDF736FF6C
:102450006F4BC2186F4B9A4200D9C3E02368D86013
:10246000002022E0694B1B68DB0604D46A48DCE7E5
:10247000FFF73AFDD6E76948D7E7082D54D8AD00F5
:10248000674B5B599F46400063685B08C0186168F2
:10249000FDF716FE83B200200F22190091435B1056
:1024A000083A13400B432268D360F8BDFFF756FE8D
:1024B000400063685B08C0186168FDF701FE83B2E5
:1024C0000020E9E7514B1B68DB060AD56368580812
:1024D000544B9C4660446168FDF7F2FD83B20020D6
:1024E000DAE763685808504B9C4660446168FDF722
:1024F000E7FD83B20020CFE7FFF7F6FC40006368FA
:102500005B08C0186168FDF7DBFD83B20020C3E7FC
:102510006368580880235B029C4660446168FDF74D
:10252000CFFD83B20020B7E701200023B4E7FFF717
:1025300003FE63685B08C0186168FDF7C1FD23688E
:102540000004000CD8600020AFE7FFF707FE6368C7
:102550005B08C0186168FDF7B3FD23680004000C38
:10256000D8600020A1E7294B1B68DB060BD561680A
:1025700048082A4B9C466044FDF7A2FD0004000C6D
:10258000F060002091E761684808234B9C46604456
:10259000FDF796FD0004000CF060002085E7FFF7D2
:1025A000A3FC63685B08C0186168FDF789FD2368B8
:1025B0000004000CD860002077E761684808802399
:1025C0001B029C466044FDF77BFD0004000CF0609C
:1025D00000206AE7012068E7002066E7012064E741
:1025E000012062E7012060E7F369FFEFFFCFFFFF03
:1025F00000480040FFF4FFFF003801400044004065
:10260000004C00400050004048CB00080010024041
:1026100000FDFFFFFFFC0F000024F40000093D0057
:102620006CCB000800127A000048E80101203CE76A
:10263000436ADB0706D5026853682C490B40816A60
:102640000B435360436A9B0706D5026853682849C9
:102650000B40C16A0B435360436A5B0706D50268AF
:10266000536824490B40016B0B435360436A1B07BB
:1026700006D50268536820490B40416B0B435360F9
:10268000436ADB0606D5026893681C490B40816BE0
:102690000B439360436A9B0606D50268936818490A
:1026A0000B40C16B0B439360436A5B060BD502681A
:1026B000536814490B40016C0B43536080235B0348
:1026C000026C9A420AD0436A1B0606D50268536818
:1026D0000D490B40816C0B4353607047026853688F
:1026E0000A490B40416C0B435360ECE7FFFFFDFFD1
:1026F000FFFFFEFFFFFFFBFFFF7FFFFFFFEFFFFF7F
:10270000FFDFFFFFFFFFEFFFFFFFF7FFFFFF9FFF71
:10271000F0B5C64600B506000C0017009846069DA9
:102720003368DB6923401B1B5A425341BB421ED115
:102730006B1CF5D0002D05D0FFF790FD4346C01A65
:10274000A842EDD9326813680B490B401360326818
:102750009368A331FF318B43936020236922B354E4
:102760000132B35448330022F254032000E0002029
:1027700004BC9046F0BDC0465FFEFFFFF0B585B0DB
:1027800004000E0017001D006923C35C202B59D1E3
:1027900000295AD0002A5AD080235B0182689A42CD
:1027A00013D06823E35C012B53D068230122E25449
:1027B0000023E36669332032E254FFF74FFD0390B4
:1027C0005023E7520233E7520AE00369002BE8D1B5
:1027D000CB07E6D5012036E0327823689A620136CD
:1027E0005223E35A9BB2002B1CD05222A35A013B26
:1027F0009BB2A3520095039B002280212000FFF78B
:1028000087FF002827D180235B01A2689A42E3D189
:102810002369002BE0D133882268DB05DB0D93624E
:102820000236DDE70095039B002240212000FFF7E0
:102830006FFF002811D169232022E254013B0022BE
:10284000E25400E0022005B0F0BD0120FBE70120CA
:10285000F9E70220F7E70320F5E70320F3E700009C
:1028600030B583B004000023C366FFF7F7FC050012
:1028700023681B681B070ED423681B685B0717D4EB
:1028800020236922A3540132A35448330022E25486
:10289000002003B030BD80210C4B009303000022C8
:1028A00089032000FFF734FF0028E5D00320F0E77C
:1028B0008021064B00932B000022C9032000FFF764
:1028C00027FF0028DCD00320E3E7C046FFFFFF011D
:1028D00010B5041E30D06923C35C002B22D06923BD
:1028E0002422E2542268136801218B431360636A37
:1028F000002B1DD12000FFF7EFFC012811D022682A
:1029000053680E490B405360226893682A218B4319
:1029100093602268136829390B4313602000FFF786
:102920009FFF10BD68330022C25402F04BFBD6E774
:102930002000FFF77DFEDDE70120F2E7FFB7FFFF94
:1029400070B5040082231B0102681A425AD0754BED
:102950009B6BDB0000D59DE0724A916B80235B0589
:102960000B4393630125704B1B68DB0500D493E098
:102970006C4B1A68C0239B031A4061680B4093425A
:1029800000D19EE0C0239B020A001A409A4200D167
:102990009FE0644B1B6DC022920213401FD0114078
:1029A000994202D02268920608D4C0229202A168FD
:1029B0000A409A4213D023681B0510D5594B186D55
:1029C0005A4A02401E6D8021090331431965196D71
:1029D000574E314019651A65C30500D580E063681C
:1029E000C022920219001140914200D188E04D4965
:1029F0000B6DC02292026068024013430B65012DEB
:102A000000D187E02368DB0706D5464AD36C032153
:102A10008B43E1680B43D36423689B0706D5414A87
:102A2000D36C0C218B4321690B43D36423685B0770
:102A300006D53C4AD36C3F490B4061690B43D364D4
:102A400023681B0706D5374AD36C3B490B40A16965
:102A50000B43D3642368DB0506D5324AD36C334974
:102A60000B40E1690B43D36423685B0606D52D4A0E
:102A7000D36C32490B40616A0B43D36423681B0655
:102A80004ED5284AD36C2E490B40216A0B43D364A0
:102A9000002070BD002566E7234A116880235B0093
:102AA0000B431360FFF7DAFB06001F4B1B68DB05C7
:102AB00000D55DE7FFF7D2FB801B6428F5D9032022
:102AC000E7E7C0239B03A0680340934200D059E787
:102AD0005FE7144B1B689B0300D45AE70120D8E73B
:102AE000FFF7BCFB06000F4B1B6D9B0500D576E77F
:102AF000FFF7B4FB801B134B9842F4D90320C8E7BF
:102B000008490A6810480240C0208003034013436C
:102B10000B606CE70A008B6B0C490B40936371E709
:102B20000020B6E70010024000700040FFFFFCFFED
:102B3000FFFFF7FFFFF3FFFFFFCFFFFFFFFFFFFBED
:102B4000FFFFF3FF88130000FFFFCFFFFFFFFFEF42
:102B500010B5102800D120E12ED8022800D1CAE0FB
:102B600017D9042800D1E5E0082859D19E4BDB6C29
:102B7000C0229201134000D102E1802292019342CF
:102B800000D100E180225201934200D102E10020F5
:102B900047E0012844D1944BDA6C0323134000D161
:102BA00096E0022B00D196E0012B00D19AE0032B96
:102BB00000D19AE0002034E0402859D016D9802373
:102BC0005B00984228D1884BDB6CC02292021340F4
:102BD00000D1EBE080229202934200D1E9E0802212
:102BE0005202934200D1EBE000201AE0202817D1D6
:102BF0007D4B196D1B6DC022920213408022520240
:102C000093420FD080229202934210D0C0229202AF
:102C1000934210D0002004E080231B019842E7D0AB
:102C2000002010BD8A05EDD580200002F9E78A0753
:102C3000ECD56E48F5E76C4B1B689B0300D4C2E0F3
:102C4000694B1B68C0229203134080229203934277
:102C500000D1BAE0C0229203934205D080225203F1
:102C6000934203D06248DCE76248DAE76248D8E77B
:102C70005D4BDB6C8022D20413401FD15A4A12688C
:102C800092011BD5584BD868D968800C0F2202409E
:102C90005A48805C8A0D032111400131DB68DB0357
:102CA00007D4514B1B68DB0601D4554B02E0504B57
:102CB00000E0544B5843FDF703FAB2E7002B00D174
:102CC00085E0494B9B689B0700D582E00020A8E780
:102CD000FFF744FAA5E7444A1268520700D463E7B5
:102CE00047489EE7FFF700F99BE73F4B1B6D9B05AD
:102CF00071D4002095E73C4BDA6C0C23134007D0CD
:102D0000082B08D0042B0CD00C2B0DD0002088E70A
:102D1000FFF712FA85E7344A12685207F2D53848AD
:102D20007FE7FFF7E1F87CE72F4B1B6D9B0555D440
:102D3000002076E72C4BDB6CC022120113400DD033
:102D40008022120193420CD08022D20093420ED0F6
:102D5000C022120193420DD0002062E7FFF7ECF988
:102D60005FE7214A12685207EED5254859E7FFF779
:102D7000BBF856E71C4B1B6D9B0532D4002050E777
:102D8000FFF7DAF94DE7184A1268520700D4F9E65E
:102D90001B4846E7FFF7A8F843E7134B9B6B5B0222
:102DA00001D400203DE7FFF7C7F93AE7FFF7C4F980
:102DB00037E70D4A1268520700D410E7104830E791
:102DC000FFF792F82DE700202BE70F4829E70020B6
:102DD00027E70E4825E78020000222E78020000236
:102DE0001FE7802000021CE70010024088900000CE
:102DF00000093D0020A1070080841E00A8CD000826
:102E00000024F40000127A0040420F00006CDC0243
:102E1000034A11688023DB000B4313607047C046F0
:102E200000700040034A116880239B000B4313602D
:102E30007047C046007000400020704770477047E0
:102E4000032803D0034B00221A707047014B012264
:102E50001A70FAE7AC0B00200120704770B504002F
:102E6000092000F057F906005A2000F053F9050038
:102E700076B2631C11DB0E2C00DD0E247021314074
:102E8000013464B20F231C402143092000F0E2F812
:102E900029005A2000F0DEF870BD01246442EDE7FD
:102EA00010B586B01422002101A803F081FE11485C
:102EB00000F07EF8104B0293022303930133049336
:102EC0008021A02001AAC900C00502F001FC0B4C22
:102ED00001AA0821200002F0FBFB01AA202120000A
:102EE00002F0F6FB01AA1021200002F0F1FB06B06F
:102EF00010BDC0460000002000001110000400506A
:102F000010B586B01422002101A803F051FE0E4B2B
:102F10000293022303938021A02001AAC900C005C7
:102F200002F0D6FB094C01AA0821200002F0D0FBD8
:102F300001AA2021200002F0CBFB01AA10212000D1
:102F400002F0C6FB06B010BD0000111000040050D6
:102F500070B504008021A02023680022C900C005AC
:102F600002F006FC094D636800220821280002F0E7
:102F7000FFFBA36800222021280002F0F9FBE36890
:102F800000221021280002F0F3FB70BD0004005065
:102F9000064B5B79002B07D1044A3033D35C002BFE
:102FA00002D130330121D1547047C046AC0B002010
:102FB000014B18607047C0467C0A0020014B18790D
:102FC0007047C046AC0B002010B586B0142200211B
:102FD00001A803F0EDFD0123029302330493A02422
:102FE000E40501AA0121200002F072FB0122012167
:102FF000200002F013FC012001F0CCFD002302931D
:1030000001AA0121200002F063FB062001F0C2FDAD
:1030100006B010BD70B504000E001500002240215E
:103020000B4802F0FBFB802040422043C0B202F07C
:1030300077FC002404E0305D02F072FC0134E4B25D
:10304000AC42F8D301224021014802F0E7FB70BDF9
:103050000004005000B583B06B46D97107330122DC
:103060001900FFF7D7FF03B000BD000030B583B0F3
:103070000500154B98601549FDF722F80402134925
:103080002800FDF759F80802114B9C4660440F498F
:10309000FDF716F82418230C6A46D11D0B70012287
:1030A0000620FFF7B7FF230A6A46911D0B70012225
:1030B0000720FFF7AFFF6B46591D0C700122082057
:1030C000FFF7A8FF03B030BDAC0B0020093D0000A6
:1030D000841E000070B504000E001500002240217F
:1030E0000B4802F09BFB7F20204002F019FC0024DB
:1030F00005E0002002F014FC30550134E4B2AC428B
:10310000F7D301224021024802F088FB70BDC0467F
:103110000004005010B582B06B46DC1D0122210076
:10312000FFF7D8FF207802B010BD0000F0B587B0DF
:103130000C00002803D0012862D0002054E07F4E0C
:10314000358C04ABDF1D012239002720FFF7C2FFB9
:103150003878F82398430130281809F06BFB2223B4
:10316000F35C002B42D00022002307F0BFFF0600D3
:103170000F0004ABDD1D012229003020FFF7AAFF5C
:103180002B78F922934334D000226D4B3000390064
:1031900007F0ACFF06000F00200009F04BFB3200E7
:1031A0003B0007F0A3FF654A2423D35C002B23D107
:1031B0000022002307F09AFF0022624B08F0E6FD90
:1031C00004000D005D4BD86909F068FB02000B009C
:1031D0002000290008F062FA00225B4B08F0D6FDBF
:1031E00007F0FAFC07F080FD07B0F0BD0022544B59
:1031F000BBE700220023C9E700228023DB05D9E7D3
:103200004E4B5B6C012B00D182E0002B00D189E09A
:10321000022B00D181E00022002300920193474D50
:10322000AE6C0120B04009F005FB02000B000098D5
:10323000019908F033FA02000B000020404908F021
:103240002DFA009001914E23E85A09F0F3FA00227A
:103250003E4B07F04BFF009A019B08F097FD029050
:103260000391E400B000241A5223E85C0001001925
:10327000023BEB5C002B5AD01424001B1C3009F0DD
:103280000DFB04000D002D4A4C23D35C002B50D0C5
:103290000220301A800009F001FB02000B00200020
:1032A000290008F0FBF907F067FB04000D00234A32
:1032B0004D23D05C043009F0BDFA02000B00200061
:1032C000290008F063FD04000D0000220023FCF734
:1032D000BDFF00282FD000221A4B2000290007F044
:1032E00005FF009A019B08F051FD02000B000298B7
:1032F000039907F0FBFE0022134B08F047FD144A28
:10330000144B07F0F3FE07F0CBFB07F0EDFC6BE787
:103310000022114B0092019381E700220F4B009293
:1033200001937CE700220E4B0092019377E7002483
:10333000A3E70020ADE700200249D2E7AC0B002054
:103340000000F03F0000204000408F40000011408E
:103350002B8716D9CEF7EF3F80840E4180841E4123
:103360008084FE4010B582B0002804D001280FD020
:10337000012040420AE06B46DC1D012221001120A1
:10338000FFF7A8FE20784008404200B202B010BD0E
:103390006B46DC1D012221001B20FFF79BFE2078DD
:1033A0008B38F3E730B583B0051E1CD0114C236871
:1033B0001B690020984723685B69280098476B4683
:1033C000DC1D012221000120FFF784FE0020205691
:1033D0000723984328432070012221000120FFF792
:1033E00019FE03B030BD034B1B681B6901209847D1
:1033F000E5E7C0467C0A002010B5064801F084FCD1
:10340000054801F081FC0020FFF7CCFF034B0022B0
:103410001A7110BD980A0020140C0020AC0B00207B
:1034200010B5064801F070FC054801F06DFC012064
:10343000FFF7B8FF034B00221A7110BD980A002055
:10344000140C0020AC0B0020F0B585B00600804BBA
:103450005B79002B03D0012B59D000273EE07C4C38
:103460002623E75C0F256D44012229004020FFF749
:1034700031FE0022AA56032313400C2213436A464E
:10348000511D0B7001224020FFF7C4FD01222900CD
:103490004120FFF71FFE2A783F235B42134301A917
:1034A0000B7001224120FFF7B5FD012229003520D4
:1034B000FFF710FE2A783F2313403E22A3546B46A9
:1034C000D91C1E230B703D3A0D20FFF7A3FD0023EE
:1034D0003022A3540132A354A38763878022520071
:1034E00000215C4803F064FB594B01221A71002E45
:1034F00000D08FE0564B5B79002B00D193E0002F7A
:1035000000D0A0E00620FFF74DFF05B0F0BD504A07
:103510005523D35C002B48D00F246C44012221009A
:103520003320FFF7D7FD2378412213436A46D11D8C
:103530000B7001223320FFF76DFD6B46991D192397
:103540000B7001223B20FFF765FD414B56229F5C2B
:10355000033A9B5C002B44D00B2169441D230B7064
:10356000523A1120FFF756FD0F246C44012221002E
:103570004020FFF7AFFD2278332313400A2169442E
:103580000B7001224020FFF745FD0F216944002404
:103590000C7001220F20FFF73DFD0E2169440C70D5
:1035A00001220D20FFF736FD98E70F246C4401221D
:1035B00021003320FFF78EFD0023E3564122934381
:1035C00001221343092169440B7001223320FFF7C4
:1035D00021FD02A91D230B7001223B20FFF71AFDDC
:1035E000B3E70D2169441F230B7001221120FFF75F
:1035F00011FD0F246C44012221004020FFF76AFDD9
:1036000022783F23134003A90B7001224020FFF7CB
:1036100001FDBAE7104C3100200001F0B5FB20009D
:1036200001F0DAFA66E70520FFF7BCFE002F00D0B4
:103630006BE7074BD96A094C200001F0A5FB20007D
:1036400001F0CAFA61E70520FFF7ACFE5DE7C0466E
:10365000AC0B0020AC0A0020980A0020840A00204D
:1036600010B582B00100404801F08EFB3F4B5B7902
:10367000002B0CD0012B39D03C4B02221A713A4856
:1036800001F0AAFA0320FFF78DFE02B010BD6B46D1
:10369000DC1D012221004020FFF71CFD0022A25664
:1036A00003231340102213436A46D11C0B700122DE
:1036B0004020FFF7AFFC012221004120FFF70AFD67
:1036C00022783E2313406A46911C0B700122412050
:1036D000FFF7A0FC012221003520FFF7FBFC227838
:1036E0003F2313403E2221498B54C5E71F4A5323F1
:1036F000D35C002B1BD16B46D91DF7230B70012225
:103700001120FFF787FC6B469C1D01222100402001
:10371000FFF7E0FC0022A2563F2313404022134350
:103720002370012221004020FFF774FCA4E76B46C0
:10373000591DF5230B7001221120FFF76BFC6B461E
:10374000DC1D012221004020FFF7C4FC0022A2560C
:10375000332313404022134301A90B700122402060
:10376000FFF758FC88E7C046140C0020AC0B002083
:1037700030B583B0114B5B79012B1CD16B46D91D41
:10378000FA230B7001221120FFF744FC6B469C1DAD
:10379000012221004020FFF79DFC23780325AB4345
:1037A0002370012221004020FFF734FC034B1D71E0
:1037B0000720FFF7F7FD03B030BDC046AC0B00207B
:1037C00030B583B004006B46DD1D012229000120C5
:1037D000FFF780FC0023EB56002B2EDB2A4B002248
:1037E0005A71294B5B79A34225D0274B5C71012C80
:1037F00027D1FFF701FE6B46DC1D012221000120CD
:10380000FFF768FC227880235B4213432370012278
:1038100021000120FFF7FEFB6B46991D00240C7070
:1038200001224020FFF7F6FB6B46591D0C70012268
:103830004120FFF7EFFB03B030BD134B01225A715B
:10384000CFE7FFF7D9FD6B46DC1D012221000120E7
:10385000FFF740FC22787F23134001A90B7001225F
:103860000120FFF7D7FB6B46D91C00230B70012208
:103870004020FFF7CFFB6B46991C30230B700122D1
:103880004120FFF7C7FBD6E7AC0B002070B582B034
:103890001F4B18601F4C21001F4801F095F92100B3
:1038A0001E4801F091F921001D4801F08DF91D4CD1
:1038B00023681B6801209847FFF786FB0020FFF76D
:1038C00071FD23689B6818489847002410E0174D45
:1038D00066003619705DFFF773FFAD196878AB7835
:1038E0006A46D11D0B700122FFF794FB0134E4B24C
:1038F000102CECD90020FFF763FF0D4B00221A714A
:10390000084B1B685B689847023002B070BDC04628
:10391000800A0020794A0008140C0020980A002030
:10392000840A00207C0A002018000020A8CC00088F
:10393000AC0B0020F8B504000D0017001E00FFF7C7
:103940003FFF2800FFF792FB0520FFF72BFD01202A
:1039500001F020F901F02AFA0500280001F02CFA04
:10396000B04206D22000FFF7FDFCB842F5DD00248E
:1039700000E00124FFF740FD2000F8BD70B582B0E3
:103980000120FFF71DFF6B46991DFF230B700122DD
:103990001120FFF73FFB0520FFF704FD0026002460
:1039A00010E0012001F0F6F86B46DD1D0122290030
:1039B0002C20FFF78FFB2A7801231340A3401E43DE
:1039C0000134E4B21F2CECD9FFF716FD300002B031
:1039D00070BD0000F0B5DE4657464E464546E0B5A0
:1039E0008FB007000C001500009318AB04CB934672
:1039F0001B8899461AAB1B8804931BAB1B7898460F
:103A00001CAB1B789A461DAB1E781EAB1B78069329
:103A10001FAB1B78079320AB1B78029321AB1B785D
:103A20000593FFF7CDFE002F09D0012F00D1E6E06E
:103A30000FB03CBC90469946A246AB46F0BDE64F5F
:103A40007C61FD615B46BB6122234246FA5401332F
:103A50005246FA540133FE5401336A46127AFA543C
:103A600001336A46127DFA544B463B84280008F025
:103A700015FF0090019102000B000020D74907F0CC
:103A80000DFE0022D64B08F081F9029003910498B4
:103A900008F0D0FE029A039B08F078F90022D14B7F
:103AA00008F074F907F020F9F862009A019B0020F1
:103AB000CD4907F0F3FD07F017F985B22B0A08AAE4
:103AC000D11D0B7001220220FFF7A4FA08AB991D4B
:103AD0000D7001220320FFF79DFA002301E001335E
:103AE000DBB2142B16D8DA00C04812589442F6D331
:103AF0005A1CD20012589442F1D2DB00C3181B7931
:103B000008AA511D0B7001221220FFF783FA00232F
:103B1000584602E0FEE70133DBB2142B31D8D9005E
:103B2000B24C09598842F6D3591CC9000959884238
:103B3000F1D2DA00A3181B7909A90B700122132016
:103B4000FFF768FA4B461B0A08AAD11C0B7001222A
:103B50002520FFF75FFA08AB991C4B460B7001223A
:103B60002620FFF757FA4346002B0BD1092108AB5B
:103B70009C466144FF230B7001223220FFF74AFA72
:103B800007E0FEE70AA953460B7001223220FFF737
:103B900041FA172408AB9C466444012221003020DE
:103BA000FFF798FA0023E3566F2213404246002A9B
:103BB00022D00022134336011E430B2108AB9C4642
:103BC00061440E7001223020FFF724FA172408AB5D
:103BD0009C466444012221003120FFF77BFA2278C1
:103BE000402313430A2108AA944661440B70012222
:103BF0003120FFF70FFA1BE780225242DAE7764BBB
:103C00005C649D644D2269460978995401324946A5
:103C10009952023241469954013251469954013227
:103C20009E5401326946097E995401326946097FE2
:103C3000995401326946097A995401326946097DDD
:103C400099540C2D00D9BAE0052D00D8B9E0002C0C
:103C500004D12B000B3B012B00D8B7E0012C00D185
:103C6000B1E05D4A4C230021D154172708AB9C4694
:103C70006744012239001D20FFF72CFAA301DBB2B3
:103C8000009AD200D2B2134342469200D2B21343FA
:103C90007600F6B2334350494C228A5C13430CA998
:103CA0000B7001221D20FFF7B5F9012239001E20FB
:103CB000FFF710FA3A780C2313402A01D2B21343CB
:103CC000049C210A03220A4013430F2108AA9446A8
:103CD00061440B7001221E20FFF79CF90E2108ABF6
:103CE0009C4661440C7001221F20FFF793F94B465C
:103CF0001B0A0D2108AA944661440B700122202062
:103D0000FFF788F90BA94B460B7001222120FFF722
:103D100081F94346002B09D0112108AB9C46614430
:103D200053460B7001222220FFF774F92A4A5323CD
:103D3000D35C002B21D0172408AB9C46644401229D
:103D400021004B20FFF7C6F9227880235B42134302
:103D5000132108AA944661440B7001224B20FFF7FF
:103D600059F91D4A5423D35C122108AA9446614490
:103D70000B7001222420FFF74DF9062D38D11724AE
:103D800008AB9C466444012221003120FFF7A2F9D0
:103D90000023E3560722934305221343152108AA63
:103DA000944661440B7001223120FFF733F90DA9CD
:103DB0000C230B7001223720FFF72CF938E60C2575
:103DC00045E7062543E70C2D00D04AE7024A4C237D
:103DD0000121D15449E7C046AC0B00200000F03F60
:103DE0000000204000408F4080847E41F8CB0008D6
:103DF000172408AB9C466444012221003120FFF7C0
:103E000069F90023E35607229343032213432370E7
:103E1000012221003120FFF7FDF8162108AB9C4656
:103E200061440A230B7001223720FFF7F3F8FFE506
:103E3000F0B5DE4657464E464546E0B58BB0070026
:103E4000009102921C0014AB40CB1B78019316AB7F
:103E50001B88994617AB1B78984618AB1D7819AB91
:103E60001B789A461AAB1B7803931BAB1B789B46B7
:103E7000FFF7A6FCC54B1B68DB6800989847002F2E
:103E800009D0012F00D196E00BB03CBC904699467A
:103E9000A246AB46F0BDBE4B6A4612781A73029832
:103EA00018615C61DE614A461A84222241469954B7
:103EB00002329D540132594699541C9A9A6208F074
:103EC000EDFC0022B34B07F0E9FB06F00DFF84B2D6
:103ED000230A0B2104AA944661440B70012204209A
:103EE000FFF798F80A2104AB9C4661440C7001224C
:103EF0000520FFF78FF8300008F0D0FC02000B001F
:103F00000020A54907F0CAFB06F0EEFE84B2230AA2
:103F1000092104AA944661440B7001220220FFF794
:103F200079F806A90C7001220320FFF773F84B46BD
:103F30001B0A04AAD11D0B7001222520FFF76AF885
:103F400004AB991D4B460B7001222620FFF762F847
:103F5000172404AB9C466444012221003020FFF763
:103F6000B9F80022A2566F2313404246002A20D1FE
:103F70008022524213432D011D430D2104AB9C4668
:103F800061440D7001223020FFF744F8172404AB80
:103F90009C466444012221003120FFF79BF82378DE
:103FA0004022134307A90B7001223120FFF732F89A
:103FB0006AE70022DEE7764B402269460978995489
:103FC0005C649E640D326946097999540132494610
:103FD0009952023241469954033251469954013262
:103FE0006946097B9954023A9D54033259469954C3
:103FF0001C9A9A650C2E03D8052E02D8062600E0DE
:104000000C26002C03D133000B3B012B75D9012C5E
:1040100071D05F4A4C230021D1545346002B71D1FB
:10402000172704AB9C466744012239001D20FFF787
:1040300051F8A401E4B2019BDB00DBB21C43434610
:104040009B00DBB21C436D00EDB22543504A4C236C
:10405000D45C2543132104AB9C4661440D700122BE
:104060001D20FEF7D7FF012239001E20FFF732F88E
:104070003A780F2313403201D2B21343122104AA1B
:10408000944661440B7001221E20FEF7C3FF4B468D
:104090001B0A112104AA944661440B7001222020BE
:1040A000FEF7B8FF08A94B460B7001222120FEF74E
:1040B000B1FF062E49D0172404AB9C46644401226C
:1040C00021003120FFF706F80023E356072293432F
:1040D000032213432370012221003120FEF79AFFAF
:1040E000162104AB9C4661440A230B700122372041
:1040F000FEF790FFC8E60C2E8BD1254A4C230121F8
:10410000D1548AE7172704AB9C4667440122390043
:104110004B20FEF7DFFF3A7880235B4213430F21E9
:1041200004AA944661440B7001224B20FEF772FFF3
:10413000174A5423D35C0E2104AA944661440B70A1
:1041400001222420FEF766FF6AE7172404AB9C4691
:104150006444012221003120FEF7BCFF0023E35616
:104160000722934305221343152104AA9446614470
:104170000B7001223120FEF74DFF09A90C230B70B3
:1041800001223720FEF746FF7EE6C0467C0A00206B
:10419000AC0B002080844E4080847E4130B58DB0D1
:1041A0000C0053019B1A9B009A18D500FEF75EFF86
:1041B0000895002307930693059304930393052220
:1041C0000292019396235B010093002300222100B9
:1041D0000020FFF72DFE2F246C4401222100312006
:1041E000FEF778FF23784022934323703F3A210063
:1041F0003120FEF70FFF2E216944F0230B700122BE
:104200004020FEF707FF2D216944A0230B700122F7
:104210004120FEF7FFFE084C2900200000F0B4FD0D
:10422000064B02221A71200000F0D6FC0320FFF793
:10423000B9F80DB030BDC046140C0020AC0B002006
:1042400070B582B04D4B1B79012B04D0022B00D1ED
:104250006BE002B070BD494B5B79002B21D0012B84
:10426000F7D1464A5323D35C002BF2D06B46591D3D
:1042700002230B7001221220FEF7CCFE404B1B687C
:10428000002BE6D05C69002CE3D06B46DD1D0122DB
:1042900029001C20FEF71EFF2B783F201840A04766
:1042A000D7E7364B3022012199541B8E012BD0D1F8
:1042B000344800F029FD314D31230122EA546B4688
:1042C000DC1D21001120FEF705FF23785B085B420F
:1042D0003222AB54313A21001B20FEF7FBFE267838
:1042E0003602012221001C20FEF7F4FE2278324320
:1042F000130A5901C91A8801411AC900C918FF20B7
:10430000104043011B1A9A01D31ADB001B1880339B
:104310001B0ACB186B63012221000C20FEF7DAFE8A
:1043200023785B093822AB5493E7144B5B79012B5C
:1043300000D08EE7114A5233D35C002B00D188E7BE
:104340006B46991D02230B7001221220FEF762FEBC
:104350000B4B1B68002B00D17BE75C69002C00D164
:1043600077E76B46DD1D012229001C20FEF7B2FE17
:104370002B783F201840A0476BE7C046AC0B0020CD
:10438000800A0020840A002010B582B0194B5B79A6
:10439000012B2CD16B46DC1D012221001220FEF7DF
:1043A00099FE2378DB0711D56B46991D05230B7009
:1043B00001221220FEF72EFE0F4B1B68002B16D099
:1043C0009B69002B13D00120984710E06B46D91D44
:1043D00004230B7001221220FEF71CFE064B1B6803
:1043E000002B04D09B69002B01D00020984702B01D
:1043F00010BDC046AC0B0020800A002070B584B010
:1044000004006B46D971594B5B79002B03D0012B0B
:104410003CD0002025E0554B00229A876A4607329F
:1044200012785A8722215B5C002B1ED101226B4639
:10443000D91D0020FEF7EEFD6B46DA79531EDBB284
:104440003F2B19D849493F23CA54484D3F26AA5DFE
:1044500021000020FEF7DEFDAB5DAA8F9B18AB8725
:10446000A86AFFF7FDF804B070BD03A90A70012225
:104470003220FEF7CFFDDFE792B221003C4800F08A
:10448000A7FC3A4A3F232021D154DEE7374A55237F
:10449000D35C002B46D00F256D4401222900332028
:1044A000FEF718FE2B7841229343092169440B70D3
:1044B000403A3320FEF7AEFD02A919230B7001220A
:1044C0003B20FEF7A7FD6B4607331B782749642284
:1044D0008B540F2169440B70633A2220FEF79AFD3A
:1044E0000E21694400250D7001220E20FEF792FD79
:1044F0000D2169440D7001220D20FEF78BFD03ADE7
:10450000012229000120FEF7E5FD2B78F8229343D4
:1045100025D06B46DA7921000020FEF77BFD134B96
:10452000986D9EE70F256D44012229003320FEF788
:10453000D1FD0023EB5641229343012213430B216B
:1045400069440B7001223320FEF764FD0A2169449F
:104550001D230B7001223B20FEF75CFDB3E7FEF745
:104560005FFF012000F016FBD3E7C046AC0B002034
:10457000AC0A002070B584B00F236B4400221A707F
:10458000C94B1B79012B04D0022B00D16BE104B085
:1045900070BDC54B5B79002B33D0012BF7D10B21BC
:1045A000694440230B7001221220FEF733FD0E24D4
:1045B0006C44012221001220FEF78CFD22780F238B
:1045C0006B441A701B789B0600D4DFE003A92023FC
:1045D0000B7001221220FEF71DFDB34A5623D35C57
:1045E000002B02D1130000221A71B04800F08CFB9E
:1045F000AF4B1B68002BCAD01B69002BC7D0984754
:10460000C5E7A94A2423D35C002B1ED1A64B5A8FA1
:10461000002A76D19B8F002B73D1A34A2233D35C1F
:10462000002B63D1110001223A310020FEF752FD28
:104630009D4CA38F9F495918628FD21AD2B2002085
:10464000FEF748FD638FA38766E00E246C440122C9
:1046500021003F20FEF73EFD22780F236B441A70A5
:104660001B789B07D2D402A90B230B7001223E209A
:10467000FEF7D0FC6B46D91D10230B7001223F20A2
:10468000FEF7C8FC894800F03FFB874A2623D35C2D
:10469000002B16D1884800F037FB834B00221A719B
:1046A000834B1B68002B03D01B69002B00D098475D
:1046B0007D4B002230215A5401315A549A875A872F
:1046C00065E70E246C44012221000D20FEF702FD57
:1046D000237840221343092169440B7001220D20E5
:1046E000FEF798FC744800F077FAD9E70E246C4482
:1046F000012221003220FEF7EDFC22786A4B5A8716
:1047000096E7694CA38F6B495918D21AD2B2002090
:10471000FEF7E0FC638FA387644800F0F5FA624A75
:104720002623D35C002B1CD1130000221A7162488F
:1047300000F0EAFA5E4B1B68002B09D09C68002C45
:1047400006D0594B32229A56598F00235948A04718
:10475000554B002230215A5401315A549A875A87B6
:1047600015E70E246C44012221000D20FEF7B2FC57
:104770002378402213430A2169440B7001220D2043
:10478000FEF748FC4C4800F027FAD3E70E246C44AF
:10479000012221001920FEF79DFC0023E356424927
:1047A00060228B54002B50DB9B103F241C400E25B5
:1047B0006D44012229001A20FEF78CFC2A7813B2DE
:1047C000002C48DB1B119B188B3B374962228B5214
:1047D0000E246C44012221001320FEF77BFC237879
:1047E000314D6426AB55012221001020FEF772FCEA
:1047F00023780D2169440B7001220D20FEF70AFC7D
:10480000AA5D2C490020FEF765FC5623EB5C002BCB
:1048100002D1254B00221A71244800F075FA244B6E
:104820001B68002B00D1B2E69C68002C00D1AEE6DC
:104830001D496023CB5662228A5E6420095C1D48B4
:10484000A0471E4800F014FBA1E65B429B103F24EA
:104850001C406442ABE71B119B181B198B3B124990
:1048600062228B52B4E7164800F04EFA0E4B5B7989
:10487000012B10D00C4B00221A710D4B1B68002B22
:1048800000D184E61B68002B00D180E698470D48D4
:1048900000F0EEFA7BE60E21694407330B7001222B
:1048A0001220FEF7B7FBE5E7AC0B0020980A0020CA
:1048B000800A0020AC0A0020840A0020DCCC00081A
:1048C000140C0020E8CC000810B582B0434B1B79D3
:1048D000012B03D0022B5ED002B010BD3F4B5B79A1
:1048E000002B1BD0012BF7D13D4800F00DFA6B4691
:1048F000D91D80230B7001221220FEF78BFB374B52
:1049000000221A71374B1B68002BE5D0DB68002BA7
:10491000E2D09847344800F0ABFADDE72F4B5B8FCD
:10492000002B0ED12D4B9B8F002B0AD12B4A22330B
:10493000D35C002B19D1110001223A310020FEF77F
:10494000C9FB264A538F908F191A3E24125D91425B
:1049500016DD264941180020FEF7BCFB1F4B3E2206
:104960009A5C998F52189A87B6E76B46DC1D012234
:1049700021003220FEF7AEFB2278184B5A87E0E781
:104980001A4941181A1AD2B20020FEF7A3FB134BA2
:104990005A8F9A87A0E7114B5B79002B9CD10F4A65
:1049A000538F908F191A3F24125D91420ADC0F49F0
:1049B00041181A1AD2B20020FEF72CFB074B5A8F6F
:1049C0009A8789E7094941180020FEF723FB034B2A
:1049D0003F229A5C998F52189A877DE7AC0B002092
:1049E000980A0020800A0020F4CC0008AC0A0020BD
:1049F00030B583B004000D00FEF7E2FE002C03D0BA
:104A0000012C0ED003B030BD0A4A2223D35C002B08
:104A1000F8D16B46991D0D7001223220FEF7FAFA8B
:104A2000F0E76B46D91D0D7001222320FEF7F2FA44
:104A3000E8E7C046AC0B002010B582B004000120AE
:104A4000FEF7BEFE0B4A5C23D454002C09D16B4602
:104A5000D91D12230B7001223920FEF7DBFA02B0B8
:104A600010BD6B46991D34230B7001223920FEF7CF
:104A7000D1FAF4E7AC0B002070B582B03C4B1B7947
:104A8000012B03D0022B44D002B070BD384B5B79B0
:104A9000002B08D0374B1B68002BF5D0DB68002BB0
:104AA000F2D09847F0E7324C3022A3540132A3549D
:104AB000A38763876B46591D0B230B70303A3E204A
:104AC000FEF7A8FA01A910230B7001223F20FEF780
:104AD000A1FA2623E35C002B14D06B46DC1D0122D7
:104AE00021000D20FEF7F6FA2378402213436A4690
:104AF000911D0B7001220D20FEF78CFA1E4800F06C
:104B00006BF8C7E71A4B00221A711B4800F0FCF83B
:104B1000C0E7FEF759FA0020FEF744FC002410E03D
:104B2000164D66003619705DFEF74AFEAD196878BD
:104B3000AB786A46D11D0B700122FEF76BFA013487
:104B4000E4B2102CECD90020FEF73AFE084C5C23AE
:104B5000E05CFFF771FF00232371064B1B68002BFD
:104B600000D191E75B68002B00D18DE798478BE778
:104B7000AC0B0020800A0020840A0020A8CC00088A
:104B800010B5034B1B685B689847023010BDC046E8
:104B90007C0A002010B500F069FC10BD70B504005F
:104BA00000F026FB050001232372266800F014FCA8
:104BB0002818864203D3206800F036FB70BD00F051
:104BC0000BFC2D182560F6E7002303604360037299
:104BD000C16003617047000070B50400EFF31085F9
:104BE00072B6002829D0264B1A681300002B04D077
:104BF0009C4201D01B69F9E70123002B1DD163689A
:104C0000236000232372002A1AD000F0E5FB2368FA
:104C10009C46604420601A4B1A68136898421ED262
:104C2000002A01D0002313722261154B1C60200062
:104C3000FFF7B4FF85F3108801E085F3108870BD9D
:104C400000F02EFC0E4B1B68002B01D000221A72C4
:104C500023610B4B1C602000FFF7A0FFEAE71369FC
:104C60001169002908D01968884202D91A001B6905
:104C7000F6E714612361DDE7146100232361D9E7BE
:104C8000280C002010B500F017FC040000F008FC10
:104C9000001B1C4B1B68002B0DD01C0002E00021E8
:104CA000116024692269002A05D011688142F6D971
:104CB000091A1160F5E7002B06D0124A1969116034
:104CC000DB68002B12D098470E4B1B68002B0FD0CF
:104CD0001C6800F081FB84420AD20A4A13681969F1
:104CE0001160DB68002B02D09847EDE7FEE7FEE796
:104CF000044B1868002804D0037A002B01D1FFF779
:104D00004DFF10BD280C002010B5EFF3108472B6D3
:104D10001C4B1A68002A0BD0002809D082420AD006
:104D20001300002B28D0834222D01A001B69F8E719
:104D300084F3108822E0137A002B0FD0106900282A
:104D400006D0002313720F4B1860FFF727FF13E004
:104D500000F058FB0B4B00221A600DE01369002B8A
:104D600002D0084A136007E0064B00221A6003E0F5
:104D70001B69002B03D0136184F3108810BD00233E
:104D80001361F9E7280C002070B50400080000F05A
:104D900031FA05002000FFF7B7FF00F029FA85423D
:104DA00002D22060606070BD2800FAE710B500F004
:104DB00021FB00F027FA10BD70B5050000F01AFBCA
:104DC0000400280000F016FA201A00F01BFA70BD4B
:104DD00004E00A7802701A0001310130531E9BB2C0
:104DE000002AF6D170470000EFF3108372B6034A31
:104DF00011680843106083F3108870472C0C002062
:104E0000EFF3108372B603490A6882430A6083F3A2
:104E1000108870472C0C0020014B18687047C04662
:104E20002C0C002010B50F480F4B0360E1235B02F0
:104E3000436000238360C360036183610C3343617B
:104E4000FDF746FD002808D1002201211C20FBF7B8
:104E500061FE1C20FBF78EFE10BD5D21034800F0B3
:104E6000D1FBF1E7300C00200044004000CD0008E9
:104E70000FB4F0B5CE46474680B5A3B02AAB02CBFF
:104E80002193EFF3108572B6219A01A801F0F4FE88
:104E9000C6B21C4B1B88FF2202409B18FF2B24DD4F
:104EA000184F3C88E4B26142CBB299463888164B21
:104EB000984640444A4601A901F036FEA419E4B2DE
:104EC00001A949442200404601F02EFEA4B23C80D4
:104ED00085F310881C20FBF757FE23B00CBC9046CE
:104EE0009946F0BC08BC04B01847064F3B880648FA
:104EF000C01801A901F018FE3C88A419A4B23C8096
:104F0000E6E7C046A20D0020A00C002010B512E07C
:104F1000EFF3108272B6114C2388114959180133EE
:104F2000FF200340238082F3108896235B00012238
:104F30000C48FDF723FC0C4B1B880133FF33074A59
:104F400012889B1AD917090E5B18FF2213405B1AAF
:104F5000002BDDDC1C20FBF723FE10BDA00D002084
:104F6000A00C0020300C0020A20D002030B589B02C
:104F7000134BD96A01221143D962D96A11400191B8
:104F80000199D96A1143D962DB6A13400293029BEB
:104F90000424039402230493059201330693079497
:104FA000A025ED0503A92800FCF79AF80823039330
:104FB000079403A92800FCF793F809B030BDC04658
:104FC0000010024010B5044A916B80239B020B43F2
:104FD0009363FFF7CBFF10BD0010024010B5084BE4
:104FE0001B78002B0BD1074B1B68984700F04CFC3B
:104FF00000F0B4F8FFF716FF014B01221A7010BD44
:10500000A40D002090CB000800B595B0142200211B
:105010000FA801F0CDFD2C22002102A801F0C8FD4F
:1050200002230193012204920F3205920B938023F5
:105030001B030D9380231B040E9301A8FCF796FC21
:10504000002821D1154A916B80235B050B439363A4
:1050500013490B68134A1A4080231B0113430B604A
:105060000F4B5B68DB06FBD40F230F930C3B1093B5
:10507000002311931293139301210FA8FCF78CFFC7
:10508000002806D115B000BDD421074800F0BAFAB7
:10509000D8E7E721044800F0B5FAF3E70010024032
:1050A00000700040FFE7FFFF10CD0008F8B50600D4
:1050B0000C0000222448FBF7A3F96768224D002268
:1050C00031002800FBF7D2F9002221002800FBF76D
:1050D00097F96268BA42F0D1F1781C4B4B43033325
:1050E0009D088B072ED01A4F7078013803011B1AC8
:1050F0009B001B180133D90FC91849104000C74045
:1051000003233B40CB1A5B19B178CB18013B590004
:10511000CB181901CB1A1901C91ACE01A778257825
:1051200029014D1B2901491B0B0160780101091A56
:1051300088001818C01980198002801A054B9C46F7
:105140006044F8BD044FCFE7D00D0020B505000046
:10515000A0AA9900FF0300005055440070B586B026
:105160001E4B1B78002B01D006B070BD1C4C1D4B94
:105170002360002565601F23A3601B4BE36025614E
:10518000A561E5612000FBF745FB6B46DD7001265C
:105190005E709E701E70002269462000FBF72EFC98
:1051A00001A90D704D708D70CD704D600D61CD6099
:1051B00000222000FBF784FB2000FDF76DF8802122
:1051C00049002000FBF77EFA084C211D2000183012
:1051D000FFF76CFF2060014B1E70C5E7A50D002096
:1051E000D00D002000280040FF030000F40D002037
:1051F0000320704710B5410EC0017D220023FBF74C
:105200005DF810BD70B504000025C30E4201121BED
:10521000AB41960F990031439000001969414B064C
:10522000C009184370BD0000F0B587B004005D4BA5
:1052300000255D5F033501A96846FFF737FF5A4B2C
:105240001B68C01A201A854228D20120FFF7D8FD1A
:10525000FFF7E2FD002825D001AD53492A000B1DC0
:10526000C1CBC1C241CB41C28B6900934F48016899
:10527000CA68FF231A404E4B1343CB60802149007C
:10528000FBF720FAAB884B4FFF1ABFB2A3059B0D6B
:10529000FF18BFB2A30A6A46907810E00120FFF71A
:1052A000A3FDD5E70130FFF7ABFD3E4B00229B5E2F
:1052B000E41AD1E7404A94466344013080B23F4A41
:1052C0009342F7D801AA147804E03D4A9446634417
:1052D0000134A4B23B4A9342F7D801AA557802E0C0
:1052E0003C3B0135ADB23B2BFAD801AA96789BB274
:1052F000F618B6B205E0344B9C466744BFB201369F
:10530000B6B22C4B9F42F6D803E03C3EB6B2013514
:10531000ADB23B2EF9D803E03C3DADB20134A4B2AE
:105320003B2DF9D803E0183CA4B2013080B2172C11
:10533000F9D86B46DB789B070BD16B465B78013B5A
:10534000224AD15C8BB298420ED9FAF749FF88B253
:105350000AE06B465B78013B1D4AD15C8BB29842F8
:1053600002D9FAF73DFF88B2124BDF1B19494F6093
:10537000A0231B058B618E704D700C702023C854C8
:1053800001ABDB78CB700023CB614B6180225200F4
:105390004A62CB600B6100220448FBF795F807B026
:1053A000F0BDC046A60D0020F40D0020D00D002059
:1053B0007FFEFFFFFF03000080AEFEFF7F51010074
:1053C000F0F1FFFF0F0E000000FCFFFF34CD0008DE
:1053D00028CD0008A80D002000B587B001A96846B7
:1053E000FFF764FE024B1B68C01A07B000BDC04641
:1053F000F40D002000B587B001A96846FFF756FEFE
:1054000007B000BD10B506480168CA68FF231A40FE
:10541000044B1343CB6080214900FBF753F910BDC7
:10542000D00D00207FFEFFFF10B50120FFF7E8FC44
:105430000B4B1B689A68D20402D5DA68D20500D4F7
:1054400010BDD968FF221140064A0A43DA60064BB4
:10545000802292025A61024800F08CF8F0E7C046C0
:10546000D00D00207FFEFFFF0004014030B587B063
:10547000410EC0017D220023FAF720FF040001A99C
:105480006846FFF713FE050000E0C04601A9684624
:10549000FFF70CFE401BA042F7D307B030BD000061
:1054A00010B5044C211D20001830FFF7FFFD2060CF
:1054B00010BDC046F40D0020014B18687047C0466F
:1054C000F40D00200020704700B583B001900198D2
:1054D000FFF760FB03B000BD10B5094A916B802354
:1054E0005B050B439363FAF783FFFDF79BFC054ACB
:1054F000136808210B431360FDF78AFC10BDC046FA
:10550000001002400020024000B599B004230A9325
:10551000002314930133FF330C930AA8FCF726FAF7
:10552000002819D12023009380235B020193684651
:10553000FDF706FA002814D10C4A116D8023DB0216
:105540000B431365002200210220FBF7E3FA02203F
:10555000FBF710FB19B000BD8D21054800F052F893
:10556000E0E79521024800F04DF8E5E70010024021
:1055700040CD000810B5FFF785FB10BD10B500F059
:1055800027F910BD042809D004D80138012803D810
:1055900005207047082801D00720FAE70620F8E721
:1055A00030B587B00C22002103A801F001FB0323D2
:1055B0000293C023DB010193104CE36A01252B43C6
:1055C000E362E36A2B400093009BA02001A9C00581
:1055D000FBF786FDE36AAB43E362626B8023DB0388
:1055E00013436363FCF740FEFCF746FEFCF74CFEFA
:1055F000636B034A1340636307B030BD0010024081
:10560000FFFFBFFF10B50A04120C01000148FFF7AD
:105610002FFC10BD5CCD000810B51748174B036078
:10562000174B4360002383600122C2600361436122
:105630008361C3610362FBF737FF00280CD10021AF
:105640000D48FCF79DFD00280BD100210A48FCF70E
:10565000C3FD00280AD110BD4F210A48FFF7D2FF31
:10566000EDE756210748FFF7CDFFEEE75D2105483E
:10567000FFF7C8FFEFE7C046100E002000540040BF
:10568000060722F070CD000800B587B002680D4B08
:105690009A4201D007B000BDC0239B0001931223A2
:1056A0000293113B0393023304930133059301A941
:1056B0000548FBF715FD054A916B80239B030B43BF
:1056C0009363E7E7005400400004005000100240DC
:1056D00030B587B0224CA04223D00FD9214CA04234
:1056E00029D0214CA04230D1204CE56A08231D432B
:1056F000E562E46A23400493049B0CE0A024E405E3
:10570000A04222D1194CE56A01231D43E562E46AF7
:1057100023400193019B11601100FBF7E1FC07B0EE
:1057200030BD124CE56A02231D43E562E46A234062
:105730000293029BEFE70D4CE56A04231D43E562EB
:10574000E46A23400393039BE5E7084CE56A802362
:105750001D43E562E46A23400593059BDBE7C046F1
:105760000004005000080050000C005000100240DF
:1057700070B51400FF2208009043021E00D00822DA
:105780000F48014201D0042002430E48014201D0DB
:10579000022002430C48014201D001200243002BA9
:1057A0000DD09200094813500800FFF7EBFE0500EA
:1057B00000222100FBF7AEF92800FBF7DBF970BDF2
:1057C000F0F0FFFFCCCCFFFFAAAAFFFF5C0E002089
:1057D00010B5FF2302009A43131E00D008230B4A82
:1057E000104201D004221343094A104201D0022280
:1057F0001343084A104201D0012213439B00064A7A
:105800009B58002B00D0984710BDC046F0F0FFFF1A
:10581000CCCCFFFFAAAAFFFF5C0E002010B5D2B2CD
:10582000FBF72CFD10BD000010B586B0142200213E
:1058300001A801F0BDF902230293039301330493FD
:10584000A024E40501AA20212000FFF741FF01AABE
:1058500040212000FFF73CFF01AA80212000FFF734
:1058600037FF012302930393064C01AA4021200035
:10587000FFF72EFF012240212000FFF7CFFF06B0E7
:1058800010BDC0460004005010B51F4B1F4A1A60DF
:105890001F4B1A6800231F498A4203D9013352085B
:1058A000062BF8D95A0724D40022990723D40021C3
:1058B0000A43DB0721D5082313431348C3610023A0
:1058C000836082225200426003614361C36083624D
:1058D0000362FC32826143620F4A516B80235B0199
:1058E0000B435363FBF7E2F9002808D1FFF79CFF55
:1058F00010BD2022D9E71021DAE70023DCE772216E
:105900000648FFF77FFEF1E79C0E002000300140C3
:1059100030000020809698000010024080CD0008E2
:1059200010B586B00E216944088016246C4401230A
:105930005B420093023322000248FBF7FBF9208808
:1059400006B010BD9C0E002010B588B0FCF76EFCB0
:10595000FFF75AFBFFF724FE154BDA6A01242243B6
:10596000DA62DA6A22400192019AD96A042211436A
:10597000D962DB6A1A400292029BFFF72FFBFFF706
:105980004BFE1422002103A801F012F90494032312
:10599000069303AA80210748FFF79AFE00F0CEF88D
:1059A000044A536980214B40536100F003F9F7E743
:1059B0000010024000080050104B1968802252006D
:1059C0000A431A60DA680E490A40DA601A680D491B
:1059D0000A401A609A6801218A439A601A680A4943
:1059E0000A401A60DA6809490A40DA6000221A613E
:1059F000074B802212059A607047C0460010024093
:105A00000C40FF88F6FFF6FEFFFFFBFFFFFF02FFE3
:105A100000ED00E07047000010B50248FFF728FADB
:105A2000C046FDE7B4CD00087047704710B5FCF7DD
:105A30000DFC10BD10B5FFF769FA10BD10B5FFF7EA
:105A4000F3FC10BD10B50120FBF71EFC0220FBF794
:105A50001BFC10BD10B50420FBF716FC0820FBF75B
:105A600013FC10BD10B51020FBF70EFC2020FBF737
:105A70000BFC4020FBF708FC8020FBF705FC802096
:105A80004000FBF701FC80208000FBF7FDFB80203D
:105A9000C000FBF7F9FB80200001FBF7F5FB80203D
:105AA0004001FBF7F1FB80208001FBF7EDFB80203C
:105AB000C001FBF7E9FB80200002FBF7E5FB10BD0E
:105AC00010B5FFF701FD10BD70B592B002AC2170AA
:105AD000002404E0151901342E7802AD2E55A3429E
:105AE000F8DC01339BB241006422009202AA034811
:105AF000FBF740FD002012B070BDC046100E002024
:105B0000F0B585B002921F000F236B441A00197084
:105B10004400094D64260096012321002800FBF76C
:105B200029FD00963B00029A21002800FBF700FEA9
:105B3000002005B0F0BDC046100E002070B5174C17
:105B4000762363700125A570154BA364154BE364A0
:105B5000154B23651548FFF78BF9200000F0E9F994
:105B60001348FFF785F902233822A3540232032198
:105B7000A154013A0131A1540232A3543C33E554FB
:105B800002330632FF32E2520233AA3AE2520233C1
:105B9000E5542100DF2000F01FFB70BDF40E002053
:105BA000015B0008C95A0008C15A0008C4CD0008AA
:105BB000E0CD0008F0B58DB0254D280000F0AFFA1B
:105BC000262402AB9C4664442900200000F028FDF6
:105BD0002088FFF779FC06AC2900200000F044FD86
:105BE0000423E05E05F006FA1A4905F025F9071CC2
:105BF000A06805F041FA174905F01EF9051CE06898
:105C000005F03AFA144905F017F9061C381C06F09D
:105C10006FFE04900591301C06F06AFE029003911D
:105C2000281C06F065FE00900191049A059B0B4824
:105C3000FFF71EF923789B0604D40948FFF718F9EB
:105C40000DB0F0BD0A990748FFF712F9F5E7C04615
:105C5000F40E00200000C84200007A44F8CD00088D
:105C6000C0CD000820CE000830B583B00C1E33D064
:105C70008D6C002D33D0CB6C002B33D00B6D002BF3
:105C800033D040B2002825DB1023E2789A422FD08F
:105C9000E370607801236A460732F321A847542352
:105CA000E054002826D16B46DA1D137810218B436F
:105CB000190003202056102303400B431370607813
:105CC00001237321E56CA8475422A054002814D165
:105CD00003B030BD0023D8E701204042F8E701209F
:105CE0004042F5E701204042F2E701204042EFE761
:105CF0000020EDE702204042EAE702204042E7E7C9
:105D000030B583B0041E19D0856C002D19D0C36C3A
:105D1000002B19D0036D002B19D0407801236A465F
:105D20000732F321A8475422A054002812D16B4611
:105D3000DA7910231340E37003B030BD01204042F4
:105D4000FAE701204042F7E701204042F4E7012052
:105D50004042F1E702204042EEE7F0B583B0050093
:105D6000019117001E1E23D09B6C002B23D0F36CD7
:105D7000002B23D0336D002B23D0B378002B0DD014
:105D8000002470783B00019A2900B56CA847542381
:105D9000F054002818D1200003B0F0BD3100FFF707
:105DA00063FF041EEDD180235B421D43EDB2E8E7A3
:105DB00001246442EFE701246442ECE701246442D9
:105DC000E9E701246442E6E702246442E3E7F0B530
:105DD000D64600B58CB005000E00140000921F00DE
:105DE0002822002102A800F0E3FE002F4AD0BB6C5D
:105DF000002B4BD0FB6C002B4CD03B6D002B4DD0BF
:105E0000631EDBB2122B03D800240023019318E099
:105E100004235B42019330E02B199A46187839002D
:105E2000FFF722FF01906300524611787F220A405B
:105E300002A9CA5463000133325D02A9CA54013475
:105E4000A4B26B461B88A34207D9BB78002BE3D0D2
:105E500063002A5D02A9CA54ECE7019A002A0CD11A
:105E60005B00013B9BB202AA117878780132FC6C8E
:105E7000A0475423F854002814D101980CB004BC56
:105E80009246F0BD01235B420193F6E701235B429A
:105E90000193F2E701235B420193EEE701235B42AA
:105EA0000193EAE702235B420193E6E730B583B052
:105EB00004006B46E022DA716B462A3A9A71002898
:105EC0002BD0836C002B2BD0C36C002B2BD0036DFD
:105ED000002B2BD08378002B05D00025002D06D079
:105EE000280003B030BDFFF70BFF0500F6E72300E5
:105EF00001226946063168460730FFF768FF050052
:105F00000A20236D9847002DEAD1A378002BE7D112
:105F10002000FFF7F5FE0500E2E701256D42DFE70F
:105F200001256D42DCE701256D42D9E701256D426F
:105F3000D6E7F0B593B0041E00D1E1E0836C002BEE
:105F400000D1E0E0C36C002B00D1DFE0036D002B3B
:105F500000D1DEE0FFF7AAFF002801D013B0F0BDAA
:105F6000230001222100D030FFF7F7FE0028F5D1F1
:105F70002378612B00D0CFE04122002101A800F05E
:105F800017FE6B460022DA70002C00D1ACE0A36C47
:105F9000002B00D1ABE0E36C002B00D1AAE0236D15
:105FA000002B00D1A9E02300193201A98920FFF7B5
:105FB000D4FE00286BD001AB2222995C0902013A81
:105FC0009A5C0A43E282997809025A780A4322834A
:105FD00003229A56A276997909025A790A43A28332
:105FE000197A0902DA790A43E28309229A562026AD
:105FF000A255197B0902DA7A0A436284997B090265
:106000005A7B0A43A28410229A56262562550F21F4
:1060100059562722A154197D0902DA7C0A432285A8
:10602000997D09025A7D0A436285D97D2C22A154AB
:10603000DF7E3F019A7E0F21114039432181597E35
:10604000090112090A4362811C229A5622731D22F9
:106050009A5662731E229A56A273DA7FE2739A5797
:10606000227425229A5662742422995C0902013A0C
:106070009A5C0A4362825B57237500280FD06B46F7
:1060800003331B785BB21B113622A35466E723004F
:1060900010221D216944E130FFF75FFE8BE76B465C
:1060A000DD1C2300012229000230FFF756FE2A786A
:1060B000302313401B113422A3540028DFD16B4638
:1060C000DD1C2300333A2900FFF747FE0022AA56C1
:1060D0003523E2540028D2D123000122694603313E
:1060E0000430FFF73AFECAE70120404236E70120BC
:1060F000404233E70120404230E7012040422DE793
:10610000012040422AE70120404227E70120404287
:1061100024E70120404221E7032040421EE770B5FA
:1061200082B006006B4674229A71002848D0836CB6
:10613000002B48D0C36C002B48D0036D002B48D0F7
:10614000002501E0002D1ED03300012269460731F1
:106150007420FFF702FE041EF4D16B4607331B7850
:1061600003251D40EED0032293436A46D11D0B70D8
:106170003300012268460630FFF729FE04000A209A
:10618000336D9847DEE74423F25C002A0BD06B4660
:10619000D91DDB79032083435BB252B20240134323
:1061A0000B70002C02D0200002B070BD3300012221
:1061B0006946073168460630FFF709FE0400F2E73A
:1061C00001246442EFE701246442ECE701246442C5
:1061D000E9E701246442E6E7F0B5D6464F46464675
:1061E000C0B586B006000C0017236B4400221A705D
:1061F0000632002104A800F0DBFC0622002102A8E0
:1062000000F0D6FC4423E35C9A46002C00D1F6E172
:10621000A36C002B00D1F5E1E36C002B00D1F4E17D
:10622000236D002B00D1F3E1330735D40020442344
:106230000022E254002800D1C9E0F30600D4CDE0EA
:1062400023003B3300D1C6E03B23E35C072B07D997
:106250003B230722E2543F32A35C02210B43A354A9
:1062600023000122172169447520FFF776FD1722CC
:106270006A4413781C218B435BB21F31655CAD000F
:106280001F3929400B43DBB2137004AA752111702A
:1062900002AA13700125A2E0002C00D18BE0A36CB0
:1062A000002B00D18AE0E36C002B00D189E0236D44
:1062B000002B00D188E000236A46138001AA1380D6
:1062C0004433E35C012B01D00120B0E759336A4627
:1062D00013701A3BE55AC72D06D95133FF339D423F
:1062E00003D9C8256D0000E0C8250423E356142017
:1062F00020565843FA218900F9F728FF03029946EE
:106300001123E356C4229200904698441222A35EC1
:10631000C14A944663446B439800C0186421F9F75E
:1063200015FFC8239B039C4660440A21F9F70EFF22
:1063300043464343D80FC018401048443423E15C1F
:106340000431F9F703FF3523E3569901C9184900D1
:10635000C91880235B029C466144F9F7F7FE0300ED
:10636000FA3B1801C018400032306421F9F7EEFE04
:1063700001AB187064236A465370223BE35AA74A64
:10638000934216D8002202E09B080132D2B23F2B82
:10639000FAD8DBB29201D2B29B18DBB201A94B70E2
:1063A0003C230022E254230002326846FFF70FFD2F
:1063B0003DE7FF23F2E70120404238E70120404259
:1063C00035E70120404232E7012040422FE720001C
:1063D000FFF7A5FE31E70120404248E70025B3065C
:1063E0002CD523003D3300D1F3E03D23E35C082BA3
:1063F00007D93D230822E2543E32A35C02210B431D
:10640000A35423000122172169447020FFF7A5FC43
:1064100017226A44137808218B435BB235316156E9
:106420008C460821674639400B43DBB2137004AA3F
:106430007021515502AA53550135EDB2B3073DD035
:106440002300393300D1C7E03923E35C052B07D99A
:1064500039230522E2544132A35C02210B43A354A9
:1064600023000122172169447420FFF776FCF3070B
:1064700009D517226A4411781F230B403921615C2A
:1064800049010B431370B3070ED517226A441378E2
:106490001C218B435BB21E31615C89008C461C2140
:1064A000674639400B43137004AB74225A551723C7
:1064B0006B441A7802AB5A550135EDB273072CD5EF
:1064C0002300383300D18AE03823E35C052B07D959
:1064D00038230522E2544132A35C02210B43A3542A
:1064E00023000122172169447220FFF736FC17228E
:1064F0006A44137807218B435BB2313161568C4675
:106500000721674639400B43DBB2137004AA72219E
:10651000515502AA53550135EDB2C02333424DD037
:1065200023003E335ED03E23E35C012B07D93E239C
:106530000122E2544532A35C02210B43A354230001
:106540003C3352D03C23E35C0A2B07D93C230A227C
:10655000E2543C32A35C02210B43A35423000122EA
:10656000172169447120FFF7F8FB73060ED5172237
:106570006A44137810218B435BB22E31615C0901B0
:106580008C461021674639400B43137033060BD5F8
:1065900017226A4413780F218B435BB22D31665664
:1065A0002D3931400B43137004AB71225A55172318
:1065B0006B441A7802AB5A550135EDB2002817D05A
:1065C00044235246E25406B01CBC90469946A2466B
:1065D000F0BD012040421BE70120404247E7012077
:1065E000404284E701204042BFE701204042BCE72F
:1065F00023002A0002A904A8FFF7E9FBE0E7012035
:106600004042E0E701204042DDE701204042DAE776
:1066100001204042D7E7C04699590200BF0F000051
:1066200070B504000D003923C85C0133CB5CC01881
:106630003823CB5CC3180A4858430A4B9C46604435
:10664000FA218900F9F73CFD013080B220803E2319
:10665000EB5C002B03D04223EB5AC018208070BDA6
:10666000AB070000B9120000F0B5DE4657464E46B3
:106670004546E0B58BB081460D1E00D1C8E18B6C5C
:10668000002B00D1C8E1CB6C002B00D1C8E10B6D11
:10669000002B00D1C8E10F22002106A800F088FAE3
:1066A000002D0ED0AB6C002B12D0EB6C002B13D056
:1066B0002B6D002B02D00023019305E0013B0193D9
:1066C00002E001235B4201930A24019E4F4628E128
:1066D00001235B420193F7E701235B420193F3E758
:1066E0000196B946029FC010EB8A5B00C01AC11721
:1066F0001823EA5ED3170290049104F0D3FA4905F7
:10670000C60A0E430499CB070298400818430200BA
:106710000B0004F0C7FA0B05000B184309131A22EB
:10672000AA561201D31704F0BDFA8904800B08435E
:106730003018286383001B1880331B124A4693804D
:106740002B6B5A10BA4B9C46624491104943C812B5
:106750002623EB5643439B102426A85F504340005A
:106760001B189B102226A85F00041B184813202129
:10677000695649014143C9101E26A85F4243521081
:10678000891889148022120294466144AA8B5143CD
:10679000C91380204003C01B1B13C01AA54B5843CC
:1067A000F9F78EFC40002A23E95EC21052435313CE
:1067B0004B431A1383102826A95F59434913061225
:1067C000330073435E432C23EB5C73435B1451181B
:1067D0005B182722AA56D2019B181B11C0184B46E2
:1067E00098602B6B9E00F618803636122F893F0179
:1067F0005B46DF1B0C20285670436421F9F7A6FC8A
:1068000040103B1A02936A8993460D202856704324
:106810006421F9F79BFC07000E2028567043642181
:10682000F9F794FC704380116421F9F78FFC3F184D
:106830008022D201944667445A465743BF12029BB6
:106840005F43E87BC3019B461020285670436421B8
:10685000F9F77CFC58440011BB135B439B12434384
:106860005B10FF18BF127B01DB1B9B00DB19DB00F9
:106870001B13714A934203DC002B02DA002300E071
:106880006D4B4A46D3603623EE563000F617310082
:10689000870FB3003B43820012184B416748002129
:1068A0008018594153469B009A46654B5246D25830
:1068B000002304F0F7F90B04060C1E430F1400210B
:1068C0004346D803FF22120601235B4212184B41B4
:1068D00092197B41049205935A4B5146CA580023A2
:1068E0003000390004F0DEF9CE05430A3343029349
:1068F0004B120393049A059BDE07500830431600A1
:106900001F005910029A039B8018594132003B0026
:10691000F9F7B0FC4B4618615EE0013CE4B2002C94
:1069200058D0002EF9D12B000F2206A91D20FFF709
:1069300014FA060006AB1B787F22190091438C469F
:10694000703A924613407B7006AB5B78BB7006AB27
:106950009A781203DB781B011A4306AB1B791B09DB
:106960001A43029206AB587900039B791B01184326
:1069700006ABDB791B09184306AB197A09025B7A6F
:1069800019438B4606AB5B7B9B00984606AB9B7B13
:106990009A099146424649460A43904652461A4051
:1069A00092465BB2994620234A46134062461343FF
:1069B0005BB206AA927B52B29146102294464A4696
:1069C00061460A4013433B7000D589E60A202B6DCF
:1069D0009847A2E70196B946002C12D0019B002BE4
:1069E00007D14B461B785BB2002B0DDB4523002201
:1069F000EA5401980BB03CBC90469946A246AB467F
:106A0000F0BD02230193E9E745230122EA54F0E7B0
:106A100001235B420193ECE701235B420193E8E72A
:106A200001235B420193E4E701235B420193E0E72A
:106A30000006FFFF350C0000A08601003C050000A9
:106A400034000020740000200D488546002103E03A
:106A50000C4B5B58435004310B480C4B42189A4284
:106A6000F6D30B4A02E0002313600432094B9A422A
:106A7000F9D3FEF7A1FF00F033F8FEF765FFFEE75C
:106A80000050002034D20008000000205C0A0020E2
:106A90005C0A0020880F0020FEE7000010B501000E
:106AA00000230022002000F0F3F810BD70B5094B60
:106AB000094CE41AA41009D0084AA518AD00ED1835
:106AC0002B68013C9847043D002CF9D105F0FEFFEE
:106AD00070BDC04630D2000834D20008FFFFFF3F2F
:106AE00070B50D4E0D4DAD1BAD1006D00024A300AA
:106AF000F35801349847A542F9D105F0E1FF084E5B
:106B0000084DAD1BAD1006D00024A300F35801348E
:106B10009847A542F9D170BD28D2000828D20008B4
:106B200028D2000830D20008F0B50F2A37D90D005E
:106B300005430C000300AD0735D11500103D2D09AC
:106B40002E013618103627681F6067685F60A768D7
:106B50009F60E7681034DF601033B342F3D10F2435
:106B600001352D01491914404519032C1DD9002365
:106B7000CE58EE500433E61A032EF9D80323043C12
:106B8000A4080134A4001A402D190919002A05D0BF
:106B90000023CC5CEC5401339342FAD1F0BD0500E4
:106BA000002AF5D1FAE70500F2E72200F8E7C0462F
:106BB000F0B5830746D0541E002A42D0CEB2020060
:106BC000032502E01A00013C3BD3531C16702B42F4
:106BD000F8D1032C2DD9FF220A40150215432A04AF
:106BE00015430F2C16D92700103F3F093E01B4462C
:106BF0001E001A0010366644156055609560D56019
:106C00001032B242F8D10F2201373F01DB19144094
:106C1000032C0ED9261FB608B700BC461A001F1D4C
:106C2000674420C2BA42FCD103220136B6009B1948
:106C30001440002C05D0C9B21C19197001339C42B4
:106C4000FBD1F0BD14000300C3E7C04600B59BB004
:106C50000091049106490591029106490391694604
:106C600000F08CF80023009A13701BB000BDC046E2
:106C7000FFFFFF7F0802FFFF10B504001300034A67
:106C800010680A002100FFF7E1FF10BDB4000020EA
:106C9000F8B5DE469B46314B45461C68A4234E465C
:106CA00057465B00E0B50500E0580E00904600280E
:106CB0004BD043681F2B0DDC5C1C002D21D102330F
:106CC0009B0044601E5000203CBC90469946A24662
:106CD000AB46F8BD224B002B3CD0C820400000E062
:106CE00000BF002836D0A42200235200A1584360E0
:106CF0000160A05040328350043283500124002DA3
:106D0000DDD09A0091468144424688214F467A5010
:106D1000C422520090468044424687399940126806
:106D20008A460A4394464246614611608422494697
:106D30005F4652008F50022DC1D1020055468D3260
:106D4000FF3211680D431560B9E720004D30FF3068
:106D5000E050AEE701204042B6E7C04630CE000822
:106D600000000000034B10B5002B02D00248FFF7D3
:106D700095FE10BD00000000AD6A0008F0B5DE46CB
:106D80004E4657464546E0B5C3B00C0007919146C4
:106D90001093089002F020FB036818001A9303F088
:106DA00093F91990A3891B0605D523690993002B34
:106DB00001D100F023FF32AB2593002325AFBB6048
:106DC0007B60189300240023169317940023CA466F
:106DD00032AE14931B930C9353461B78002B47D071
:106DE0005446252B02D11BE0252B03D001342378F8
:106DF000002BF9D15346E51A0FD03360BB6875609C
:106E00005B19BB607B6801337B60072B27DC08368E
:106E10000C9B9C46AC4463460C932378002B27D0F4
:106E2000631C9A46002316AAD37701225242934646
:106E300000220B922032904620329146383A6378F5
:106E400094460021002400255246180020380132C3
:106E5000099158283ED8BF498000085887463A0013
:106E60000799089803F062F9002809D132AECFE7FC
:106E7000BB68002B04D03A000799089803F056F934
:106E8000079B9B895B0601D501F058F90C9843B02C
:106E90003CBC90469946A246AB46F0BD0021303B33
:106EA0001800099B0A959A460D00AB005D191378EE
:106EB0006D0045191800511C30380A000928F4D912
:106EC00052468A46099252460B950A9D1800203870
:106ED0005828C0D9099913939246002901D001F08E
:106EE0001CFA139A002AC3D028AB1A70002216A9E4
:106EF000CA770A9501327EE1802309991D431378F0
:106F0000A3E7531C0A9313782A2B01D101F0CFF980
:106F10001800002230389346092801D901F097F86B
:106F2000099B5946A2469B460A9A8B005B185B0058
:106F300019181378541C1800303822000928F4D985
:106F400020005A465446824609928B465246BDE777
:106F5000099913780420054377E7137801212B243E
:106F600073E710980999036804300B9310900B98FD
:106F70001378002800DB68E740420B90EAE7012322
:106F800009991D43137860E709991378002C00D004
:106F90005BE70121203458E70999139392460029B1
:106FA00001D001F0B2F96C4B1493AB0600D409E3A5
:106FB0000722109B07339343013294469C44624658
:106FC0005C681B680E930F9410920223EA0769D540
:106FD0000E990F9A0800104364D030211EAA117038
:106FE0004C206946091809781D435170002216A9E2
:106FF000CA775A4601325BD1002291460A95012B8D
:1070000000D1CFE0022B01D100F036FC0E980F9991
:107010005B4632AA90460993B34600E0A0464A0771
:107020009446434665465C1EC6080723CA08354396
:1070300011002A0003403033237028000A43EDD1A9
:107040000E900F9109995E468B460A99424612941A
:10705000C90701D500F0F1FC32AB1B1B0D935B4659
:1070600009930D9B9B4500DA0993002315934B462A
:10707000002B00D1C8E0099B01330993C4E01393AE
:107080009246AB0600D4B2E20722109B073393432B
:10709000013294469C4462465C681B680E930F94D0
:1070A00001231092002216A9CA775A460132A3D0B2
:1070B000002291468022290091430A910E990F9A4D
:1070C000080010439BD15A46002A01D000F047FE29
:1070D000002B01D000F071FC0120030032AA2B40EC
:1070E0000D931292BBD02723302128AAD15416AA7F
:1070F0009446483363441293B1E71393109B92462E
:107100001C1D1B6816A91A0012930023CB77002AB6
:1071100001D100F0A5FD5B46013301D100F08DFEE9
:107120005A460021129802F023FC002801D100F0F9
:1071300096FF129BC21A16ABDB7F0D929946D34382
:10714000DB171A400023099210940A959B46159369
:107150008DE7C04634CE0008BCCF000809991393D0
:107160009246002901D001F0D4F8AB0600D40FE21A
:107170000722109B07339343013294469C44624696
:107180005C681B680E930F9410920F9B002B01DA22
:1071900000F077FC16ABDB7F99465A46012301329B
:1071A00088D10A950E9B0F9C002C01D000F07EFD2B
:1071B000092B01D900F07AFD27220E9B28A9303334
:1071C0008B54012316AA94460D936E336344129395
:1071D00045E7109992460A68242009926A461218D7
:1071E0001278139328AB1A70002216A8C2770A1DD2
:1071F000109201220A9509920022914601320D92C5
:10720000002293461592129302230A9A1A4090463E
:1072100002D0099B0233099384230A9ABC681A405E
:10722000119238D10B9B099A9D1A002D33DDCC4A5F
:107230007B689146102D1FDD22004C4603E0103D77
:107240000836102D16DD10211032013334607160C4
:10725000BA607B60072BF2DD3A000799089802F0CC
:1072600065FF002800D00BE6103DBA687B6832AE9F
:10727000102DE8DCA14614004A466419013332603F
:107280007560BC607B60072B01DD00F03BFD16AB39
:10729000DB7F083699464B46002B0FD016AA1F23DA
:1072A000944663443360012373607B680134013387
:1072B000BC607B60072B00DDC6E208364346002B2E
:1072C0000CD01EAB3360022373607B680234013341
:1072D000BC607B60072B00DDC2E20836119B802B6F
:1072E00000D120E25B460D9A9B1A9B46002B32DDB3
:1072F0005A467B689B4D102A22DD1022A8469146F3
:107300005D4603E0103D0836102D17DD4246326021
:107310004A46103401337260BC607B60072BF1DD9C
:107320003A000799089802F001FF002800D0A7E56D
:10733000103DBC687B6832AE102DE7DCAB4645469D
:107340005A465C44013335607260BC607B60072B39
:1073500000DDAFE208360A9BDB0500D584E1129B15
:1073600033600D9B9C4673607B6864440133BC6052
:107370007B60072B00DD6BE108360A9B5B0731D58C
:107380000B9B099A9D1A002D2CDD754A7B6891464E
:1073900010229046102D04DC1BE0103D0836102D05
:1073A00017DD6F4A10343260424601337260BC60B0
:1073B0007B60072BF1DD3A000799089802F0B6FED2
:1073C000002800D05CE5103DBC687B6832AE102D13
:1073D000E7DC4A466419013324C6BC607B60072B96
:1073E00000DD36E30B9A099B9A4200DA1A000C9BE7
:1073F0009C46944463460C93002C00D0CEE10023BD
:1074000032AE7B60E8E413939246AB0651D5072277
:10741000109B07339343013294469C4462465C6858
:107420001B6810920E930F9400233BE60999924635
:10743000002901D000F061FF109A08CA1092AA0634
:1074400000D52BE3EA0601D500F058FC6A0601D40A
:1074500000F054FC6A46128E1A80BDE44346099936
:107460001D431378F1E4109992460B683E4A0E933F
:1074700000230F9302331D431EAB1A8078220B1D8D
:1074800010933A4B1392149302230BE61378099945
:107490006C2B00D1D2E310200543D6E44B4609996A
:1074A0001D431378D1E4139310231D439246AB067A
:1074B000ADD4109A08CA1092EA0602D46A0600D522
:1074C0009BB20E9300230F93ECE5634609991D438D
:1074D0001378BAE4099913939246002901D000F079
:1074E00010FF0722109B073393431A0018CA9846CF
:1074F00010920122169317946400640852421C4BA8
:107500004046210005F048F9002800D0CCE20122D5
:10751000174B524240462100F8F78EFE002800D05B
:10752000C2E21698179900220023F8F77BFE002884
:1075300001D000F048FD16ABDB7F9946139B472B2B
:1075400001DD00F080FC0B4B129380239D437D3BBB
:1075500009930D9300230A959B46159387E5C04632
:10756000DCCF0008ECCF000830780000BCCF00086A
:10757000FFFFEF7F98CF00080999139392460029E7
:1075800001D000F0ABFE10231D43AB0600D5EFE5A4
:10759000109A08CA1092EA0600D56AE26A0600D478
:1075A00067E21BB20E93DB170F93EEE50999139375
:1075B0009246002901D000F09CFEC44B1493AB0608
:1075C00000D5F5E4109A08CA1092EA0600D54BE2FD
:1075D0006A0600D448E29BB20E9300230F93F4E4B2
:1075E000139310231D439246AB0600D54CE5109A29
:1075F00008CA1092EA0602D46A0600D59BB20E931E
:1076000000230F9301334DE501330D931300A3467F
:1076100091460C0008334A465946156051600D9A50
:107620005C44BC607A60072A00DDF6E21E009946E1
:1076300001320D9208364A4621AB13601B9B9C46D3
:1076400053600D9B6444BC607B60072B00DC94E6B8
:107650003A000799089802F069FD002801D0FFF769
:107660000FFCBC6832AE88E6139B652B00DC9FE004
:107670001698179900220023F8F7CEFD002800D1B4
:107680002AE1934B01343360012373607B68BC6053
:1076900001337B60072B00DDB6E308361F9B189A89
:1076A000934204DB0A9BDB0701D4BC6865E61A9BA6
:1076B000BA683360199B9C4673607B6862440133EF
:1076C0001400BA607B60072B00DDBDE20836189B12
:1076D000013B9846002B00DC4FE642467B687D4D1F
:1076E000102A00DC43E3102291462200444604E0C5
:1076F0000836103C102C00DC37E3494610320133C9
:1077000035607160BA607B60072BF1DD3A00079944
:10771000089802F00BFD002801D0FFF7B1FBBA6812
:107720007B6832AEE5E70B9B099A9B1A9846002BC3
:1077300000DCD7E542467B68664D102A22DD102228
:1077400091462200444603E0103C0836102C17DD19
:1077500049461032013335607160BA607B60072B97
:10776000F2DD3A000799089802F0E0FC002801D009
:10777000FFF786FB103CBA687B6832AE102CE7DC62
:10778000A046140042464444013335607260BC6038
:107790007B60072B00DDF6E20836A3E53A00079987
:1077A000089802F0C3FC002800D128E6FFF768FB28
:1077B000082189467A6818990134531CB14401297B
:1077C00000DC29E1129ABC60326001227B607260A9
:1077D000072B00DDA6E24A461A9901331160199A77
:1077E0004946944664444A60BC6098467B60072BD7
:1077F00000DDA5E208239C46E1444346169817990C
:107800004E465D1C189B0022013B9B4600231195B0
:107810000D950836F8F700FD002800D0D3E04A4661
:10782000129B5C44013313604B465A46BC605A605D
:107830007D60072D00DDF0E1434602330D934B469A
:107840001033B1461E00F6E63A000799089802F098
:107850006DFC002801D0FFF713FBBC6832AE2DE5AC
:107860003A000799089802F061FC002801D0FFF760
:1078700007FBBC6832AE31E50F20B44632AB1900CD
:107880000E9A0F9B0400149D14402C5D16091D07D1
:10789000013935430C701C0923002C002A001C43BD
:1078A000F0D10E920F9332AB5B1A129166460D9394
:1078B000FFF7D5FB3A000799089802F037FC00283B
:1078C00001D0FFF7DDFABC6832AE44E5A8CF00086E
:1078D000D8CF0008ECCF00081F99002900DC5FE238
:1078E000159B1D00189B9D4200DD5DE1002D0BDD09
:1078F000129B641933607B6875600133BC607B60E8
:10790000072B00DD53E30836EB43DB171D40159BC7
:107910005B1B9846002B00DD4AE11F9B189A93429F
:1079200000DAB4E10A9AD20700D5B0E11899159AA5
:10793000CB1A8A1A1D00934200DD1500002D0EDDC2
:107940001599129A8C46624432607A686419013241
:107950007560BC607A60072A00DD69E30836EA4397
:10796000D21715405B1B9846002B00DC05E542460C
:107970007B68E04D102A00DCF9E1102291462200DC
:10798000444604E00836103C102C00DCEDE149468A
:107990001032013335607160BA607B60072BF1DD16
:1079A0003A000799089802F0C1FB002801D0FFF7C0
:1079B00067FABA687B6832AEE5E700230D9332AB15
:1079C0001293FFF74CFB5B46002B00DC33E6102BD9
:1079D00001DC00F042FC2100C64D10264A465C4600
:1079E000119B05E00832103C102C00DC0CE6013342
:1079F000103115605660B9607B60072BF2DD3A00EC
:107A00000799089802F092FB002801D0FFF738FA96
:107A1000B9687B6832AAE6E701210A98014200D0E2
:107A2000D0E6129871603060BC607B60072B00DD8F
:107A3000F3E0931C0D931036FDE5302B00D120E1CF
:107A40003023023A137032AB9B1A0D931292FFF758
:107A500006FB3A000799089802F068FB002801D05D
:107A6000FFF70EFABC68BDE40E9300230F93FFF7F7
:107A7000ACFA0E93DB170F930F9B002B01DBFFF784
:107A800089FB0E990F9A00244B4294410E930F9458
:107A90002D2316AAD3779946FFF77FFB0C9A1A601D
:107AA000D2175A60FFF798F91698179902000B0041
:107AB00004F072FE002800D0ACE32023139A9A430E
:107AC0005B469146013300D1C6E2472A00D1C7E1A7
:107AD00080235B002B430A93179B002B00DA78E28C
:107AE000169A0993002390461193139B662B00D19D
:107AF00088E2462B00D1E7E24B46452B00D1B6E1A8
:107B000023AB049320AB03931FAB02935B4601931B
:107B10000223424600930898099B00F0B3FC139B94
:107B20001290672B00D0D6E3129B1A005A4414001F
:107B3000EA0700D4D2E10023002240460999F8F771
:107B40006BFB2300002809D1239B3021A34205D2DF
:107B50005A1C23921970239B9C42F9D8129A9B1AA3
:107B600018931F9B15934B46472B00D1BEE1139BE7
:107B7000662B00D0C2E1159B002B00DC64E35B4662
:107B8000002B00D053E3EB0700D550E3159B09937E
:107B90000D93119B002B00D0E0E116ABDB7F9946E3
:107BA00000239B46FFF763FA1D1E00DDA0E6ABE64F
:107BB00042467B684F4D102A00DC32E1102291468C
:107BC0002200444604E00836103C102C00DC26E17C
:107BD00049461032013335607160BA607B60072B13
:107BE000F1DD3A000799089802F0A0FA002801D0C8
:107BF000FFF746F9BA687B6832AEE5E7402108989E
:107C000001F0F6FB079B18601861002800D169E3BA
:107C10004023079A5361FFF7CEF83A000799089876
:107C200002F084FA002801D0FFF72AF97B68BC68CB
:107C300001330D9332AB34AE9946FCE44346013236
:107C40001D431378FFF701F93A000799089802F0ED
:107C50006DFA002801D0FFF713F9BC6832AE36E5A3
:107C60005B460993062B00D9F1E0099B10940D9314
:107C7000002399469B4615931F4B0A951293FFF7D5
:107C8000C3FA129A32AB9B1A0D93FFF7E8F91A9ACE
:107C90003260199A944672607A6864440132BC601A
:107CA0007A60072A00DD75E108363FE632ABB04660
:107CB0000E9C0F9D1E00200029000A220023F8F7C9
:107CC000FDFA013E303232700023200029000A22E2
:107CD000F8F7F4FA030004000D000B43EBD1320077
:107CE00032AB9B1A12960E940F9546460D93FFF7F2
:107CF000B6F9C046ECCF0008D0CF00080C9A1A6045
:107D0000FFF76AF83A000799089802F00FFA00287E
:107D100001D0FFF7B5F816ABDB7FBC68994632AEF1
:107D2000FFF7B9FA3A000799089802F0FFF900281E
:107D300001D0FFF7A5F832AABC687B6891464AE5F6
:107D40003A000799089802F0F1F9002801D0FFF7EE
:107D500097F87B68BC68984632AB99464DE5012B95
:107D600001D0FFF74FF9FFF727FAA046140042466B
:107D70004444013335607260BC607B60072B01DCDA
:107D8000FFF7FAFA64E43A000799089802F0CEF98E
:107D9000002801D0FFF774F8BC6832AEFFF7A2FAF2
:107DA000D64B01343360012373607B68BC600133C0
:107DB0007B60072B00DD18E10836002902D1189BF3
:107DC000002B47D01A9B3360199B9C4673607B68DD
:107DD00064440133BC607B60072B00DD4CE1320062
:107DE0000832002900DA82E11299013311601899F2
:107DF0007B608C4664445160BC60072B00DD27E447
:107E000008321600FFF7B9FA3A000799089802F00D
:107E10008DF9002801D0FFF733F832AE3EE4A046DA
:107E2000140042464444013335607260BC607B609C
:107E3000072B00DD3CE108366FE5129802F044F9AB
:107E40000200FFF778F9AE4B1293FFF77EFB062393
:107E500009930AE70A9BDB0701D4FFF78EFAB1E723
:107E60005B46002B00D033E601239B4630E65B46A1
:107E70005A1C23AB049320AB03931FAB0293022342
:107E80000D92019200934246099B089800F0FAFA7D
:107E90001290139B472B00D003E2EB0700D4ECE1D8
:107EA0000D9A129B944663441C00139B462B00D0F2
:107EB00041E6129B1B78302B02D01F9BE4183AE658
:107EC0000022002340460999F8F7A6F90028F4D1CA
:107ED00001230D9A9B1A1F93E4182CE6239AD31AB8
:107EE00018931F9B15934B46472B07D1159BDA1C04
:107EF00001DB9B453ADA139B023B13936A464C2104
:107F0000159B521812785C1E21AB1F9499461A706B
:107F1000002C00DA6CE12B234A465370092C00DD5B
:107F200011E130234A4630349370D47022AB4A4674
:107F30009B1A189A9C46110061441B930D91012ACB
:107F400000DC5CE1199B0D9A9C466244D343DB172D
:107F50000D921A400023099215931AE62D2316AAB2
:107F6000D377994600239B46FFF785F8159B189910
:107F70008B4200DA8EE0EA0700D42FE1199B159AB4
:107F80009C4662440D92D343DB171A406723099243
:107F90001393FEE53A000799089802F0C7F8002805
:107FA00001D0FEF76DFF1F9BBC6832AEBEE43A0005
:107FB0000799089802F0BAF8002801D0FEF760FF90
:107FC000BC6832AEA0E42D2316AAD3779946FFF7FA
:107FD000B5FA8022169B179C1206984694462300F9
:107FE000634409932D2311937FE53A00079908987C
:107FF00002F09CF8002801D0FEF742FF1F99BC68F0
:1080000032AEDAE623AB049320AB03931FAB0293AB
:108010005B4601930323424600930898099B00F0B6
:1080200031FA03005B441C005B4612900D9340E75D
:108030003A000799089802F079F8002801D0FEF775
:108040001FFF189B1F9ABC689B1A32AE87E40A9ADE
:1080500092465246FEF73AFF06239B4638E516AB9A
:10806000DB7F109499465B4609930D9300230A9594
:108070009B461593FEF7FBFF3A000799089802F01C
:1080800055F8002801D0FEF7FBFE1F99BC687B68FD
:1080900032AAA6E6199B189A9C46159B62440D923B
:1080A000002B00DD6FE7159A0D9B981A421C69E7BB
:1080B0003A000799089802F039F8002801D0FEF735
:1080C000DFFEBC6832AE28E423AB049320AB0393FD
:1080D0001FAB02935B46019303234246009308982B
:1080E000099B00F0CFF95B4612900D93D8E64E4203
:1080F000044D103168DA1021884609E0D8CF000815
:108100009CCF0008ECCF00080832103E102E5BDD3B
:1081100041461034013315605160BC607B60072B11
:10812000F2DD3A000799089802F000F8002801D023
:10813000FEF7A6FEBC687B6832AAE6E701235B4235
:108140000C93FEF7A3FE16AA3B2394466344B34662
:10815000A8461E0000E02E0020000A21F8F740F893
:10816000751E3031297020000A21F7F7EFFF040057
:108170000928F0DC32002B0016A95E4645469346DE
:1081800098468C4613003B223034E4B2023B6244F2
:108190001C709A4200D899E03B235A4663449A1ACD
:1081A000012358465B4201E0C45C01334946C918CB
:1081B000CC709A42F8D116A98C462E2243466244CE
:1081C0009446FB1A6344B2E6A41901331560566065
:1081D000BC607B60072B57DC083205E61A00DB43E6
:1081E0001100DB171940672309910D921393D0E416
:1081F0000124159B4A46E41A2D2353708EE6012371
:108200002B40159300D09DE6CB430A00DB171A40A4
:108210000992BEE4179B002B27DB16ABDB7F994648
:10822000139B472B1DDC3F4B1293FFF78EF9199AD6
:10823000159B94466344180002005A44D343DB174D
:108240000D921A400992A4E45B46002B12D1EB0771
:1082500010D4012309930D939BE43300324DFFF7B3
:10826000DAF9324B1293FFF770F92D2316AAD37760
:108270009946D5E7199B581CDEE7239B129A9B1A57
:1082800018931F9B159331E63A000799089801F05F
:108290004DFF002801D0FEF7F3FDBC687B6832AAD1
:1082A000A2E5129A0D9B944663441C0043E4109B84
:1082B0000999181D1B689B46002B02DA01235B42BB
:1082C0009B46537810900A9AFEF7BFFD16AA2E23FC
:1082D000944663442BE65B460D93DAE516ABDC77F8
:1082E000FFF751F90C23089A13600D3B0C93FEF72E
:1082F000CDFD16ABDC77FFF760F916ABDC77FFF747
:108300009BF816ABDC77FFF7ECF816ABDC77FEF7E3
:108310004AFE16ABDC77FEF728FF16ABDC77FEF7DC
:10832000E0FDC046A0CF0008ECCF0008A4CF0008B5
:10833000F0B5454680465746DE464E464346E0B5D4
:108340001B690D6985B00F000020AB4200DA92E096
:1083500014239C468C446246013DAB000292D61821
:10836000142242449146994433680192591C4B4669
:108370001868F7F7A5FE041E46D0029A002392461D
:10838000002001994A46A446B1465446BB46AA4637
:1083900006000D001F000392634604CC1004000C7D
:1083A0005843120C5A43C019030CD2182B6800040E
:1083B0001904090C8919170C000C1204091A120C63
:1083C0001B0C9B1A0A149B1809041E14090C1B048D
:1083D000194302C5A145DFD2039B4E4699461B684F
:1083E000644655465F46002B0ED14B46019A043B2E
:1083F0009A4204D306E0043B013D9A4202D2196836
:108400000029F8D043461D613900404601F040FD87
:1084100000282FDB029B01340020A4461900019F95
:108420003B6810C91A04120C10182204120C821A8C
:108430001B0C200C1B1A10141B1812041814120CFD
:108440001B04134308C78E42EAD2019A644694463D
:10845000AB006344196800290CD1043B9A4204D351
:1084600006E0043B013D9A4202D219680029F8D087
:1084700043461D61200005B03CBC90469946A2468B
:10848000AB46F0BDF0B557464E46DE464546E0B534
:1084900016001F00016C9DB004000296039700298E
:1084A00008D00123426C93404A608B6001F0CCFA03
:1084B000002323643D1E00DAB8E10023299A1360EB
:1084C0002A00CC4B1A409A4200D1BBE1029E039F86
:1084D0000022002330003900F7F79EFE002813D059
:1084E0000123289A13602A9B002B00D1D4E1C24BB0
:1084F0002A9A1360013B9A4650461DB03CBC9046F8
:108500009946A246AB46F0BD1AAB01931BAB009354
:1085100032003B00200001F067FD2B0D834600D0A8
:10852000ADE11A9B98461B9B43441E00B34BF318C6
:10853000202B01DC00F096FC4022D31A9D40B04B6A
:108540000298F318D840284304F0A8F90123AD4D50
:1085500016934919751E0022AB4B03F03DFEAB4A42
:10856000AB4B03F013FCAB4AAB4B02F0BFFD060074
:1085700028000F0004F05EF9A84AA94B03F006FC9E
:1085800002000B003000390002F0B0FD06000F00C1
:1085900004F01CF900220690002330003900F7F7A0
:1085A00041FE00280DD0069B1800994604F042F9C0
:1085B0003B003200F7F730FE434258414B461B1A4E
:1085C00006930123069E0A93162E10D89549F300B0
:1085D000C91808684968029A039BF7F737FE002814
:1085E00001D100F045FC0023013E06960A93434664
:1085F0005D1B002304932B00013B984604D5012307
:108600005B1B049300239846069B002B00DA8AE24A
:108610009C46099300239946E044269B092B00D9E8
:108620003DE10126052B02DD0026043B2693269B17
:10863000032B01D100F043FD01DC00F0F9FC269B87
:10864000042B01D100F06EFC01230893269B052B1F
:1086500001D000F0F3FC279A069B944663440B93E9
:10866000013307931F1E00DC01270023079D63646D
:108670000021172F00DC20E1012204335B001800E9
:10868000143011000132B842F8D96164200001F0C1
:10869000B3F9824620640E2D00D816E11B9B002BF7
:1086A00000DA22E2069A0E2A00DD1EE25D4BD200BD
:1086B0009B181A685B6804920593279B002B01DACC
:1086C00000F03BFC029E039F049A059B300039009A
:1086D00002F0E4FF04F07AF8814604F0ABF8049A63
:1086E000059B03F053FB02000B003000390003F040
:1086F00073FD53465D1C4B46524630331370079B47
:1087000006000F00012B45D00022474B03F03EFB33
:108710000022002306000F00F7F77EFD002800D09E
:1087200069E30222079B5244534402931500A14679
:108730000EE000223C4B03F029FB00220023060040
:108740000F000135F7F768FD002801D000F0C2FCEA
:10875000049A059B3000390002F0A0FF04F036F8BF
:10876000040004F067F8049A059B03F00FFB020075
:108770000B003000390003F02FFD22006B1E303259
:108780001A70029B06000F00A846AB42D1D14B469F
:10879000A1461C0032003B003000390002F0A6FC6C
:1087A000049A059B06000F00F7F750FD00280CD136
:1087B000049A059B30003900F7F72EFD002800D100
:1087C00019E34B46DB0700D415E36B1E19785046BE
:1087D00007E0984201D100F002FD023D29781D001A
:1087E000013B1A003929F4D082460291029E0136DB
:1087F000167000E30000F07FD9CF000832040000BB
:1088000012040000000010FE0000F83F61436F6397
:10881000A787D23FB3C8608B288AC63FFB799F5099
:108820001344D33F48D00008000024400123299A74
:108830007D006D0813602A00BF4B03951A409A42D1
:1088400000D043E6BD4B289A1360029B002B0CD14D
:108850002D030AD12A9B002B01D100F0ABFDB84BB0
:108860009A4608332A9A136046E62A9B002B02D1C7
:10887000B44B9A4640E6B34B9A460333F2E73A03C9
:10888000B14D120B1543B14A29009D181A9B3000B7
:108890009846002316935EE6AD4B9A462CE60125DA
:1088A0000023012201266D42269308920795279303
:1088B000002300216364079B0B93200001F09CF8C8
:1088C000824620640E2D00D9E8E6002E00D1E5E6B0
:1088D000029A039B069F0E920F93002F00DC52E337
:1088E0000F213B000B40DA009A4B9B181D685E6815
:1088F0000C950D963D11EB0601D400F008FC964B4B
:108900000D401A6A5B6A0E980F9902F0C7FE0323A6
:10891000109011910293002D18D00C980D992300FE
:1089200001274C4699468C4E2F4206D0029B0133BC
:1089300002933268736803F029FA6D100836002D2F
:10894000F2D14B46A1461C000C900D910C9A0D9B48
:108950001098119902F0A2FE0C900D910A9B002B29
:1089600009D00C980D990022774BF7F75BFC002893
:1089700001D000F082FC029803F05CFF0C9A0D9B82
:1089800003F004FA754B002202F0B0FB744B0500B3
:10899000CE18079B002B00D16FE3069B1893079B13
:1089A00010930C980D9903F011FF12951396060081
:1089B000109D684B6A1ED2009B18303619685A68A1
:1089C000F3B256460136149115920293179603F0AE
:1089D00031FF02000B000C980D9903F0FDFB149A77
:1089E000159B060008980F00002800D1ADE3002079
:1089F0005C4902F053FE129A139B03F0EDFB6B46A9
:108A000052461B7A0C900D91137032003B00F7F721
:108A10001DFC002801D000F0BDFC32003B0000200E
:108A2000494903F0D9FB0C9A0D9BF7F7FBFB002893
:108A300001D000F0B1FC012D00D178E34A46149238
:108A4000424619925A46179B554402951294109229
:108A500099460C9C0D9DD34612E032003B0000204D
:108A6000394903F0B9FB22002B00F7F7DBFB0028A4
:108A700001D000F065FC029BD146534500D14EE386
:108A80000022394B2000290003F080F90022364BE8
:108A900004000D003000390003F078F90F000600E3
:108AA00003F094FE804603F0C5FE02000B00300088
:108AB000390003F091FB01234B449A46434630337F
:108AC000DBB298464B4642461A7022002B00060045
:108AD0000F00F7F7A7FB0028BFD0109B5546DA46DA
:108AE0009B46189B129C069385E1089A002A3DD06C
:108AF000269A012A00DC05E2079B5D1E4B46A9452C
:108B000000DAEAE25D1B079B002B00DA15E39C46C6
:108B1000049AE0441700624404920121200001F00D
:108B20002DF8060025E0049A069BD21A5B4299466E
:108B300000230492099370E50000F07F0F270000E6
:108B4000FCCF000808D000080000F03F01FCFFFF48
:108B5000D8CF000848D0000820D0000800001C40F2
:108B60000000C0FC0000E03F000024404D4600260D
:108B7000049F002F0DDD4346002B0ADD3B004745D7
:108B800000DD92E1049AFF1AD21A04924246D31AE7
:108B900098464B46002B0ED0089B002B05D04B4629
:108BA0005B1B9946002D00D081E159464A462000C2
:108BB00001F0AAF883460121200000F0DFFF099AA6
:108BC0008146002A00D037E1269B012B00DC53E1CF
:108BD00001231F204344184000D12BE120231B1AFE
:108BE000042B00DCE0E31C23181A049B3F189C466E
:108BF0008444634680440493049B002B05DD59465E
:108C00001A00200001F0E0F883464346002B05DD02
:108C100049464246200001F0D7F881460A9B002BC6
:108C20007AD1079B002B00DCF5E1089B002B00D1DB
:108C300090E0002F00DD50E1099B0496002B00D04E
:108C4000D0E1079A53469446013B9C4463460893FF
:108C50000123029A5D461A405346D046CB460792FE
:108C60000A9359462800FFF763FB0300099030334D
:108C700031002800029301F00BF9049A07005946CD
:108C8000200001F01FF9C3688146002B00D0CEE020
:108C90000100280001F0FCF882464946200000F05F
:108CA000D3FE5246269B134303D1079B002B00D1D2
:108CB00025E3002F00DA19E2269B1F4303D1079B0F
:108CC000002B00D112E243465F1C5346002B00DD0F
:108CD000A2E26A464346127A1A70089B434500D1C5
:108CE000A9E2002329000A22200000F0B7FE049B1D
:108CF00005009E4200D190E0310000230A222000AE
:108D000000F0ACFE002306000A220499200000F0C7
:108D1000A5FEB8460490A4E74946584601F0B8F8C5
:108D2000002800DB7DE7069B5946013B06930A229B
:108D30000023200000F092FE089B8346002B00D009
:108D400012E30B9B002B04DC269B022B00DD35E39A
:108D50000B9B0793079B5746984623005C46B346F8
:108D60004E46994607E0210000230A22484600F0BB
:108D700075FE2F00040031002000FFF7D9FA53469A
:108D800030307D1C3870EB1A4345ECDB4B46002736
:108D9000B1465E46A3461C000290012259462000BF
:108DA00001F012F84946834601F072F86B1E1A78FA
:108DB000002800DC98E0514606E0994200D182E1AB
:108DC000023D2A781D00013B392AF6D08A4601323D
:108DD0001A704946200000F037FE002E0BD0002FFD
:108DE00005D0B74203D03900200000F02DFE31003D
:108DF000200000F029FE5946200000F025FE002347
:108E00002B70069B289A013313602A9B002B01D1FB
:108E1000FFF772FB1D60FFF76FFB310000230A2292
:108E2000200000F01BFEB8460600049019E701235D
:108E30009A4632E71C20D8E60100200000F064FFCB
:108E4000269B8146012B00DCE0E0002309934B4682
:108E50001B6903339B004B44586800F045FE2023F8
:108E60001B1AB6E620220298D31A9840FFF76CFB33
:108E700000230A93FFF7BBFB029B002B00D0A7E661
:108E80000298039900220B0309D1DA4B0B4206D05A
:108E9000049B01320133049301239C46E044099B67
:108EA0000992002B00D193E6D1E743466AE62A00F7
:108EB0003100200000F028FF5A4601000600200083
:108EC00000F066FE59460500200000F0BDFD4B464F
:108ED000AB46002B00D16EE667E631003A00200079
:108EE00000F072FF0600A7E6002808D10299C90722
:108EF00000D560E703E0023D2A781D00013B302ADF
:108F0000F9D066E7169A002A00D19CE1BA4A944645
:108F10006344049A984494469C4463464D46170023
:108F20000493FAE501230893279B002B00DCC0E0A3
:108F30000B9307931F00FFF798FB079B002B01DDA6
:108F4000FFF7C0FB00D0B0E0049805990022AB4BBE
:108F500002F01CFF029A039BF7F782F90023002618
:108F6000994600285FD1534652465D1C3123137049
:108F7000069B013306934946200000F065FD002E54
:108F800000D034E737E7069B002B00D16DE10E9847
:108F90000F995D420F239A4A2B40DB00D3181A68C1
:108FA0005B6802F0F3FE2D110C900D91002D00D1A5
:108FB000ECE1022200230127924E02922F4207D0B9
:108FC000029B013302933268736802F0DFFE0123D3
:108FD0006D100836002DF1D1002B00D1BEE40C90AD
:108FE0000D91BBE47168200000F006FD3100050022
:108FF00033690C319A1C92000C30FDF795FD01226B
:109000002900200000F0E0FE04901AE6029B002BED
:1090100000D135E719E7269B022B00DC05E6079B0C
:10902000002B00D113E1279B5546DB430693A2E7B3
:1090300000230893269B022B00D175E70023002113
:109040006364200000F0D8FC0023279301330893C9
:10905000023B824620640B930793FFF71FFB0298A5
:1090600003F0E8FB0C9A0D9B02F090FE664B002289
:1090700002F03CF80500654BCE1800220C980D99C3
:109080005E4B03F0A9F82A00330002900391F7F732
:10909000DDF8002855D18021090673182A000298AE
:1090A0000399F7F7BFF8002841D00023002699461E
:1090B000B9E70123012507932793FFF7F9FB002365
:1090C0000893FFF7C8FA069B8A46013306933123BB
:1090D0000B707EE645464C468DE6EE1A099BA94686
:1090E0009C46B4446346002509930CE50A9A53460E
:1090F00092464246D946AB46551C002B00DDE3E0C4
:109100006A464346127A37001A70049E61E60E9A48
:109110000F9B1092119302230293FFF7FCFB149B09
:10912000DA469946199B129C9846109B9B460E9ACC
:109130000F9B02920393FFF7B1FA049B079A9F1AC1
:10914000EBE40023002699460DE71298139902F0EC
:109150001DFE6A465346127A0C900D911A70109BB0
:10916000179D012B27D0109B534402934B46C146B9
:10917000A0462C0010930022254B3000390002F04D
:1091800005FE0F00060003F021FB050003F052FB73
:109190000B0002003900300003F01EF83035029B4E
:1091A0002570013406000F00A342E4D1109B444611
:1091B000C8469946029D00220C980D99154B01F066
:1091C00095FF32003B00F7F72DF8002800D1A2E010
:1091D000189A6B1E197806925046FFF702FB069B01
:1091E0008246013306933023020003700293FFF797
:1091F000FDFAC0460000F07F330400000000144078
:1092000048D0000820D0000800001C400000C0FC2E
:10921000000024400000E03F0A9BD9469A46029B8A
:10922000AB463D00392B61D04246029B37000133EB
:109230001370049ECDE50A9BD9469A46AB463D0085
:109240003700049EA9E536231A9A9B1A61E649461F
:109250000522200000F002FC81460100584600F083
:1092600017FE002800DD7EE6DDE60E9A0F9B0C92CD
:109270000D9302230293FFF771FB079B002B00D194
:10928000EDE60B9F002F00DC51E70C980D99069B33
:109290000022013B18934B4B02F078FD05000E00B5
:1092A00002980C950D96013003F0C4FA2A003300A1
:1092B00002F06CFD444B002201F018FF434B050007
:1092C000CE181097FFF76DFB59460122200000F0E1
:1092D0007BFD4946834600F0DBFD00283CDD029B18
:1092E000392B03D0099B3133029309E739234246D6
:1092F00037001370049E39226B1E514664E50A9BA9
:10930000D9469A464346AB465D1C029B392BEDD0AD
:10931000002FE7DCF4E60C9A0D9B00202C4902F0AC
:109320005BFF32003B00F6F791FF002801D1FEE61B
:109330001D006B1E1A78302AFAD0189B06935AE546
:109340005546DA46109A4B469346189A4146129C67
:1093500006925046FFF745FA002800D0D0E6029B5F
:10936000DB0700D4CCE6BAE7002331000A22200054
:1093700000F074FB0B9B0600002B01DD079358E403
:10938000269B022B1ADC0B9B079352E402230293C9
:10939000FFF7E4FA179DD0E7189B179D06930299F3
:1093A00053465046FFF71DFA042B00D124E43C231A
:1093B000181A1AE4074B9A46FFF79EF80B9B07937F
:1093C0002DE6C0460000244000001C400000C0FC08
:1093D0000000E03FFCCF0008034B1B68586B0028DF
:1093E00000D10248F0307047B4000020E0040020B3
:1093F000F0B557464546DE464E46E0B50D000B3506
:1094000083B00700162D28D8102900D9C1E000F03C
:10941000EFFA102518230220CC4EF3181A005C68CE
:10942000083A944200D15BE1032362689A43130037
:10943000E268A168CA6091600122E31859683800A7
:109440000A435A6000F0D6FA2000083003B03CBC52
:1094500090469946A246AB46F0BD07239D4300D5F2
:1094600097E0A94200D994E000F0C2FAF823FF3354
:109470009D4200D859E1680A00D18EE0042800D945
:1094800034E138239846A80980443930C100AF4EF2
:1094900071180839CC68A14218D0032362689A4336
:1094A0001300521B0F2A00DD18E1002AC0DA032343
:1094B0009C4608E06246636893435A1B0F2A00DD0E
:1094C0000CE1002AB4DAE468A142F3D13200346935
:1094D0000832944267D00323616899438A460B009F
:1094E000491B0F2900DD0DE1726132610029A3DA09
:1094F000974A924500D94AE1DB08FF3A9910FF3AB2
:109500008A40DB0071689B190A4399687260E360C6
:10951000A1609C60CC60012183109940914248D8A1
:109520000A4205D103239843490004300A42FBD084
:1095300003239846C3009946B144CC46824663460D
:10954000DC68A44507D1F4E0002A00DB10E1E46800
:10955000A44500D1EDE04246636893435A1B0F2AAD
:10956000F2DD01208046611905436560A068E56869
:109570000836C560A8604046F160B160104348609D
:10958000CE608E603800E25000F034FA20000830DF
:109590005CE70C2300203B6058E780213F238900D3
:1095A0004020984673E701217268831099409142E8
:1095B000B6D90323B46862689A439046AA4202D39C
:1095C000531B0F2B7CDC634A634B93461B6812686A
:1095D000EB18013200D13BE1604A944663441B0B17
:1095E0001B0301930199380000F05CFD03008146E4
:1095F000013300D1F9E04346E318834200D9F2E099
:10960000574A019992461268944652466144116045
:10961000834200D13EE15A461268013200D155E141
:109620004A46D31A59185346196007234A4613402D
:1096300000D123E1082189464A49D21A9144CB1A24
:10964000019A38004A441105090D5B1A19009B461E
:1096500000F028FD431C00D134E14B46C01A012321
:109660005844184353461B685B441900534619601D
:109670004B46B3605860B44212D043460F2B00D81B
:109680001CE1072260680C3B9343063A0240052028
:109690001A436260E218506090600F2B00D933E1EA
:1096A000314B1A68914200D919600323B46862688B
:1096B0009A432E4B1868814200D89AE0196098E0CE
:1096C0000122290013431143651961603800B56018
:1096D0006B6000F08FF920000830B7E64046F5E6F1
:1096E000DC680230A34200D1F0E69DE6142874D96C
:1096F000542800D9AFE06E239846280B80446F3081
:10970000C100C4E6012360191D43656070613061CA
:10971000C26082601A0053460A4342603800E1503A
:1097200000F068F92000083090E62B00E8080833C4
:1097300072E608239B46073BDC449B46DA444346DB
:109740005246134200D0FAE66DE0C0464C060020B7
:10975000FF010000540A00207C0F00200F100000C1
:109760004C0F002008100000740F0020780F00201C
:109770000122E318596838000A435A60E368A26876
:10978000D3609A6000F036F9200008305EE65A0A8D
:10979000042A39D9142A74D85B23984690445C3241
:1097A000D20008235B429C46B218944463469968F1
:1097B000032399468C4559D04B464A689A435245F3
:1097C00002D989688C45F7D1CB6872689C4663469C
:1097D000A160E3609C60CC609DE65B23984680447A
:1097E0005C30C10053E6B44274D00323B4686268AD
:1097F0009A43531B954202D80F2B00DD60E73800D7
:1098000000F0F8F8002021E69A09382398469044A1
:109810003932D200C5E74B461A68083B01389146F9
:109820009A4200D087E043460342F4D173688B43E9
:1098300073604900994200D9BBE6002904D1B8E61B
:10984000042294464900E2440B42F9D0504671E6A6
:1098500010330193C6E6AA235B00984224D8DD3B6F
:109860009846E80B80447830C10010E64346012258
:109870009B109A4073681A437260A8E780235B01CB
:10988000DEE6542A2FD81A0B6E23984690446F3286
:10989000D20086E71A0500D0BDE60120019BB26820
:1098A000434403435360FBE6244B984226D87C2371
:1098B0009846A80C80447D30C100E8E501234A4663
:1098C00053609CE7002301209B46CBE65B464A465B
:1098D0001A60AAE61A4A01999246126894465246BC
:1098E0006144116097E6AA2149008A4214D8DA0B34
:1098F0007723984690447832D20052E7FE217E23A7
:1099000089007F209846C2E521003800083100F028
:1099100023FD53461968C3E608498A4206D89A0CC3
:109920007C23984690447D32D2003AE7FE227E2383
:109930009200984635E773687BE7C04654050000FF
:109940004C0F002082B000290AD0002A0BD0002B37
:109950000BD013780B601078431E984102B070470B
:1099600001A9002AF3D10020F8E702204042F5E7E0
:1099700070B5CCB2830734D0531E002A1BD00278B6
:10998000A24219D0032504E0013B14D30278A2427D
:1099900012D001302842F7D1032B0ED8002B0AD069
:1099A0000278A24208D0C31802E00278A24203D093
:1099B00001308342F9D1002070BDFF220D062D0C2D
:1099C000114029430D04084E0D43026807496A40BF
:1099D000511891433142E3D1043B0430032BF4D8B6
:1099E000DCE71300D8E7C04680808080FFFEFEFEE3
:1099F0007047C0467047C04670B50400C06C0D008B
:109A000000280AD0AB00C318186800280FD00268DD
:109A10001A6000230361C36070BD2122042120006D
:109A200000F01EFCE0640028ECD10020F4E70126E1
:109A3000AE40721D92000121200000F011FC0028B0
:109A4000F3D045608660E4E7002906D04B689A00B1
:109A5000C36C9B181A680A6019607047F8B5CE4647
:109A600047468146080080B50D000C691F000021A3
:109A70001430036801311E04360C56431B0C53434B
:109A8000F619370CDB1936041F0C360C1B049B1916
:109A900008C08C42EDDC002F08D0AB68A3420ADD81
:109AA000231D9B00EB1801345F602C6128000CBC67
:109AB00090469946F8BD6B684846591CFFF79CFFD5
:109AC00029002B6980469A1C92000C310C30FDF75E
:109AD0002BF86B689A004B46DB6C9B181A682A605F
:109AE0001D604546DCE7C0460300020C0020002A4A
:109AF00001D11B0410301A0E01D108301B021A0FBD
:109B000001D104301B019A0F01D102309B00002BC0
:109B100002DB5B0001D5013070472020FCE7C04626
:109B200003685A0709D00022D90704D49A071ED522
:109B300001225B080360100070471904002200290D
:109B400001D11B0C1032FF21194201D108321B0A2E
:109B5000190701D104321B09990701D102329B0870
:109B6000D90702D45B0806D001320360E3E79B0803
:109B700003600222DFE72022DDE7C04610B50C00BB
:109B80000121FFF739FF01234461036110BDC04685
:109B9000F0B557464E464546DE46E0B514690E69B7
:109BA00085B00F001500A64204DA33001700260026
:109BB0000D001C0033199846BB687968434500DAEC
:109BC0000131FFF719FF14220300944663449A46BB
:109BD00043469B0019005144029003918A4504D2E8
:109BE0005346002204C39942FCD83B0014339C46E0
:109BF00001931423B2006244A4009C462300AC44A9
:109C0000634400939C4562D2914608E0240C32D113
:109C100004239B46009BDC44DA44634557D96346E2
:109C20001C682604360CF1D0554600224C46019F94
:109C300002CF28680B041B0C73430004000C1B1894
:109C4000994691442A680B0C100C4A4649467343C6
:109C5000120C1B189B1809041A0C090C1B040B434B
:109C6000AB4608C5BC42E3D85B465A606346A14692
:109C70001C68240CCCD0534600221B684946504631
:109C80001E009146019D2A88360C624392194A446F
:109C90001B0416041B0C33434668036037043F0C57
:109CA000B94608CD120C1B0C63434B449B181A0C8D
:109CB000834691460430A942E5D85F467B60042381
:109CC0009B46009BDC448946DA446345A7D843465B
:109CD000002B0EDD039B043B1A68002A09D1424683
:109CE00003E0043B1968002902D1013A002AF8D1A7
:109CF0009046029B424618001A6105B03CBC904653
:109D00009946A246AB46F0BDF8B54746CE4603237A
:109D100080B588460700140013403AD1A410464687
:109D200026D0BD6C002D3DD0012346469846002329
:109D300099464346234208D1641019D02868002868
:109D40001BD0050043462342F6D02A0031003800DC
:109D5000FFF71EFF002E1AD0FA6C736894469B0022
:109D600063441A68641032601E600600002CE5D15E
:109D700030000CBC90469946F8BD2A0029003800F6
:109D8000FFF706FF4B46286003600500DAE7060090
:109D9000D2E70B4A013B9B009A580023FFF75EFE77
:109DA0008046BBE701213800FFF726FE054B050082
:109DB0004361012303610023B8640360B4E7C04634
:109DC00010D1000871020000F0B5DE4657464E463D
:109DD0004546E0B50D002B6956119B46B3445B46E2
:109DE0005C1CAB6883B00190170049689C4203DD9E
:109DF00001315B009C42FBDC0198FFF7FDFD030095
:109E000084461433002E06DD0022B100591804C325
:109E10009942FCD10B0029692A008E001F211432BF
:109E2000394096198946002929D020214846091A27
:109E3000884600271900484613688A4683403B43FA
:109E400008C1434680CADF409642F4D853465F605B
:109E5000002F01D05C46023463466046013C1C6121
:109E60006B689A00019BDB6C9B181A682A601D6066
:109E700003B03CBC90469946A246AB46F0BD02CA30
:109E800002C39642E8D902CA02C39642F7D8E3E772
:109E90000A69036930B50500981A12D19200143589
:109EA0001431AB18891801E09D420AD2043B0439F1
:109EB0001C680A689442F7D0944280410123984379
:109EC000013030BDF8B5454657464E461400DE46D3
:109ED000E0B50E00250013690A698846D71A1436C2
:109EE0001435002F16D19B00F218EB1802E0B24295
:109EF00000D86FE0043A1168043B8C4619688C4521
:109F0000F5D00AD233002E001D0043460127A0469B
:109F10001C0002E0002FF5DB002743465968FFF7DD
:109F20006BFD434681461B69C7609C4698002369C8
:109F300082469B0098464F46B244A84414370020FE
:109F400000E0260004CD34009346594608CC0904AD
:109F50001A04120C1218090C521A190C5B461B0C2D
:109F6000CB1A11145B1812041814120C1B04391D9F
:109F700013433B600F00A845E3D8A24515D908CC90
:109F80001A04120C121815141B0C5B191204181465
:109F9000120C1B04134308C7A245F0D85246961B67
:109FA000053EB6080136B60089190439002B07D1E1
:109FB00001235B42984604390B68C444002BF7D058
:109FC0004B4662461A6148463CBC90469946A246BA
:109FD000AB46F8BD0021FFF70FFD0123036100230D
:109FE00081464361EFE7C046F0B501211C0083B014
:109FF0001500089FFFF700FD2303640006001B0BFC
:10A00000640D02D08022520313430193002D19D016
:10A0100068460095FFF784FD002830D1009B019D24
:10A020007361B5616B1E9D4101353561002C14D003
:10A03000194B9C46352364442418181A099B3C602C
:10A04000186019E001A8FFF76BFD019B20307361D8
:10A05000012301253361002CEAD1104B9C46104BA3
:10A060006044EB189B00F31838605869FFF73CFD1B
:10A070006D01099B281A1860300003B0F0BD019DE6
:10A0800020232A001B1A9A401300C540009A01950C
:10A0900013437361C5E7C046CDFBFFFFCEFBFFFF57
:10A0A000FFFFFF3F002370B5064C0500080023604A
:10A0B00000F0EAFD431C00D070BD2368002BFBD0EC
:10A0C0002B60F9E7840F002010B5040083070AD045
:10A0D0000378002B23D0032202E00378002B1CD04E
:10A0E00001301042F9D102680E4B0F49D318934347
:10A0F0000B420FD1043002680A4BD31893430B4232
:10A1000008D104300268074BD31893430B42F1D0B7
:10A1100000E001300378002BFBD1001B10BD0020B4
:10A12000FCE7C046FFFEFEFE80808080F0B557460B
:10A130004E46DE464546E0B5936883B001900E007A
:10A140009246002B6CD0136808688D681F0044E0AD
:10A150009022B389D20013422ED03169421A93461D
:10A16000706942001218D00F8218601C52105844B7
:10A170009046904201D9804602008020C0000342F0
:10A1800037D011000198FFF733F9051E53D05A4616
:10A190003169FCF7C9FCB389294A13408022134373
:10A1A000B381434628005A463561A04625005844ED
:10A1B00073619B1A3060B3604246494600F0B6F9BD
:10A1C000B3685D1B3368B560434433601800534681
:10A1D0009B681C1B53469C6022D03B687C68994658
:10A1E0000837A846002CF8D0AC42B1D22500A046D2
:10A1F000E2E7019800F0E8F9051ED2D1019C31692F
:10A20000200000F0A9F80C2323604022B38901202C
:10A210001343B3815246002340429360536003E0EE
:10A22000002352460020536003B03CBC9046994640
:10A23000A246AB46F0BD0C23019A1360E5E7C04689
:10A240007FFBFFFF002904D0FF2A04D801200A70F9
:10A2500070470020FCE78A23036001204042F7E7B3
:10A2600010B55143FFF7C4F8041E1CD00300083B8F
:10A270005A6803239A43043A242A16D80300132A5F
:10A280000DD900210833016041601B2A07D9816084
:10A29000C160242A0DD103000161183341610022FD
:10A2A0001A605A609A60200010BD0021FCF780FC03
:10A2B000F9E703001033F2E7F8B50C000600FFF7EA
:10A2C00097FB204FBB685D6803239D431E4B2C1BEF
:10A2D0009C466444240B1D4B013C24039C4207DD37
:10A2E00000213000FFF7DEFEBB685B19984204D006
:10A2F0003000FFF77FFB0020F8BD61423000FFF720
:10A30000D1FE431C0DD00122BB682D1B15435D609F
:10A310000F4B30001A68141B1C60FFF76BFB012009
:10A32000EAE700213000FFF7BDFEBA68831A0F2B61
:10A33000DEDD08490968401A0549086001210B4320
:10A340005360D5E74C060020EF0F0000FF0F000020
:10A350004C0F0020540A0020F8B5CE4647460500B1
:10A3600080B50C1E55D0FFF743FB210008394F681C
:10A37000012438000323A0430A1856689E43B146BF
:10A38000644EB368934229D04B465360D3189C4621
:10A390003C4242D10F68C91B8B68C019984663467E
:10A3A0005F6808239C46B4442740E0456AD0434692
:10A3B000CC68DC60A360002F32D101244844044300
:10A3C000A0469368544C0F18A34200D17FE0D26896
:10A3D000DA60936043464B60386025E003004B44ED
:10A3E0003C4206D10A68891A88689B18CA68C2600C
:10A3F000906001221A434A60484AB16012689A424A
:10A4000004D8474B28001968FFF756FF2800FFF7CC
:10A41000F1FA0CBC90469946F8BD5F682740CCD055
:10A42000012303434B6008503E4B98421AD9430A1C
:10A43000042B33D88209140039323834D200B218D0
:10A44000083A936803279A4239D05C68BC43844237
:10A4500033D99B689A42F8D1D368CB608A609960FF
:10A46000D160D3E7C008FF3B8210FF3B9340726886
:10A47000C000134373608619B368CE608B60B1600F
:10A48000D960C3E7002F41D1030090684B44D268E4
:10A490001C43C26090604C60CB50B7E7142B07D9C7
:10A4A000542B1CD8020B14006F326E34D200C6E756
:10A4B0001C005C335B34DA00C1E71A00CCE70123EF
:10A4C000A410A3407068034373601300C5E7D9600C
:10A4D0009960CB608B6043464B60386096E7AA2258
:10A4E0005200934205D8C20B140078327734D20060
:10A4F000A5E70D4A934205D8820C14007D327C34C6
:10A50000D2009CE7FE227E24920098E704434C6030
:10A5100010607BE74C06002054060020580A0020FB
:10A520007C0F0020FF01000054050000F0B58842B8
:10A530000AD98B18984207D2531E002A03D0CA5C4E
:10A54000C254013BFBD2F0BD0F2A09D80500002AF6
:10A55000F9D00023CC5CEC5401339342FAD1F2E7FA
:10A560000D0005430C000300AD0729D11500103D77
:10A570002D092F013F18103726681E6066685E603F
:10A58000A6689E60E6681034DE601033BB42F3D1EB
:10A590000F2401352D01491914404519032C11D9F7
:10A5A0000023CE58EE500433E61A032EF9D80323C5
:10A5B000043CA4080134A4002D1909191A40C6E767
:10A5C0000500C6E72200C2E7F0B5DE46574645461D
:10A5D0004E46E0B5934685B007000D1E00D1A9E0B8
:10A5E0002E00083EFFF704FA736803221C00944310
:10A5F0005A460B32B146162A43D810229246009290
:10A60000D34543D8009A31198846944276DAD44A21
:10A610009168414500D1B6E04246506801210200F0
:10A620008A439446C444624652680A4200D186E096
:10A63000194230D059463800FEF7DAFE804600282D
:10A640001BD0012372689A43B3180200083A934260
:10A6500000D125E1221F242A00D931E12968030015
:10A66000132A00D912E12A001960516859609268D2
:10A670009A6029003800FFF76FFE3800FFF7BAF93B
:10A6800050E007218A4392460092B9D50C233B60E3
:10A690000023984646E03368F31A01935B680293FF
:10A6A0000323029A9A431300009AE11802919142FF
:10A6B000C0DB0198844606008268C3686144D360A9
:10A6C0009A60221F08368846242A00D9EFE02968BC
:10A6D0003300132A09D981606B68C3601B2A00D933
:10A6E00004E110300300A968083519606A68029C0B
:10A6F0005A60AA6835009A60019B994653464A46BB
:10A70000E01A012352681A400F282AD849462243EA
:10A710004A60424652681343424653603800FFF78E
:10A7200069F9A846404605B03CBC90469946A24609
:10A73000AB46F0BD1100FEF75BFE8046F2E7032258
:10A7400090439446009A02902018904269DB434659
:10A750004246B046DB6892688044D36004009A6049
:10A76000CCE7544622434C46494662604246514437
:10A77000184348605268083113434246380053601A
:10A78000FFF7EAFDCAE703225046496810309143BB
:10A7900009199446814200DB96E0DB0700D549E7C2
:10A7A00062463368F31A01935B689343CA180292B6
:10A7B000904200DD78E701988268C3688446D360E0
:10A7C0009A60082262449046221F242A00D9B7E0EA
:10A7D00029684346132A09D981606B68C3601B2A24
:10A7E00000D9B2E00300A9681033083519606A681F
:10A7F0005A60AA689A600198594B020052449A60C4
:10A8000011005246029B9A1A01231A434A6041687A
:10A8100000910B4051460B4343603800FFF7EAF8C4
:10A8200080E7194200D005E762463368F31A0193C6
:10A830005B6803939343029AD1180A190099029214
:10A840008A4200DA30E743464246DB689268019864
:10A85000D3609A608268C3680600D3609A60029BE6
:10A8600084469846221F0836E044242A1FD82968C7
:10A870003300132A00D838E781606B68C3601B2A55
:10A8800034D80300A968103308352EE701606968E1
:10A8900041601B2A35D82A0008330832A968E3E64C
:10A8A0000322B0465B689343E418A04426E72900DE
:10A8B0003000FFF73BFE019B3500029C99461DE7E7
:10A8C0002900FFF733FED4E65346254AF318936078
:10A8D00052460124891A21435960736838001C408C
:10A8E00014437460FFF786F8A8461BE7A968019B2C
:10A8F0001961E9685961242A0ED029691833103585
:10A90000F3E6A9688160E968C160242A0ED02A00B4
:10A91000103310322969A7E62B69019A936113005D
:10A9200069692033D161A9691835DEE62A69010019
:10A9300002612A006869183248611833A96993E6F0
:10A9400029004046FFF7F2FD55E7A968019B196110
:10A95000E9685961242A05D029691833103545E77B
:10A960004C0600202B69019A93611300696920331A
:10A97000D161A969183539E7434AF0B54F46914688
:10A980004B005B0D99444646D6464A46C0B5050085
:10A990000C000E0088460700132A25DC002A56DB2F
:10A9A0003A4B13419A460B0052461340034316D0CC
:10A9B000374A384B00F09AFB00220023F5F746FC9B
:10A9C00000280AD0002C04DD80234A465B03134193
:10A9D00098444646534600279E43380031001CBC2D
:10A9E00090469946A246F0BD332A08DD8023DB005D
:10A9F0009945F4D102000B0000F078FBEFE7264AFE
:10AA00009446012263445242DA4092460242E6D022
:10AA10001F4A204B00F06AFB00220023F5F716FCCA
:10AA20000028DAD0002C0EDD4B46142B22D0342324
:10AA30004A4601249B1A9C406519BD4222D201233B
:10AA40009C462F00E044534646469F43C5E7104AC4
:10AA5000104B00F04BFB00220023F5F7F7FB00281A
:10AA6000BBD0002C0ADB2C4300270026002CB4D0DE
:10AA70000A4EB2E7133B9C46E044E4E780260027F9
:10AA80003606AAE72F00DEE701FCFFFFFFFF0F00FD
:10AA90009C7500883CE4377EEDFBFFFF0000F03F33
:10AAA000474AF0B54F4691464B005B0D99444646E8
:10AAB000D6464A46C0B505000C000E008846070081
:10AAC000132A27DC002A4BDB3E4B13419A460B002E
:10AAD00052461340034318D03B4A3C4B2800210008
:10AAE00000F004FB00220023F5F7B0FB002847D05C
:10AAF000002C04DA80234A465B03134198444646FF
:10AB0000534600279E43380031001CBC90469946AE
:10AB1000A246F0BD332A08DD8023DB009945F4D13D
:10AB200002000B0000F0E2FAEFE7294A9446012206
:10AB300063445242DA4092460242E6D0224A234B14
:10AB40002800210000F0D2FA00220023F5F77EFB56
:10AB5000002815D0002C1EDB534646469F430FE0CD
:10AB6000194A1A4B2800210000F0C0FA00220023E5
:10AB7000F5F76CFB002803D0002C04DB002700262F
:10AB800038003100C1E76400640825430027002D28
:10AB9000F6D0104EF4E74B46142B0BD03422D21AC9
:10ABA000012393405D19BD4208D201239C462F002A
:10ABB000E044D1E7133B9C46E044CDE72F00CBE7D0
:10ABC00001FCFFFFFFFF0F009C7500883CE4377E0F
:10ABD000EDFBFFFF0000F0BFF8B5274A4B005B0D0F
:10ABE0009A180C000700132A10DC002A36DB234BCE
:10ABF00013410B423AD080242403144100206418EE
:10AC00009C430600250030002900F8BD332A0EDDE4
:10AC100080230600DB000D009A42F4D102000B00F5
:10AC20003800210000F062FA06000D00EBE7144D39
:10AC30000600AC46012563446D42DD40AC466346E8
:10AC40000D000342DFD033239A1A323B9340181889
:10AC5000874200D94C1C63469843D2E7C90FCC0702
:10AC60000020531CCDD1074B1C43CAE706000D0042
:10AC70000028C0D1C7E7C04601FCFFFFFFFF0F005F
:10AC8000EDFBFFFF0000F03F044A1368002B00D1EA
:10AC9000034B1818106018007047C046800F002042
:10ACA000880F0020F7B597B201933B00140C86B2D1
:10ACB000050C73436F4366436543F6191C0CA419D6
:10ACC0009C46A74202D980235B02ED186346260CFE
:10ACD000751924049EB2019BA419434320005143DB
:10ACE0005B19591803B0F0BD70B500220B4B04007E
:10ACF0000D00F5F7B5FA00280BD0084B0022200014
:10AD0000290001F069FA01F061FD80231B06C018DB
:10AD100070BD2000290001F059FDF9E70000E04175
:10AD2000F0B5060085B00F0015001C008B4265D8F9
:10AD300001D1824262D821002800F5F729FB3900B1
:10AD400000903000F5F724FB009B21001B1A1A002D
:10AD500028000393F5F7F2FA00900191019BBB42A2
:10AD600046D802D1009BB34242D8009B019C039A73
:10AD700001200021F61AA741F5F7E0FA039B002B0A
:10AD80002FD0019B009ADB0754081C43019B5D08F0
:10AD9000039B9C46BD422ED801D1B4422BD8320031
:10ADA0003B00121BAB41012692185B410027B618ED
:10ADB0005F4101235B429C446346002BEAD180192A
:10ADC0007941039A04000D0030003900F5F7AAFA22
:10ADD000039A06000F00F5F7B1FA241A8D412000FE
:10ADE00029000A9B002B01D01E605F6005B0F0BDFA
:10ADF00000200021C2E7B6197F41DAE700200021D8
:10AE0000EFE7F7B516001F000090019101F0C0FDBB
:10AE100004000D0002000B0030003900FFF742FF74
:10AE2000009A019B121A8B41089920000A604B601E
:10AE3000290003B0F0BD0000F0B5C30F85B0440297
:10AE400045000F1C640A2D0E03931E00002D0AD02E
:10AE5000FF2D39D080200023E400C0047F3D04434F
:10AE6000029500930BE0002C34D02000F5F772FA25
:10AE7000431F9C4076235B421B1A029300957B0084
:10AE80007D021B0E6D0A0193FF0F002B25D0FF2BB7
:10AE90002ED08023ED00DB041D43019B7F3B00216E
:10AEA0000298039AC31A00987A4080000843013838
:10AEB0000E2831D8F5F722FA987976799479769830
:10AEC000989476252525690002950323002CC8D186
:10AED0000223C6E702940123C3E7002D0ED0280009
:10AEE000F5F738FA431F9D4076235B421B1AD6E7DD
:10AEF000019B0321002DD3D10221D1E72B00012199
:10AF0000CEE70099022900D16FE0032945D001293D
:10AF10001AD1002420002BE064016D01AC4230D333
:10AF20001A210120641B0126270040006400002F25
:10AF300001DBA54201D8641B304301390029F3D15C
:10AF4000611E8C411600044318007F3000282EDD5E
:10AF5000620704D00F222240042A00D004342201C8
:10AF600003D580331800224A1440FE283DDCE40853
:10AF70006402C3B2DB05600AF6071843304305B02C
:10AF8000F0BD013B1B210020CDE78023DB031C42E9
:10AF900003D01D4201D12C003E008020C003044399
:10AFA000FF20E5E72C003E00ACE71600B1E70122E8
:10AFB000101A1B28ADDC9E3322009C40C240631E49
:10AFC0009C411443630704D00F232340042B00D07B
:10AFD00004348020C0042040C9D000240120C7E7E9
:10AFE00080240026E403D8E716000024D8E7C046F2
:10AFF000FFFFFFF770B5041E38D0C317C4185C40BC
:10B00000C50F2000F5F7A6F99E231B1A962B0BDC23
:10B01000082801DD083884406002DBB2DB05400A05
:10B02000ED071843284370BD992B0ADD0522210046
:10B03000121AD1400A0001001B318C40611E8C4164
:10B040001443052801DD421F9440220009490A40AB
:10B05000660704D00F263440042C00D0043254017B
:10B0600002D59F230A401B1AD408D5E70300050028
:10B07000D2E7C046FFFFFFFB002370B504009842F3
:10B0800009D0F5F767F99E231B1A962B09DC0828CF
:10B0900001DD083884406002DBB2DB05400A18435A
:10B0A00070BD992B0ADD020021001B3291400A007D
:10B0B000511E8A410521091ACC401443052801DD9F
:10B0C000421F9440220008490A40650704D00F251A
:10B0D0002C40042C00D00432540102D59F230A4096
:10B0E0001B1AD408D7E7C046FFFFFFFBF7B50D00DA
:10B0F00009036C00ED0F0095490A450F5E002943D6
:10B100001D03DB0F9C466B0A550F2B43009D640DFE
:10B11000760DC700D200A01B654500D035E10028A0
:10B1200061DD002E25D11D00154300D196E2461E9B
:10B13000002E19D1BA18BA42A441C918644209199B
:10B14000170001240B0200D4BEE0BC4B01349C422A
:10B1500000D180E2BA487B080140012007401F432C
:10B16000C80707434908AFE0B44DA84209D1B34C22
:10B17000AAE0B24DAC4200D1A6E0802506002D0425
:10B180002B43382E2ADC1F2E17DC20201D00801BAD
:10B190008540AC4615000190F54060460543019896
:10B1A000F3408240501E82411543ED195B18BD42A9
:10B1B0008941494259182F00C4E730001D0020384A
:10B1C000C5400020202E03D04030861BB34018001D
:10B1D0000243501E824115430023E6E71A4315003F
:10B1E0006A1E9541F8E7002850D0002C2ED10C00A3
:10B1F0003C4300D125E2441C07D1BF189742A4412B
:10B20000C9186442091934009CE78C4CA64200D14D
:10B210001DE2C443382C34DC1F2C20DC2025281BE5
:10B2200001900800019DE140A84084463800654631
:10B23000E0402843019DAF407D1EAF413843871851
:10B2400097429241C91852428918DCE77B4CA642CA
:10B2500000D1FCE14442802000040143DAE72000F1
:10B260000D002038C54028000025202C03D0403593
:10B270002C1BA1400D002F437D1EAF413843002100
:10B28000DDE70F433800471EB841F8E7661C750537
:10B290006D0D012D00DD68E008003843002C49D118
:10B2A000002800D1D0E1180010430DD0BA18BA42DE
:10B2B000B641C9188023764289191B041700194228
:10B2C00002D05F4B013419407B0709D00F233B406C
:10B2D000042B05D03B1DBB42BF417F42C9191F0053
:10B2E0000B0206D5554B01349C4200D1CCE1544BA6
:10B2F0001940524B4807FF083843C9089C4206D101
:10B3000003000B4300D1C2E180231B031943002734
:10B3100009033B0D1B05090B19434A4B64051940F2
:10B3200064080C43009B6400D90764080C432100A7
:10B3300003B0F0BD002800D189E118003F4C104354
:10B34000C2D080204C07FF08C908000327430142F0
:10B3500006D0DC08044203D12100D7085B071F4355
:10B36000780FC9000143FF0001E7344CA64200D129
:10B3700070E1BA18C918BA429B415B42CB18DF078B
:10B3800052081743590834009EE700285CDD002E60
:10B3900035D11D00154300D160E1461E002E0ED1AF
:10B3A000BA1A9742BF41C91A7F42C91B012417002C
:10B3B0000B0200D488E749024D0A3E00F7E01F4D1A
:10B3C000A84200D1D3E6382E33DC1F2E20DC20200B
:10B3D0001D00801B8540AC4615000190F54060467D
:10B3E00005430198F3408240501E824115437D1B66
:10B3F000CB1AAF4289414942591A2F00D8E70F4D65
:10B40000AC4200D160E780252D042B430600DAE72B
:10B4100030001D002038C5400020202E03D04030D1
:10B42000861BB34018000243501E8241154300237F
:10B43000DDE71A4315006A1E9541F8E7FF07000093
:10B44000FFFF7FFFFFFF0F8000284CD0002C2AD188
:10B450000C003C4300D103E1441C09D1D71BBA4284
:10B460009241591A63465242891A340000939FE769
:10B47000884CA64200D1F7E0C443382C2EDC1F2CA8
:10B480001ADC2025281B00900800009DE140A84000
:10B4900005003800E0402843009DAF407D1EAF41CD
:10B4A0003843171ADBE77B4CA64200D1DCE044426C
:10B4B000802000040143E0E720000D002038C54053
:10B4C00028000025202C03D040352C1BA1400D0066
:10B4D0002F437D1EAF4138430021E2E70F43380080
:10B4E000471EB841F8E7601C4005400D01284CDCC0
:10B4F0000D0018003D431043002C24D1002D07D12E
:10B50000002800D1B4E01900170063460093DBE681
:10B51000002800D1D8E6BD1AAF42B641C81A76421B
:10B52000801B80263604304206D0D71BBA42924197
:10B53000591A5242891AE8E72F00074300D19BE0CD
:10B5400001002F00C0E6002D07D1002800D196E0B1
:10B55000190063461700009309E64E4C002800D1FD
:10B56000B2E680204C07FF08C908000327430142C8
:10B5700000D1F5E6DC08044200D0F1E65B07D7080D
:10B580001F43634621000093EAE6BE1AB74280419A
:10B59000CD1A40422D1A8020000405422DD0D61B22
:10B5A000B242AD41591A63466D424D1B0093002DC6
:10B5B00029D02800F4F7CEFE0300083B1F2B27DC20
:10B5C000202231009E40D21A9D40D14037000D43C9
:10B5D0009C4232DC1C1B661C1F2E1EDC20233A0002
:10B5E00029009B1B9940F2409F400A43791E8F41DE
:10B5F0002900F1401743002466E637002F43D6D1D7
:10B6000039003C0039E03000F4F7A4FE2030D3E7E5
:10B610003500283885400027DAE72A001F3CE24041
:10B620000023202E03D040339E1B2B00B3401F432A
:10B630007B1E9F4100211743DDE71749E41A29408B
:10B6400042E6190017009EE6190017003CE61900B3
:10B6500017008CE50F4C00210F0035E6040033E69F
:10B6600019001700340050E719001700094C4CE787
:10B6700021002700009427E63900009724E6802166
:10B680000700C903034CF8E700210F0031E6190059
:10B690003DE6C046FF070000FFFF7FFFF0B587B023
:10B6A000060002930400CB0F0D03480000922D0BFF
:10B6B000400D0493039344D0674B984265D0EB0050
:10B6C00080252D041D43654B770F2F43F400C318CD
:10B6D00000260193029B009A1D035800DB0F2D0BDF
:10B6E000400D059360D05C4B984200D181E08023EF
:10B6F000ED001B0459491D43530F2B43D200411841
:10B700008C4600210598049D4540029565460198A8
:10B71000401B0190B000084301380E2800D9A3E077
:10B72000F4F7F6FD20028200CF01820017028200AA
:10B73000CF01200220021702CF01760076007600AA
:10B74000BE012F00374327D0002D13D02800F4F777
:10B7500001FE01000B391C2911DC02001D233700FA
:10B760003400083A5B1A9540DF4094402F433C4B2D
:10B770001B1AADE73000F4F7EDFD2030E9E70300D8
:10B78000283B9E4000243700F1E72E43371E07D0A8
:10B790002F00019003269DE73C000197012699E7C1
:10B7A00034000190022695E7009B2B4328D0002D02
:10B7B00013D02800F4F7CEFD03000B3B1C2B11DC4B
:10B7C0001D220100D21A009B0839D340009A8D40F7
:10B7D0008A402B432249091A92E71000F4F7BAFD78
:10B7E0002030E9E70300009A283B9A40130000222A
:10B7F000F0E7009B2B4307D02B008446032181E711
:10B800001A009C4601217DE71A008446022179E74F
:10B810003100049B0293022900D1A6E1032900D143
:10B820009DE1012900D014E100252C002B0000210E
:10B830002D030A0D12052D0B15430A4A5B05154011
:10B840005B082B43029A5B00D2075B08134320007E
:10B85000190007B0F0BDC046FF07000001FCFFFF64
:10B860000DFCFFFFFFFF0F809F4204D800D012E1C4
:10B87000A24200D90FE1F80761080843E607040077
:10B880007F08150E1B021D43130200933800ABB254
:10B89000290C0393F4F750FCABB243430A04210C88
:10B8A000114307008B4207D94919013F8D4203D844
:10B8B0008B4201D9871E4919C81A290CF4F73CFCA0
:10B8C000AAB242430904A4B2214303008A4207D921
:10B8D0004919013B8D4203D88A4201D9831E491977
:10B8E000891A009C009A3F043B43120C24040392E3
:10B8F000240C9AB204945443049F0594039C180C9E
:10B90000474362436043059CD219240CA446624419
:10B91000974202D9802464020019059C170C38183C
:10B92000270412043F0CD219814204D31F00814224
:10B930001CD196421AD2009C5F1E3619A642A44121
:10B940006442641909198D4203D30FD1009CB4429B
:10B950000CD8884202D809D1B24207D99F1E009B59
:10B96000F6189E429B415B425B19C918B31A091A2B
:10B970009E42804140420593081A854200D1A5E0CD
:10B98000290CF4F7D9FBABB243430A040599040030
:10B99000090C11438B4207D94919013C8D4203D848
:10B9A0008B4201D9841E4919C81A290CF4F7C4FB2B
:10B9B0006B46AAB242439B8A0904194303008A4298
:10B9C00007D94919013B8D4203D88A4201D9831E08
:10B9D0004919240423430498891A9AB25043049CB9
:10B9E000059003981E0C7443424346430598121970
:10B9F000000C84466244944202D9802040023618EA
:10BA00000598140C00041204000CA6191218B14277
:10BA100004D31C00B1421AD1002A1AD069185C1E46
:10BA2000A9420FD3B14203D311D1009890420BD257
:10BA30009C1E009B00985B00834280414042451958
:10BA400049190093B14202D1009B9A4201D00123CF
:10BA50001C43019B4A4A9B18002B3ADD620709D020
:10BA60000F222240042A05D0221DA242A441644292
:10BA70003F191400FA0106D58022D2009446414BAA
:10BA80001F40019B6344404A93426EDCE4087907FF
:10BA90000C43FD08CBE60199002601390191F0E63F
:10BAA000802109030F4205D00B4203D114001F006F
:10BAB000059903918025039B2D033D430293334B4E
:10BAC000B5E61F00059B14000293A4E6012464421E
:10BAD000BFE70122D21A382A4ADC1F2A24DC2C496B
:10BAE000019B8C466344180021003B00D1408340F9
:10BAF00084403D000B43611E8C41D5401C436307CD
:10BB000009D00F232340042B05D0231DA342A441B9
:10BB100064422D191C0080231B042B402CD1690783
:10BB2000E4080C43ED0882E61F214942CB1A390094
:10BB3000D9400B000021202A05D01649019A8C46D5
:10BB40003900624491400C43611E8C4100251C4326
:10BB5000D5E70023802703931C003F03AAE7029B3D
:10BB60000393A7E700252C00A9E700242500A6E7FA
:10BB70000024250023005AE6002501232C0056E668
:10BB8000FF030000FFFFFFFEFE070000FF070000AD
:10BB90001E0400003E040000F0B50C0385B04D000B
:10BBA0000600C90F17481F0301915900DB0F240B32
:10BBB0006D0D03923F0B490D0293854206D1230080
:10BBC000012033431AD1A94218D101E0814203D1A7
:10BBD0003A430120002A11D101208D420ED1BC42EE
:10BBE0000CD1039A964209D1019B029A934207D045
:10BBF000002D03D134432000441EA04105B0F0BD08
:10BC00000020FBE7FF070000F0B51F0385B05E00D2
:10BC1000DB0F01932B4B0C034D000290240B6D0D99
:10BC2000C90F03923F0B760D9D4204D123000343BD
:10BC300041D0022029E09E4207D13A43F9D1002D9C
:10BC40000FD120434242504109E0002D35D120431D
:10BC5000434243411800002E01D13A4328D0002826
:10BC600008D1019B99420AD00120002900D0023856
:10BC700005B0F0BD019B002BFAD1012005E0B542D3
:10BC8000F2DC04DA01200029F2D14042F0E7BC42A4
:10BC9000EAD809D1029B039A9342E5D8029B039A02
:10BCA00000209342EED3E3E7BC42EBD30020DFE772
:10BCB0000028FBD1D8E7AE42BFD000208642CCD0CE
:10BCC000CFE7C046FF070000F0B51F035E00DB0FA3
:10BCD0009C462D4B85B00C034D0001920290240B25
:10BCE0006D0DC90F03923F0B760D9D4206D12200C8
:10BCF0000223024342D0180005B0F0BD9E4209D194
:10BD0000019A02233A43F6D1002D0FD1204343423A
:10BD1000434109E0002D33D1204343424341002EEB
:10BD200002D1019A3A4326D0002B06D1614509D0B1
:10BD300001230029DFD0023BDDE76246002ADAD189
:10BD4000012305E0B542F3DC04DA01230029D2D156
:10BD50005B42D0E7BC42EBD809D1029B039A9342E5
:10BD6000E6D8029A039800238242EED3C3E7BC428E
:10BD7000EBD30023BFE7002BFBD1D9E7AE42BFD006
:10BD800000239E42CDD0D1E7FF070000F0B58BB075
:10BD9000060003930400CB0F0D03480000922D0B07
:10BDA000400D0593049346D05D4B984267D0EB005D
:10BDB00080252D041D435B4B770F2F43F400C318E0
:10BDC00002930023039A019316035000D20F009BA5
:10BDD000360B400D069261D0514A904200D181E06D
:10BDE0008025F6002D044F4A2E435D0F3543DB00BE
:10BDF000801800220599069E71400391029941180E
:10BE000007910131009101998800104301380E28F3
:10BE100000D98BE0F4F77CFA7600760079017300A4
:10BE20007300BC0179017300BC01730079017401D6
:10BE3000740174016A012F00374327D0002D13D0FD
:10BE40002800F4F787FA01000B391C2911DC0200E5
:10BE50001D2337003400083A5B1A9540DF409440B8
:10BE60002F43314B1B1AABE73000F4F773FA203045
:10BE7000E9E70300283B9E4000243700F1E72E430A
:10BE8000371E07D02F00029003239BE73C00029748
:10BE9000012397E734000290022393E7009D354386
:10BEA00026D0002E13D03000F4F754FA01000B39DD
:10BEB0001C2911DC1D230200009D5B1A083ADD409D
:10BEC000009B964093403543174A101A91E718009B
:10BED000F4F740FA2030E9E70300009D283B9D403D
:10BEE0000023F1E7009D354306D03500032281E7AA
:10BEF0002B00280001227DE72B0002227AE73D007B
:10BF00002300019A022A00D151E1032A00D14BE11A
:10BF1000012A00D0B4E000252C002A00D2E0C0465F
:10BF2000FF07000001FCFFFF0DFCFFFF220C190CB6
:10BF3000A4B29BB2019120001900584351430290D2
:10BF400008000199019E51436643049102993618F5
:10BF5000090C8919884206D9049E30008026760291
:10BF6000B44660440490684600890E0C0904091820
:10BF70000991290CADB2029128002100B446029E1D
:10BF8000504374436943724324180E0C3419A04281
:10BF900002D9802040021218200C8218240489B291
:10BFA000B8B20592621806920600069962468C465F
:10BFB000390C019F5E4347434B4362449446019CC6
:10BFC000FF18320CD2194C43934202D980235B02F2
:10BFD000E418130C1B19089303001204B6B2961947
:10BFE000029A6B4350434D43514340191C0C241893
:10BFF0000191A54203D9802252028A180192049A23
:10C000009BB262441000069A9042AD412204D218BD
:10C01000059B6D42D3185F191900089B059A9C4631
:10C0200091429241BC44AF42BF418019B042B641F7
:10C03000634652427F42240C3A4376421219089CCE
:10C040009B19B342B641A445A441764264423443AD
:10C05000019912195118099A4D024102DE0D11433E
:10C0600035434E1EB141C00D08435B020343EA0154
:10C070004ED501245A0823401343EC0723436D088F
:10C08000009A4E495218002A45DD590709D00F2160
:10C090001940042905D0191D99429B415B42ED18B6
:10C0A0000B00E90106D58021C9008C46444A1540A1
:10C0B000009A624443498A4200DD78E0DB086C075D
:10C0C0001C43ED0800212D030E0D36053E4B2D0BB4
:10C0D000354352051D4052082A43039B5200DB079B
:10C0E00052081A43200011000BB0F0BD8022120349
:10C0F000174252D0154250D12F00069A04924BE0BD
:10C10000059A3D0023000392FBE606990391F9E6A8
:10C11000079A0092B4E70120801A382800DDFAE679
:10C120001F2820DC2949009A8C462C006244190003
:10C1300093409440C1405A1E9341C5400C431C4358
:10C14000630709D00F232340042B05D0231DA342EE
:10C15000A44164422D191C00802212042A4029D1D6
:10C16000E4086B07ACE71F2149428A1A2900D14035
:10C170000022202805D01648009A84466244954043
:10C180002A001A431400621E944100250C43D7E78D
:10C19000802700233F0304931C008025049B2D036C
:10C1A0003D4303930B4A8DE72F00039AA6E7002532
:10C1B0002C00F7E7002501222C0083E7FF03000095
:10C1C000FFFFFFFEFE070000FFFF0F801E040000C0
:10C1D0003E040000FF070000F7B50D0009036C00E6
:10C1E000ED0F0095490A450F29431D035E00C70066
:10C1F000D80F6B0A550F2B43C04D640D760DD2003E
:10C20000AE4203D11D008446154302D101254540AD
:10C21000AC46009DA01BAC4500D035E1002861DD97
:10C22000002E25D11D00154300D195E2461E002E9B
:10C2300019D1BA18BA42A441C918644209191700A1
:10C2400001240B0200D4BEE0AC4B01349C4200D16F
:10C250007FE2AB487B080140012007401F43C8072D
:10C2600007434908AFE0A54DA84209D1A34CAAE075
:10C27000A24DAC4200D1A6E0802506002D042B4340
:10C28000382E2ADC1F2E17DC20201D00801B854045
:10C29000AC4615000190F540604605430198F34017
:10C2A0008240501E82411543ED195B18BD42894101
:10C2B000494259182F00C4E730001D002038C540FE
:10C2C0000020202E03D04030861BB34018000243CC
:10C2D000501E824115430023E6E71A4315006A1EEB
:10C2E0009541F8E7002850D0002C2ED10C003C439B
:10C2F00000D124E2441C07D1BF189742A441C918B9
:10C300006442091934009CE77C4CA64200D11CE22F
:10C31000C443382C34DC1F2C20DC2025281B019042
:10C320000800019DE140A840844638006546E04091
:10C330002843019DAF407D1EAF4138438718974287
:10C340009241C91852428918DCE76C4CA64200D1D0
:10C35000FBE14442802000040143DAE720000D00A5
:10C360002038C54028000025202C03D040352C1B48
:10C37000A1400D002F437D1EAF4138430021DDE772
:10C380000F433800471EB841F8E7661C75056D0D70
:10C39000012D00DD68E008003843002C49D1002859
:10C3A00000D1CFE1180010430DD0BA18BA42B641FF
:10C3B000C9188023764289191B041700194202D03C
:10C3C0004F4B013419407B0709D00F233B40042B0E
:10C3D00005D03B1DBB42BF417F42C9191F000B0264
:10C3E00006D5464B01349C4200D1CBE1444B194069
:10C3F000424B4807FF083843C9089C4206D1030056
:10C400000B4300D1C1E180231B031943002709031B
:10C410003B0D1B05090B19433A4B64051940640891
:10C420000C43009B6400D90764080C43210003B04F
:10C43000F0BD002800D188E11800104300D115E7B5
:10C4400080204C07FF08C90800032743014206D09B
:10C45000DC08044203D12100D7085B071F43780F93
:10C46000C9000143FF0001E7244CA64200D16FE15F
:10C47000BA18C918BA429B415B42CB18DF07520871
:10C480001743590834009EE700285CDD002E3BD19D
:10C490001D00154300D15FE1461E002E0ED1BA1AD1
:10C4A0009742BF41C91A7F42C91B012417000B02E2
:10C4B00000D488E749024D0A3E00F6E00F4DA8423D
:10C4C00000D1D3E6382E39DC1F2E26DC20201D00BB
:10C4D000801B8540AC4615000190F5406046054341
:10C4E0000198F3408240501E824115437D1BCB1AB8
:10C4F000AF4289414942591A2F00D8E7FF0700008F
:10C50000FFFF7FFFFFFF0F80A14DAC4200D15AE734
:10C5100080252D042B430600D4E730001D00203871
:10C52000C5400020202E03D04030861BB3401800A9
:10C530000243501E824115430023D7E71A431500DA
:10C540006A1E9541F8E700284CD0002C2AD10C0037
:10C550003C4300D102E1441C09D1D71BBA429241AD
:10C56000591A63465242891A340000939FE7884C57
:10C57000A64200D1F6E0C443382C2EDC1F2C1ADC76
:10C580002025281B00900800009DE140A8400500E0
:10C590003800E0402843009DAF407D1EAF41384346
:10C5A000171ADBE77A4CA64200D1DBE04442802038
:10C5B00000040143E0E720000D002038C5402800BA
:10C5C0000025202C03D040352C1BA1400D002F430B
:10C5D0007D1EAF4138430021E2E70F433800471E7C
:10C5E000B841F8E7601C4005400D01284BDC0D0008
:10C5F00018003D431043002C24D1002D07D1002802
:10C6000000D1B3E01900170063460093DBE6002871
:10C6100000D1D8E6BD1AAF42B641C81A7642801B97
:10C6200080263604304206D0D71BBA429241591AAE
:10C630005242891AE8E72F00074300D19AE001002F
:10C640002F00C0E6002D07D1002800D195E0190089
:10C6500063461700009309E6002800D106E6802013
:10C660004C07FF08C90800032743014200D1F6E642
:10C67000DC08044200D0F2E65B07D7081F4363469C
:10C6800021000093EBE6BE1AB7428041CD1A40422A
:10C690002D1A8020000405422DD0D61BB242AD4198
:10C6A000591A63466D424D1B0093002D29D0280076
:10C6B000F3F750FE0300083B1F2B27DC202231003C
:10C6C0009E40D21A9D40D14037000D439C4232DC3F
:10C6D0001C1B661C1F2E1EDC20233A0029009B1BFE
:10C6E0009940F2409F400A43791E8F412900F14052
:10C6F0001743002467E637002F43D6D139003C00AA
:10C7000039E03000F3F726FE2030D3E73500283833
:10C7100085400027DAE72A001F3CE2400023202E54
:10C7200003D040339E1B2B00B3401F437B1E9F4111
:10C7300000211743DDE71749E41A294043E61900B1
:10C7400017009FE6190017003DE6190017008DE558
:10C750000F4C00210F0036E6040034E619001700E4
:10C76000340051E719001700094C4DE7210027005C
:10C77000009428E63900009725E680210700C903C8
:10C78000034CF8E700210F0032E619003EE6C046F0
:10C79000FF070000FFFF7FFF70B50B4E0D031C036A
:10C7A00049005B002D0B490D240B5B0DB14203D1F9
:10C7B00005430120002D06D10020B34203D12243BE
:10C7C0001000421E904170BDFF070000134B30B5B2
:10C7D0004A000C030500240B520DC90F00209A4299
:10C7E00004DD0F4B9A4202DD0E4BC81830BD80238A
:10C7F0005B0323430C4CA41A1F2C09DC0B481218B2
:10C8000028009340E04018430029EFD04042EDE774
:10C810000748821AD3401800F6E7C046FE0300001E
:10C820001D040000FFFFFF7F33040000EDFBFFFF4E
:10C8300013040000F8B5002827D0C317C5185D40C1
:10C84000C40F2800F3F786FD1249091A0A2817DCDD
:10C850000B232A001B1A1530DA40854000271203EB
:10C86000130B3A0D0C4812051A434B0502405B08A6
:10C8700013435B00E4075B08234328001900F8BD5D
:10C880002A000B3882400025E8E70200050001007D
:10C890000400E3E71E040000FFFF0F8070B5041ED4
:10C8A0001FD0F3F757FD104D2D1A0A2814DC0B2367
:10C8B00022001B1A1530DA40844000211203130BAA
:10C8C0000A0D20001205094C1A436B0522405B0833
:10C8D00013435B00590870BD22000B3882400024CE
:10C8E000EBE702000500E8E71E040000FFFF0F80F1
:10C8F000F8B54600360E731C4202DBB2540AC50F6F
:10C90000012B16DDE0239B00F318120B64070027B0
:10C910001203110B3A0D1B4812050A435B05024036
:10C920005B0813435B00ED075B082B4320001900F5
:10C93000F8BD002E17D1002C1ED02000F3F70AFD01
:10C940000A280ADC0B222300121AD3401A00030023
:10C9500015339C400C4B1B1AD9E7030022000B3BFC
:10C960009A403400F6E7002C09D08023120B1B03F9
:10C9700064071A43054BCAE722002300C7E72200D9
:10C98000F8E7C046FFFF0F8089030000FF070000A3
:10C99000F0B585B000900191002103910199002923
:10C9A00009DA009C019D00216042A941009001919B
:10C9B000012149420391002B07DA03991000C94372
:10C9C00003911900002342428B41009E019F1C00ED
:10C9D000019B15009C4200D96FE003D1009B9A4255
:10C9E00000D96AE021002800F3F7D2FC02900098F9
:10C9F0000199F3F7CDFC029B21001B1A1A002800B5
:10CA00000293F3F79BFC019B04000D0099424ED862
:10CA100002D1009B98424AD8009E019F029A0120B1
:10CA20000021361BAF41F3F789FC029B002B34D069
:10CA3000EB079C4662466308134300936B0801931F
:10CA4000029B01249C460025019BBB4232D802D1A7
:10CA5000009BB3422ED832003B00009E019F921BE8
:10CA6000BB4192185B4112196B4116001F00012354
:10CA70005B429C446346002BE6D180197941029ABF
:10CA800004000D0030003900F3F74CFC029AF3F774
:10CA900055FC241A8D4120002900039B002B04D053
:10CAA00003000C0000215842A14105B0F0BD002058
:10CAB0000021BAE7B6197F41D9E700200021ECE751
:10CAC000F8B5C046F8BC08BC9E467047F8B5C046ED
:08CAD000F8BC08BC9E4670474B
:10CAD8004932435F576169744F6E54584953466CE5
:10CAE8006167556E74696C54696D656F7574202D36
:10CAF8003E4932435F497341636B6E6F776C65647F
:10CB080067654661696C6564206572726F720D0AAB
:10CB1800000000004932435F576169744F6E5458F2
:10CB28004953466C6167556E74696C54696D656FDD
:10CB380075742074696D656F75740D0A00000000C6
:10CB48002E2500084A250008662500082C2600081E
:10CB58009E2500082C2600082C2600082C260008F4
:10CB6800BA25000886240008AC240008C42400085C
:10CB780028250008F824000828250008282500088A
:10CB88002825000810250008A12E0008012F0008FC
:10CB98008D380008BD2F0008C13700086D30000827
:10CBA800353900087D390008D5390008313E0008BC
:10CBB800592E00082D310008FD430008F9330008FC
:10CBC8002134000849340008713700089D410008E5
:10CBD8006533000855300008153100081530000885
:10CBE800D5300008F1490008394A0008814B00088F
:10CBF800280A0000170000001C0C00000F000000AD
:10CC08003C0F000007000000501400001600000050
:10CC18009C1800000E000000781E000006000000AE
:10CC2800A028000015000000D43000000D0000000E
:10CC3800F03C000005000000405100001400000016
:10CC4800A86100000C000000447A00000400000005
:10CC5800E4A200001300000050C300000B00000015
:10CC680024F40000030000008545010012000000C4
:10CC7800A08601000A00000048E801000200000048
:10CC88002C8B020011000000400D03000900000079
:10CC980090D0030001000000E093040000000000B1
:10CCA800000C23000D1E000ED2001A01001FAA005E
:10CCB80024070027120028C1002994002AC1003047
:10CCC800D800358F003B020040000041300131435D
:10CCD800012340007278446F6E650A0D0000000061
:10CCE8007478446F6E650A0D00000000727854690C
:10CCF8006D654F75740A0D002E2F5372632F76637E
:10CD08006F6D2E63000000002E2F5372632F737413
:10CD18006D33326C3078785F68772E6300000000DE
:10CD28001F1C1F1E1F1E1F1F1E1F1E1F1F1D1F1E15
:10CD38001F1E1F1F1E1F1E1F2E2F5372632F73745B
:10CD48006D33326C3078785F68616C5F6D73702E0C
:10CD580063000000494E4954204552524F522C203E
:10CD680025733A25640000002E2F5372632F6877CD
:10CD78005F6932632E6300002E2F5372632F68772A
:10CD88005F7370692E63000000000000000000005F
:10CD98000102030406070809000000000102030459
:10CDA800030406080C101820300000000D0A484142
:10CDB80052444641554C54210D0A0000424D453617
:10CDC800383020696E697469616C697A696E672E9A
:10CDD8002E2E0D0A00000000424D453638302063E3
:10CDE8006F6E6669677572696E672E2E2E0D0A0062
:10CDF800543A20252E326620646567432C20503A29
:10CE080020252E3266206850612C204820252E329D
:10CE180066202525724820002C20473A20256420CA
:10CE28006F686D7300000000B8000020886F00086C
:10CE3800D46E0008D46E00087E6F0008D46E000817
:10CE4800D46E0008D46E0008D46E0008D46E0008B2
:10CE5800D46E0008626F00085A6F0008D46E00088C
:10CE6800506F0008026F0008D46E0008F86E0008C2
:10CE78009C6E00089C6E00089C6E00089C6E000862
:10CE88009C6E00089C6E00089C6E00089C6E000852
:10CE98009C6E0008D46E0008D46E0008D46E00089A
:10CEA800D46E0008D46E0008D46E0008D46E000852
:10CEB800D46E0008D46E0008D46E00087875000897
:10CEC800D4740008D46E0008D4740008D46E000826
:10CED800D46E0008D46E0008D46E0008CA74000826
:10CEE800D46E0008D46E0008A6740008D46E00083A
:10CEF800D46E0008D46E0008D46E0008D46E000802
:10CF0800E0750008D46E0008D46E0008AC750008FF
:10CF1800D46E0008D46E0008D46E0008D46E0008E1
:10CF2800D46E0008D46E0008D46E0008D46E0008D1
:10CF3800D46E0008D46E0008D27100085C71000835
:10CF4800D4740008D4740008D47400089C740008D1
:10CF58005C710008D46E0008D46E00088C74000858
:10CF6800D46E00082C740008067400086674000863
:10CF78005C740008D46E0008FA700008D46E0008CB
:10CF88007E700008D46E0008D46E0008986F000800
:10CF9800494E4600696E66004E414E006E616E0055
:10CFA80030313233343536373839414243444546D7
:10CFB8000000000030313233343536373839616299
:10CFC8006364656600000000286E756C6C290000BB
:10CFD8003000000020202020202020202020202099
:10CFE8002020202030303030303030303030303079
:10CFF80030303030496E66696E697479000000001F
:10D008004E614E0043000000504F53495800000045
:10D018002E000000000000000080E03779C3414383
:10D02800176E05B5B5B89346F5F93FE9034F384D86
:10D03800321D30F94877825A3CBF737FDD4F157532
:10D04800000000000000F03F000000000000244045
:10D0580000000000000059400000000000408F4020
:10D06800000000000088C34000000000006AF8408B
:10D078000000000080842E4100000000D0126341AF
:10D088000000000084D797410000000065CDCD4125
:10D09800000000205FA00242000000E87648374206
:10D0A800000000A2941A6D42000040E59C30A242A4
:10D0B8000000901EC4BCD64200003426F56B0C4319
:10D0C8000080E03779C3414300A0D88557347643C0
:10D0D80000C84E676DC1AB43003D9160E458E14321
:10D0E800408CB5781DAF154450EFE2D6E41A4B4496
:10D0F80092D54D06CFF08044F64AE1C7022DB544DB
:10D10800B49DD9794378EA4405000000190000006D
:10D118007D0000000020202020202020202028281A
:10D1280028282820202020202020202020202020DF
:10D13800202020202088101010101010101010101F
:10D14800101010101004040404040404040404104F
:10D1580010101010101041414141414101010101DD
:10D1680001010101010101010101010101010101A7
:10D1780010101010101042424242424202020202B3
:10D188000202020202020202020202020202020277
:10D198001010101020000000000000000000000027
:10D1A8000000000000000000000000000000000077
:10D1B8000000000000000000000000000000000067
:10D1C8000000000000000000000000000000000057
:10D1D8000000000000000000000000000000000047
:10D1E8000000000000000000000000000000000037
:10D1F8000000000000000000000000000000000027
:10D208000000000000000000000000000000000016
:08D2180000000000000000000E
:08D2200000DBFF7F01000000AC
:08D22800656D0008D103000848
:04D23000A903000846
:10D234003D2E0008392E0008512F00085D2E0008ED
:10D244003F2E0008412E000875450008C948000813
:10D254004142000889430008912F000800000000A3
:10D2640080841E00FFFFFF7FFFFFFF7FFFFFFF7F24
:10D27400FFFFFF7FFFFFFF7FEA51B87EFFFFFF7FC5
:10D2840021DBF97EFFFFFF7FFFFFFF7FC776BE7FB5
:10D29400F4285C7FFFFFFF7FEA51B87EFFFFFF7F2A
:10D2A400FFFFFF7F000024F40000127A0000093D14
:10D2B4000080841EFF583E0F548C93070090D003C7
:10D2C4001038EC019062F40000127A0000093D006D
:10D2D40080841E0040420F0020A1070090D003006C
:10D2E40048E80100B800002000000000A40300206A
:10D2F4000C04002074040020000000000000000062
:10D304000000000000000000000000000000000019
:10D314000000000000000000000000000000000009
:10D3240000000000000000000000000000000000F9
:10D3340000000000000000000000000000000000E9
:10D3440000000000000000000000000000000000D9
:10D3540000000000000000000000000000000000C9
:10D3640000000000000000000000000000000000B9
:10D3740000000000000000000000000000000000A9
:10D384000000000000000000000000000000000099
:10D3940001000000000000000E33CDAB34126DE636
:10D3A400ECDE05000B00000000000000000000009F
:10D3B4000000000000000000000000000000000069
:10D3C4000000000000000000000000000000000059
:10D3D4000000000000000000000000000000000049
:10D3E4000000000000000000000000000000000039
:10D7140043000000000000000000000000000000C2
:10D7240000000000000000000000000000000000F5
:10D7340043000000000000000000000000000000A2
:10D7440000000000000000000000000000000000D5
:10D754004300000000000000000000000000000082
:10D7640000000000000000000000000000000000B5
:10D774004300000000000000000000000000000062
:10D784000000000000000000000000000000000095
:10D794004300000000000000000000000000000042
:10D7A4000000000000000000000000000000000075
:10D7B4004300000000000000000000000000000022
:10D7C4000000000000000000000000000000000055
:10D7D4004300000000000000000000000000000002
:10D7E4000000000000000000000000000000000035
:10D7F40045A2000845990008000000001CD100085B
:10D8040018D00008DCCD0008DCCD0008DCCD000811
:10D81400DCCD0008DCCD0008DCCD0008DCCD000840
:10D82400DCCD0008DCCD0008FFFFFFFFFFFFFFFF9A
:10D83400FFFFFFFFFFFF0000010041534349490080
:10D8440000000000000000000000000000000000D4
:10D85400000000000000000000004153434949005B
:10D8640000000000000000000000000000000000B4
:10D8740000000000000000000000000000000000A4
:10D88400000000004C0600204C0600205406002036
:10D89400540600205C0600205C060020640600207C
:10D8A400640600206C0600206C060020740600202C
:10D8B400740600207C0600207C06002084060020DC
:10D8C400840600208C0600208C060020940600208C
:10D8D400940600209C0600209C060020A40600203C
:10D8E400A4060020AC060020AC060020B4060020EC
:10D8F400B4060020BC060020BC060020C40600209C
:10D90400C4060020CC060020CC060020D40600204B
:10D91400D4060020DC060020DC060020E4060020FB
:10D92400E4060020EC060020EC060020F4060020AB
:10D93400F4060020FC060020FC060020040700205A
:10D94400040700200C0700200C0700201407002007
:10D95400140700201C0700201C07002024070020B7
:10D96400240700202C0700202C0700203407002067
:10D97400340700203C0700203C0700204407002017
:10D98400440700204C0700204C07002054070020C7
:10D99400540700205C0700205C0700206407002077
:10D9A400640700206C0700206C0700207407002027
:10D9B400740700207C0700207C07002084070020D7
:10D9C400840700208C0700208C0700209407002087
:10D9D400940700209C0700209C070020A407002037
:10D9E400A4070020AC070020AC070020B4070020E7
:10D9F400B4070020BC070020BC070020C407002097
:10DA0400C4070020CC070020CC070020D407002046
:10DA1400D4070020DC070020DC070020E4070020F6
:10DA2400E4070020EC070020EC070020F4070020A6
:10DA3400F4070020FC070020FC0700200408002055
:10DA4400040800200C0800200C0800201408002002
:10DA5400140800201C0800201C08002024080020B2
:10DA6400240800202C0800202C0800203408002062
:10DA7400340800203C0800203C0800204408002012
:10DA8400440800204C0800204C08002054080020C2
:10DA9400540800205C0800205C0800206408002072
:10DAA400640800206C0800206C0800207408002022
:10DAB400740800207C0800207C08002084080020D2
:10DAC400840800208C0800208C0800209408002082
:10DAD400940800209C0800209C080020A408002032
:10DAE400A4080020AC080020AC080020B4080020E2
:10DAF400B4080020BC080020BC080020C408002092
:10DB0400C4080020CC080020CC080020D408002041
:10DB1400D4080020DC080020DC080020E4080020F1
:10DB2400E4080020EC080020EC080020F4080020A1
:10DB3400F4080020FC080020FC0800200409002050
:10DB4400040900200C0900200C09002014090020FD
:10DB5400140900201C0900201C09002024090020AD
:10DB6400240900202C0900202C090020340900205D
:10DB7400340900203C0900203C090020440900200D
:10DB8400440900204C0900204C09002054090020BD
:10DB9400540900205C0900205C090020640900206D
:10DBA400640900206C0900206C090020740900201D
:10DBB400740900207C0900207C09002084090020CD
:10DBC400840900208C0900208C090020940900207D
:10DBD400940900209C0900209C090020A40900202D
:10DBE400A4090020AC090020AC090020B4090020DD
:10DBF400B4090020BC090020BC090020C40900208D
:10DC0400C4090020CC090020CC090020D40900203C
:10DC1400D4090020DC090020DC090020E4090020EC
:10DC2400E4090020EC090020EC090020F40900209C
:10DC3400F4090020FC090020FC090020040A00204B
:10DC4400040A00200C0A00200C0A0020140A0020F8
:10DC5400140A00201C0A00201C0A0020240A0020A8
:10DC6400240A00202C0A00202C0A0020340A002058
:10DC7400340A00203C0A00203C0A0020440A002008
:0CDC8400440A0020FFFFFFFF0000020028
:0400000508006A493C
:00000001FF
